 kitl

 Timestamp is 4fb05c83 (Mon May 14 13:14:43 2012)

 Preferred load address is 10000000

 Start         Length     Name                   Class
 0001:00000000 000089c8H .rdata                  CODE
 0001:000089c8 00000021H .rdata$debug            CODE
 0001:000089ec 00029b18H .text                   CODE
 0001:00032504 00000060H .xdata                  CODE
 0001:00032570 00000031H .edata                  CODE
 0002:00000000 00005438H .data                   DATA
 0002:00005440 0004a2b4H .bss                    DATA
 0003:00000000 00000e00H .pdata                  DATA

  Address         Publics by Value              Rva+Base       Lib:Object

 0000:00000000       ___safe_se_handler_table   00000000     <absolute>
 0000:00000000       ___safe_se_handler_count   00000000     <absolute>
 0001:0000001c       ??_C@_1BG@JBMELNEE@?$AAU?$AAS?$AAB?$AA_?$AAS?$AAE?$AAR?$AAI?$AAA?$AAL?$AA?$AA@ 1000101c     kitl.obj
 0001:00000034       ??_C@_1BE@LBNFCPIJ@?$AAC?$AAS?$AAP?$AAS?$AAE?$AAR?$AAI?$AAA?$AAL?$AA?$AA@ 10001034     kitl.obj
 0001:00000048       ??_C@_17KDBLIHPA@?$AAF?$AAE?$AAC?$AA?$AA@ 10001048     kitl.obj
 0001:00000050       ??_C@_1BG@GIAHOCLI@?$AAU?$AAS?$AAB?$AA_?$AAR?$AAN?$AAD?$AAI?$AAS?$AA?5?$AA?$AA@ 10001050     kitl.obj
 0001:000000f8       ??_C@_1FK@FNONLNGN@?$AA?$CF?$AAs?$AA?3?$AA?5?$AAD?$AAE?$AAB?$AAU?$AAG?$AAC?$AAH?$AAK?$AA?5?$AAf?$AAa?$AAi?$AAl?$AAe?$AAd?$AA?5?$AAi?$AAn?$AA?5?$AAf?$AAi?$AAl?$AAe?$AA?5?$AA?$CF?$AAs?$AA?5?$AAa@ 100010f8     kitl.obj
 0001:00000154       ??_C@_1CO@EHGNHHJF@?$AAI?$AAn?$AAv?$AAa?$AAl?$AAi?$AAd?$AA?5?$AAT?$AAi?$AAm?$AAe?$AAr?$AA?5?$AAs?$AAo?$AAu?$AAr?$AAc?$AAe?$AA?$AN?$AA?6?$AA?$AA@ 10001154     kitl.obj
 0001:00000184       ??_C@_1CI@OHCJFJPM@?$AAE?$AAR?$AAR?$AAO?$AAR?$AA?3?$AA?5?$AA?$CF?$AAs?$AA?5?$AAl?$AAi?$AAn?$AAe?$AA?5?$AA?$CF?$AAd?$AA?3?$AA?5?$AA?$AA@ 10001184     kitl.obj
 0001:000001b0       ??_C@_1HM@JFDFJIPB@?$AAC?$AA?3?$AA?2?$AAW?$AAI?$AAN?$AAC?$AAE?$AAR?$AAO?$AAO?$AAT?$AAS?$AA?2?$AAT?$AAo?$AAp?$AAa?$AAz?$AA?2?$AAW?$AAI?$AAN?$AAC?$AAE?$AA6?$AA0?$AA0?$AA?2?$AAP?$AAL?$AAA@ 100011b0     kitl.obj
 0001:0000022c       ??_C@_0BL@HDGIOPOJ@?9OEMKitlStartup?$CIrc?5?$DN?5?$CFd?$CJ?$AN?6?$AA@ 1000122c     kitl.obj
 0001:00000248       ??_C@_0DG@PJLKPGLN@KITL?3?5Increasing?5KITL?5thread?5pri@ 10001248     kitl.obj
 0001:00000280       ??_C@_05DFLKGENG@Topaz?$AA@ 10001280     kitl.obj
 0001:00000288       ??_C@_0CP@HIPALHGN@WARN?3?5Boot?5arguments?5not?5found?0?5@ 10001288     kitl.obj
 0001:000002b8       ??_C@_0CG@DGCHFGBG@?$CLOEMKitlStartup?3?5EPIT?5null?5point@ 100012b8     kitl.obj
 0001:000002e0       ??_C@_0BC@JLFFBIBG@?$CLOEMKitlStartup?$AN?6?$AA@ 100012e0     kitl.obj
 0001:000002f4       ??_C@_0CA@PHILFGNL@Changed?5KITL?5zone?5mask?5to?50x?$CFX?6?$AA@ 100012f4     kitlcore:ethdbg.obj
 0001:00000314       ??_C@_0CP@OKNACMFC@KITL?3?5DEBUGCHK?5failed?5in?5file?5?$CFs@ 10001314     kitlcore:ethdbg.obj
 0001:00000344       ??_C@_0DF@HLOKAGOO@d?3?2yzkiqfe?2private?2winceos?2COREO@ 10001344     kitlcore:ethdbg.obj
 0001:0000037c       ??_C@_0DC@LLJMBDFH@?$CBKITLRegisterDfltClient?3?5Fail?5to@ 1000137c     kitlcore:ethdbg.obj
 0001:000003b0       ??_C@_0CF@PIAHHHCH@?$CLKITLRegisterDfltClient?0?5service@ 100013b0     kitlcore:ethdbg.obj
 0001:000003d8       ??_C@_0EE@LCCLDMNC@?9KITLRegisterClient?$CI?$CFs?$CJ?3?5Flags?3?5@ 100013d8     kitlcore:ethdbg.obj
 0001:00000420       ??_C@_1JC@DNGAJENF@?$AAK?$AAI?$AAT?$AAL?$AAR?$AAe?$AAg?$AAi?$AAs?$AAt?$AAe?$AAr?$AAC?$AAl?$AAi?$AAe?$AAn?$AAt?$AA?3?$AA?5?$AAp?$AAB?$AAu?$AAf?$AAf?$AAe?$AAr?$AAP?$AAo?$AAo?$AAl?$AA?5@ 10001420     kitlcore:ethdbg.obj
 0001:000004b8       ??_C@_0EE@DHNHGKFP@?$CLKITLRegisterClient?$CI?$CFs?$CJ?3?5Flags?3?5@ 100014b8     kitlcore:ethdbg.obj
 0001:000004fc       ??_C@_0DN@GDEGDLCL@?$CBKITLRegisterClient?$CI?$CFs?$CJ?3?5Client?5@ 100014fc     kitlcore:ethdbg.obj
 0001:0000053c       ??_C@_0DG@FHPIAJCD@?$CBKITLRegisterClient?$CI?$CFs?$CJ?3?5No?5avai@ 1000153c     kitlcore:ethdbg.obj
 0001:00000574       ??_C@_0CP@LFECMIMJ@?$CBDoRegisterClient?$CI?$CFs?$CJ?3?5Invalid?5w@ 10001574     kitlcore:ethdbg.obj
 0001:000005a4       ??_C@_0DO@NHOEDOMO@?$CBDoRegisterClient?$CI?$CFs?$CJ?3?5Need?5to?5s@ 100015a4     kitlcore:ethdbg.obj
 0001:000005e4       ??_C@_0CK@GNMBECNI@?$CBDoRegisterClient?$CI?$CFs?$CJ?3?5Invalid?5p@ 100015e4     kitlcore:ethdbg.obj
 0001:00000610       ??_C@_04HIBGFPH@NULL?$AA@  10001610     kitlcore:ethdbg.obj
 0001:00000618       ??_C@_0CB@GAEKFKGC@?9RegisterClientPart2?5returns?5?$CFd?6@ 10001618     kitlcore:ethdbg.obj
 0001:0000063c       ??_C@_0CA@NGKEKANM@Closing?5Handle?5of?5Timer?5Thread?6?$AA@ 1000163c     kitlcore:ethdbg.obj
 0001:0000065c       ??_C@_0BN@FPKBKHBK@Error?5creating?5timer?5thread?6?$AA@ 1000165c     kitlcore:ethdbg.obj
 0001:0000067c       ??_C@_0BP@CEIGPPLL@?$CLRegisterClientPart2?3?5Id?50x?$CFX?6?$AA@ 1000167c     kitlcore:ethdbg.obj
 0001:0000069c       ??_C@_0CF@HHGPCOPG@?9KITLDeregisterClient?0?5Id?3?$CFu?5ret@ 1000169c     kitlcore:ethdbg.obj
 0001:000006c4       ??_C@_0CP@KBFNKJIP@KITLDeregisterClient?$FL?$CFu?$FN?9already@ 100016c4     kitlcore:ethdbg.obj
 0001:000006f4       ??_C@_0CG@LJKJDKF@KITLDeregisterClient?3?5invalid?5ID@ 100016f4     kitlcore:ethdbg.obj
 0001:0000071c       ??_C@_0BO@GDFIOKBN@?$CLKITLDeregisterClient?0?5Id?3?$CFu?6?$AA@ 1000171c     kitlcore:ethdbg.obj
 0001:0000073c       ??_C@_0CB@GFDDAGEF@Error?5creating?5interrupt?5thread?6@ 1000173c     kitlcore:ethdbg.obj
 0001:00000760       ??_C@_0BD@OAGEIDKN@KITL?5Creating?5IST?6?$AA@ 10001760     kitlcore:ethdbg.obj
 0001:00000774       ??_C@_0CE@DNEFLEAI@KITL?5Checking?5client?5registratio@ 10001774     kitlcore:ethdbg.obj
 0001:00000798       ??_C@_0CE@FKCJJLLC@KITL?3?5Leaving?5polling?5mode?4?4?4?50x@ 10001798     kitlcore:ethdbg.obj
 0001:000007bc       ??_C@_0DH@MFOCECCL@?$AN?6?$CBUnable?5to?5establish?5KITL?5conn@ 100017bc     kitlcore:ethdbg.obj
 0001:000007f4       ??_C@_0DN@NDJFLFHF@?$AN?6?$CBKitl?5buffer?5specified?5by?5OAL?5@ 100017f4     kitlcore:ethdbg.obj
 0001:00000834       ??_C@_0BI@OFAMBHJH@Connecting?5to?5Desktop?$AN?6?$AA@ 10001834     kitlcore:ethdbg.obj
 0001:0000084c       ??_C@_0CF@GGNNPHKD@Connecting?5to?5Desktop?5?4?4?5resendi@ 1000184c     kitlcore:ethdbg.obj
 0001:00000874       ??_C@_04MOKOCOLM@KDBG?$AA@ 10001874     kitlcore:ethdbg.obj
 0001:0000087c       ??_C@_04JMJJJNGP@PPSH?$AA@ 1000187c     kitlcore:ethdbg.obj
 0001:00000884       ??_C@_06MCCIJHBO@DBGMSG?$AA@ 10001884     kitlcore:ethdbg.obj
 0001:0000088c       ??_C@_0BK@OPBJDOAA@Enabling?5adapter?5ints?4?4?4?6?$AA@ 1000188c     kitlcore:ethdbg.obj
 0001:000008a8       ??_C@_0EO@CEOOKDBM@?$CBKITL?5Interrupt?5thread?5got?5error@ 100018a8     kitlcore:ethdbg.obj
 0001:000008f8       ??_C@_0BL@PLNAMGGN@Processed?5Interrupt?5event?6?$AA@ 100018f8     kitlcore:ethdbg.obj
 0001:00000914       ??_C@_0BG@IBEGMBIN@KITL?5Interrupt?5event?6?$AA@ 10001914     kitlcore:ethdbg.obj
 0001:0000092c       ??_C@_1BA@LEPJIIOK@?$AAU?$AAn?$AAk?$AAn?$AAo?$AAw?$AAn?$AA?$AA@ 1000192c     kitlcore:ethdbg.obj
 0001:00000940       ??_C@_1GK@HKJDDLOJ@?$AAd?$AA?3?$AA?2?$AAy?$AAz?$AAk?$AAi?$AAq?$AAf?$AAe?$AA?2?$AAp?$AAr?$AAi?$AAv?$AAa?$AAt?$AAe?$AA?2?$AAw?$AAi?$AAn?$AAc?$AAe?$AAo?$AAs?$AA?2?$AAC?$AAO?$AAR?$AAE?$AAO@ 10001940     kitlcore:ethdbg.obj
 0001:000009ac       ??_C@_0CB@PCGPHMPD@KITL?5InterruptInitialize?5failed?6@ 100019ac     kitlcore:ethdbg.obj
 0001:000009d0       ??_C@_0BK@HDMNDFBA@KITL?5CreateEvent?5failed?$CB?6?$AA@ 100019d0     kitlcore:ethdbg.obj
 0001:000009ec       ??_C@_1BK@PPDMEPMD@?$AAE?$AAd?$AAb?$AAg?$AAI?$AAn?$AAt?$AAE?$AAv?$AAe?$AAn?$AAt?$AA?$AA@ 100019ec     kitlcore:ethdbg.obj
 0001:00000a08       ??_C@_0EI@HCIGFCPA@KITL?5Interrupt?5thread?5started?5?$CIh@ 10001a08     kitlcore:ethdbg.obj
 0001:00000a50       ??_C@_0M@CDHNGIPM@?$CFu?4?$CFu?4?$CFu?4?$CFu?$AA@ 10001a50     kitlcore:debug.obj
 0001:00000a5c       ??_C@_0DA@KOJGDENJ@?$CBExchangeConfig?3?5WaitForMultiple@ 10001a5c     kitlcore:edbgprot.obj
 0001:00000a8c       ??_C@_0DL@JCMIMDFC@Waiting?5for?5service?5?8?$CFs?8?5to?5conn@ 10001a8c     kitlcore:edbgprot.obj
 0001:00000ac8       ??_C@_0CF@ELFKFCIB@?$CBSendConfig?3?5Error?5in?5KitlSendFr@ 10001ac8     kitlcore:edbgprot.obj
 0001:00000af0       ??_C@_0N@DPCKIDMJ@?$DO?$DOSendConfig?$AA@ 10001af0     kitlcore:edbgprot.obj
 0001:00000b00       ??_C@_0BO@OHFCENNA@?$CBSendConfig?3?5Stack?5overflow?$AN?6?$AA@ 10001b00     kitlcore:edbgprot.obj
 0001:00000b20       ??_C@_0CB@MCDILJMK@?$CBKITLPollData?3?5STACK?5OVERFLOW?$CB?$AN?6@ 10001b20     kitlcore:edbgprot.obj
 0001:00000b44       ??_C@_0BE@LJGMDJBF@?9Send?5?$CI?$CFu?$CJ?3?5Ret?5?$CFu?6?$AA@ 10001b44     kitlcore:edbgprot.obj
 0001:00000b58       ??_C@_0EJ@GPALBKID@KITLSend?3?5Id?3?5?$CFu?5Timed?5out?5waiti@ 10001b58     kitlcore:edbgprot.obj
 0001:00000ba4       ??_C@_0CD@CLDOKAPO@?$CBKITLSend?3?5Error?5in?5KitlSendFram@ 10001ba4     kitlcore:edbgprot.obj
 0001:00000bc8       ??_C@_0L@GNNICFIO@?$DO?$DOKITLSend?$AA@ 10001bc8     kitlcore:edbgprot.obj
 0001:00000bd4       ??_C@_0DC@NFAJIDMM@KITLSend?$CI?$CFu?$CJ?3?5Client?5de?9register@ 10001bd4     kitlcore:edbgprot.obj
 0001:00000c08       ??_C@_0FD@BAMAHPPH@0x?$CFx?5?$CI0x?$CFx?$CJ?3?5KITLSend?$CI?$CFu?$CJ?3?5Timed@ 10001c08     kitlcore:edbgprot.obj
 0001:00000c5c       ??_C@_0DP@NKADLCEM@KITLSend?$CI?$CFu?$CJ?3?5Tx?5window?5full?5?$CIAc@ 10001c5c     kitlcore:edbgprot.obj
 0001:00000c9c       ??_C@_0DJ@CHBCIFD@?$CLKITLSend?$CI?$CFu?$CJ?0?5Len?3?5?$CFu?0?5Seq?3?5?$CFu?0@ 10001c9c     kitlcore:edbgprot.obj
 0001:00000cd8       ??_C@_0DI@DLCMJFKN@?$CBKITLSend?$CI?$CFu?$CJ?3?5KITL_USE_SYSCALLS@ 10001cd8     kitlcore:edbgprot.obj
 0001:00000d10       ??_C@_02DKCKIIND@?$CFs?$AA@ 10001d10     kitlcore:edbgprot.obj
 0001:00000d14       ??_C@_0DP@FELNBMKM@?$CBKITLSend?$CI?$CFu?$CJ?3?5In?5syscall?5with?5C@ 10001d14     kitlcore:edbgprot.obj
 0001:00000d54       ??_C@_0DI@BNMJMCKD@KITLSend?$CI?$CFu?$CJ?3?5InSysCall?5or?5InPow@ 10001d54     kitlcore:edbgprot.obj
 0001:00000d8c       ??_C@_03OFAPEBGM@?$CFs?6?$AA@ 10001d8c     kitlcore:edbgprot.obj
 0001:00000d90       ??_C@_0DD@OOGFOEID@?$CBKITLSend?$CIDBGMSG?$CJ?3?5Reentrant?5cal@ 10001d90     kitlcore:edbgprot.obj
 0001:00000dc4       ??_C@_0DK@DPCAMIHE@?$CBKITLSend?3?5Data?5to?5be?5send?5overl@ 10001dc4     kitlcore:edbgprot.obj
 0001:00000e00       ??_C@_0BN@OHMKNAC@?$CBKITLSend?3?5Buffer?5too?5large?6?$AA@ 10001e00     kitlcore:edbgprot.obj
 0001:00000e20       ??_C@_0CM@CLKKFLBC@?$CBRetransmitFrame?3?5Error?5in?5KitlS@ 10001e20     kitlcore:edbgprot.obj
 0001:00000e4c       ??_C@_0DK@IEKHHEOI@RetransmitFrame?$CIId?3?$CFu?$CJ?0?5Seq?3?5?$CFu?0@ 10001e4c     kitlcore:edbgprot.obj
 0001:00000e88       ??_C@_0N@MAHOMCPK@?$DO?$DORetransmit?$AA@ 10001e88     kitlcore:edbgprot.obj
 0001:00000e98       ??_C@_0DJ@FKGIBMLE@?$CBRetransmitFrame?3?5Frame?5seq?5?$CFu?5n@ 10001e98     kitlcore:edbgprot.obj
 0001:00000ed4       ??_C@_0DH@PPIJALHK@?9KITLRecv?$CI?$CFu?$CJ?3?5Read?5?$CFu?5bytes?5fro@ 10001ed4     kitlcore:edbgprot.obj
 0001:00000f0c       ??_C@_0DO@DJKEMME@KITL?$CI?$CFu?$CJ?3?5Client?5de?9registered?5w@ 10001f0c     kitlcore:edbgprot.obj
 0001:00000f4c       ??_C@_0CL@BNPAPIIB@KITL?$CI?$CFu?$CJ?3?5Timed?5out?5waiting?5for?5@ 10001f4c     kitlcore:edbgprot.obj
 0001:00000f78       ??_C@_0CL@FAMFOGBN@KITL?$CI?$CFu?$CJ?3?5Timed?5out?5polling?5for?5@ 10001f78     kitlcore:edbgprot.obj
 0001:00000fa8       ??_C@_0EN@PICLEEHD@?$CLKITLRecv?$CI?$CFu?$CJ?3?5Waiting?5for?5messa@ 10001fa8     kitlcore:edbgprot.obj
 0001:00000ff8       ??_C@_0CP@HOJLGBBA@?$CBKITLRecv?$CI?$CFu?$CJ?3?5SYSCALLS?5for?5clie@ 10001ff8     kitlcore:edbgprot.obj
 0001:00001028       ??_C@_0CO@HBIBEOCJ@?$CBKITLRecv?$CI?$CFu?$CJ?3?5In?5syscall?5with?5C@ 10002028     kitlcore:edbgprot.obj
 0001:00001058       ??_C@_0BL@EKCNDGH@KITLRecv?$CI?$CFu?$CJ?3?5InSysCall?$CI?$CJ?6?$AA@ 10002058     kitlcore:edbgprot.obj
 0001:00001074       ??_C@_0DJ@KKFBBHCF@?$CBKITLRecv?3?5Receive?5buffer?5overla@ 10002074     kitlcore:edbgprot.obj
 0001:000010b0       ??_C@_0CL@OPFPPJCH@?$AN?6?$CBKITLRecv?3?5Client?5?$CI?$CFd?$CJ?5not?5reg@ 100020b0     kitlcore:edbgprot.obj
 0001:000010dc       ??_C@_0CJ@KPACHCHO@?$AN?6?$CBKITLRecv?3?5Invalid?5client?5ID?5?$CF@ 100020dc     kitlcore:edbgprot.obj
 0001:00001108       ??_C@_0CH@PDOCBOKH@?$CBKITL?3?5Error?5in?5KitlSendFrame?5fo@ 10002108     kitlcore:edbgprot.obj
 0001:00001130       ??_C@_0P@MAADMIHH@?$DO?$DOSendAckNack?5?$AA@ 10002130     kitlcore:edbgprot.obj
 0001:00001140       ??_C@_0BP@EJOKEGGJ@?$CBSendAckNack?3?5Stack?5overflow?$AN?6?$AA@ 10002140     kitlcore:edbgprot.obj
 0001:00001160       ??_C@_0CA@NAACODDG@Rx?5win?3?5?$CFu?0?$CFu?0?5usesyscalls?3?5?$CFu?6?$AA@ 10002160     kitlcore:edbgprot.obj
 0001:00001180       ??_C@_0CN@BBCENBHL@?$CBKITL?3?5Received?5data?5message?5wit@ 10002180     kitlcore:edbgprot.obj
 0001:000011b0       ??_C@_0DA@OPFEGEEE@?$CBKITL?$CI?$CFu?$CJ?3?5Dropped?5frame?5?$CIseq?3?5?$CF@ 100021b0     kitlcore:edbgprot.obj
 0001:000011e0       ??_C@_0DP@JICFCGAN@KITL?$CI?$CFu?$CJ?3?5Received?5frame?5Seq?3?5?$CFu@ 100021e0     kitlcore:edbgprot.obj
 0001:00001220       ??_C@_0DE@NDJGOJN@KITL?$CI?$CFu?$CJ?3?5Tossing?5frame?5?$CFu?5?$CICan?8@ 10002220     kitlcore:edbgprot.obj
 0001:00001258       ??_C@_0EJ@IGCHOLJ@KITL?$CI?$CFu?$CJ?3?5Received?5duplicate?5?$CISe@ 10002258     kitlcore:edbgprot.obj
 0001:000012a4       ??_C@_0CK@NCOCPCB@KITL?$CI?$CFu?$CJ?3?5Lost?5ACK?5?$CIseq?3?5?$CFu?0?5win@ 100022a4     kitlcore:edbgprot.obj
 0001:000012d0       ??_C@_0DK@KIPJLMPC@KITL?$CI?$CFu?$CJ?3?5Received?5msg?5outside?5w@ 100022d0     kitlcore:edbgprot.obj
 0001:00001310       ??_C@_0EH@GEPCHLAC@?$CBKITL?$CI?$CFu?$CJ?3?5Received?5NACK?5outside@ 10002310     kitlcore:edbgprot.obj
 0001:00001358       ??_C@_0DC@DOOEJJGK@?$CBKITL?$CI?$CFu?$CJ?3?5NACK?5in?5window?0?5but?5T@ 10002358     kitlcore:edbgprot.obj
 0001:0000138c       ??_C@_0DG@NIAKHBIH@KITL?$CI?$CFu?$CJ?3?5Received?5NACK?5for?5msg?5@ 1000238c     kitlcore:edbgprot.obj
 0001:000013c4       ??_C@_0DF@IFNFDEOL@KITL?$CI?$CFu?$CJ?3?5Received?5ack?5for?5msg?5?$CF@ 100023c4     kitlcore:edbgprot.obj
 0001:000013fc       ??_C@_0CJ@CFLKBFAK@?$CBKITL?$CI?$CFu?$CJ?5tossing?5msg?5?$CFu?5?$CICan?8t?5@ 100023fc     kitlcore:edbgprot.obj
 0001:00001428       ??_C@_0EL@IBLAMFGF@?$CBProcessKITLMsg?3?5Mismatch?5in?5ser@ 10002428     kitlcore:edbgprot.obj
 0001:00001474       ??_C@_0CL@FHFBAKPK@?$CBProcessKITLMsg?3?5Client?5?$CFu?5not?5r@ 10002474     kitlcore:edbgprot.obj
 0001:000014a0       ??_C@_0CI@KKKLHIBN@?$CBProcessKITLMsg?3?5Invalid?5Service@ 100024a0     kitlcore:edbgprot.obj
 0001:000014c8       ??_C@_0L@HMANIGEC@?$DM?$DMKITLRecv?$AA@ 100024c8     kitlcore:edbgprot.obj
 0001:000014d4       ??_C@_0BJ@GGJGBCL@KITL?3?5Invalid?5length?5?$CFu?6?$AA@ 100024d4     kitlcore:edbgprot.obj
 0001:000014f0       ??_C@_0CA@IJGFJJIG@KITL?3?5Got?5unrecognized?5Id?3?5?$CFX?$AN?6?$AA@ 100024f0     kitlcore:edbgprot.obj
 0001:00001510       ??_C@_0CM@PPFMALGC@ProcessRecvFrame?3?5Received?5Unhan@ 10002510     kitlcore:edbgprot.obj
 0001:0000153c       ??_C@_0CK@HJLKKHDE@?$CBProcessAdminMsg?3?5Unhandled?5comm@ 1000253c     kitlcore:edbgprot.obj
 0001:00001568       ??_C@_0BE@JFHHMBPA@?5KeyIndex?5?$CFd?5?$DN?5?$CFd?5?6?$AA@ 10002568     kitlcore:edbgprot.obj
 0001:0000157c       ??_C@_0CM@CCHLHCID@?$CBHost?5config?5message?5size?5mismat@ 1000257c     kitlcore:edbgprot.obj
 0001:000015a8       ??_C@_0DH@FAHMLBID@KITL?3?5IOCTL_HAL_REBOOT?5not?5suppo@ 100025a8     kitlcore:edbgprot.obj
 0001:000015e0       ??_C@_0BJ@HLKLCDLN@KITL?3?5Got?5RESET?5command?6?$AA@ 100025e0     kitlcore:edbgprot.obj
 0001:000015fc       ??_C@_0DI@OCIAAPLH@ProcessAdminMsg?3?5Receive?5Config?5@ 100025fc     kitlcore:edbgprot.obj
 0001:00001634       ??_C@_0CO@OMAAFIHE@?$CBReceived?5config?5for?5unrecognize@ 10002634     kitlcore:edbgprot.obj
 0001:00001664       ??_C@_0DF@JFLDKAPD@?$CBProcessAdminMsg?3?5Invalid?5legnth@ 10002664     kitlcore:edbgprot.obj
 0001:0000169c       ??_C@_0P@LGFIPJFJ@?0?5DataLen?3?5?$CFu?6?$AA@ 1000269c     kitlcore:edbgprot.obj
 0001:000016ac       ??_C@_01PKGAHCOL@?$CJ?$AA@ 100026ac     kitlcore:edbgprot.obj
 0001:000016b0       ??_C@_04MFNBCIME@DEV?5?$AA@ 100026b0     kitlcore:edbgprot.obj
 0001:000016b8       ??_C@_05HOBGPFOJ@NACK?5?$AA@ 100026b8     kitlcore:edbgprot.obj
 0001:000016c0       ??_C@_04DMKEMIEL@ACK?5?$AA@ 100026c0     kitlcore:edbgprot.obj
 0001:000016c8       ??_C@_01ODHLEDKK@?$CI?$AA@ 100026c8     kitlcore:edbgprot.obj
 0001:000016cc       ??_C@_0BM@DFJEJNKL@?5?5Seq?3?$CFu?$CI0x?$CFX?$CJ?0?5Flags?30x?$CFX?5?$AA@ 100026cc     kitlcore:edbgprot.obj
 0001:000016e8       ??_C@_09CODJGAOM@?5Svc?30x?$CFX?$AA@ 100026e8     kitlcore:edbgprot.obj
 0001:000016f4       ??_C@_0BI@HBHDLBHB@Unrecognized?5cmd?3?50x?$CFX?5?$AA@ 100026f4     kitlcore:edbgprot.obj
 0001:0000170c       ??_C@_0BO@FKGFLAJH@TRANSPORT?5CONFIG?0?5flag?5?$DN?50x?$CFx?$AA@ 1000270c     kitlcore:edbgprot.obj
 0001:0000172c       ??_C@_0M@NMHJJIOD@RETRANSMIT?5?$AA@ 1000272c     kitlcore:edbgprot.obj
 0001:00001738       ??_C@_0CK@EGCFFJGL@DESK?5?$CFs?0?5ProtoVer?3?$CFu?0?5Service?3?5?$CF@ 10002738     kitlcore:edbgprot.obj
 0001:00001764       ??_C@_0DO@HJLCOKEN@DEV?5?$CFs?0?5ProtoVer?3?$CFu?0?5Service?3?5?$CFs@ 10002764     kitlcore:edbgprot.obj
 0001:000017a4       ??_C@_03LLENEDKC@CMD?$AA@  100027a4     kitlcore:edbgprot.obj
 0001:000017a8       ??_C@_04DIFPBPL@RESP?$AA@  100027a8     kitlcore:edbgprot.obj
 0001:000017b0       ??_C@_03JMDFPPIA@CFG?$AA@  100027b0     kitlcore:edbgprot.obj
 0001:000017b4       ??_C@_06KEAEPMBK@RESET?5?$AA@ 100027b4     kitlcore:edbgprot.obj
 0001:000017bc       ??_C@_08LKBCIGBL@JUMPIMG?5?$AA@ 100027bc     kitlcore:edbgprot.obj
 0001:000017c8       ??_C@_07PKBANKEN@BOOTME?5?$AA@ 100027c8     kitlcore:edbgprot.obj
 0001:000017d0       ??_C@_07LMOBHLFA@?5ADMIN?5?$AA@ 100027d0     kitlcore:edbgprot.obj
 0001:000017d8       ??_C@_06LEIODCGK@?5KDBG?5?$AA@ 100027d8     kitlcore:edbgprot.obj
 0001:000017e0       ??_C@_06KLAGIGLH@?5PPSH?5?$AA@ 100027e0     kitlcore:edbgprot.obj
 0001:000017e8       ??_C@_08GOJDHIDC@?5DBGMSG?5?$AA@ 100027e8     kitlcore:edbgprot.obj
 0001:000017f4       ??_C@_0DM@HHCOAHOB@?$CBKitlSendFrame?3?5transport?5failed@ 100027f4     kitlcore:edbgprot.obj
 0001:00001830       ??_C@_0BP@FOBICGNC@TimerEnt?3?5slot?5?$CFu?0?5expire?3?5?$CFu?6?$AA@ 10002830     kitlcore:timer.obj
 0001:00001850       ??_C@_0DE@DOKGNEAI@d?3?2yzkiqfe?2private?2winceos?2COREO@ 10002850     kitlcore:timer.obj
 0001:00001884       ??_C@_0DD@GEBJPFDB@KITL?5Timer?5thread?5started?0?5?$CIhTh?3@ 10002884     kitlcore:timer.obj
 0001:000018b8       ??_C@_0DC@FKEAIDLA@Timer?3?5Inserted?5entry?50x?$CFX?0?5slot@ 100028b8     kitlcore:timer.obj
 0001:000018ec       ??_C@_0CE@HDEHCBNJ@KITL?5Error?5allocating?5timer?5memo@ 100028ec     kitlcore:timer.obj
 0001:00001910       ??_C@_0CL@NCIDHHCH@?$CBTimerStop?3?5Timer?5not?5started?5fo@ 10002910     kitlcore:timer.obj
 0001:0000193c       ??_C@_0CN@NMGOCIEE@Timer?3?5Removing?5entry?0?5slot?3?5?$CFu?0@ 1000293c     kitlcore:timer.obj
 0001:0000196c       ??_C@_0BM@CKNAHOAO@?$CLCancelTimersForClient?$CI?$CFs?$CJ?6?$AA@ 1000296c     kitlcore:timer.obj
 0001:00001988       ??_C@_1CC@FONLHMJH@?$AAH?$AAa?$AAl?$AAt?$AAi?$AAn?$AAg?$AA?5?$AAs?$AAy?$AAs?$AAt?$AAe?$AAm?$AA?$AN?$AA?6?$AA?$AA@ 10002988     oemstub:oemstub.obj
 0001:000019b0       ??_C@_1HC@KKBKCDL@?$AAd?$AA?3?$AA?2?$AAy?$AAz?$AAk?$AAi?$AAq?$AAf?$AAe?$AA?2?$AAp?$AAr?$AAi?$AAv?$AAa?$AAt?$AAe?$AA?2?$AAw?$AAi?$AAn?$AAc?$AAe?$AAo?$AAs?$AA?2?$AAC?$AAO?$AAR?$AAE?$AAO@ 100029b0     oemstub:oemstub.obj
 0001:00001a28       ??_C@_1FM@EIKOCJDA@?$AA?$CB?$AA?$CB?$AA?5?$AAP?$AAr?$AAo?$AAf?$AAi?$AAl?$AAi?$AAn?$AAg?$AA?5?$AAi?$AAs?$AA?5?$AAn?$AAo?$AAt?$AA?5?$AAi?$AAm?$AAp?$AAl?$AAe?$AAm?$AAe?$AAn?$AAt?$AAe?$AAd?$AA?5@ 10002a28     oemstub:oemstub.obj
 0001:00001b18       ??_C@_0BI@GBPEIAJI@?9OEMKitlInit?$CIrc?5?$DN?5?$CFd?$CJ?$AN?6?$AA@ 10002b18     oal_kitl:kitl.obj
 0001:00001b30       ??_C@_0BH@DJPAMHLI@?$CLOEMKitlInit?$CI0x?$CF08x?$CJ?$AN?6?$AA@ 10002b30     oal_kitl:kitl.obj
 0001:00001b48       ??_C@_0BI@KCIPJAAG@?9OALKitlInit?$CIrc?5?$DN?5?$CFd?$CJ?$AN?6?$AA@ 10002b48     oal_kitl:kitl.obj
 0001:00001b60       ??_C@_0CG@NCCHEHBN@ERROR?3?5OALKitlInit?3?5KitlInit?5fai@ 10002b60     oal_kitl:kitl.obj
 0001:00001b88       ??_C@_0FG@GMOHKIKA@ERROR?3?5OALKitlInit?3?5No?5supported@ 10002b88     oal_kitl:kitl.obj
 0001:00001be0       ??_C@_0CD@KFHIJAFP@WARN?3?5OALKitlInit?3?5KITL?5Disabled@ 10002be0     oal_kitl:kitl.obj
 0001:00001c04       ??_C@_0CB@ICNOHDED@pDevice?9?$DOpDriver?4?4?4?4?4?4?4?4?4?50x?$CFx?$AN?6@ 10002c04     oal_kitl:kitl.obj
 0001:00001c28       ??_C@_0BP@LAJLJKFE@pDevice?9?$DOtype?4?4?4?4?4?4?4?4?4?4?4?4?5?$CFd?$AN?6?$AA@ 10002c28     oal_kitl:kitl.obj
 0001:00001c48       ??_C@_0BP@OJPECLKF@pDevice?9?$DOresource?4?4?4?4?4?4?4?4?5?$CFd?$AN?6?$AA@ 10002c48     oal_kitl:kitl.obj
 0001:00001c68       ??_C@_0CB@JAOILBKH@pDevice?9?$DOid?4?4?4?4?4?4?4?4?4?4?4?4?4?4?50x?$CFx?$AN?6@ 10002c68     oal_kitl:kitl.obj
 0001:00001c8c       ??_C@_0BP@ELIKEIPK@pDevice?9?$DOifcType?4?4?4?4?4?4?4?4?4?5?$CFd?$AN?6?$AA@ 10002c8c     oal_kitl:kitl.obj
 0001:00001cac       ??_C@_0CA@MADPCADD@pDevice?9?$DOName?4?4?4?4?4?4?4?4?4?4?4?4?5?$CFhs?$AN?6?$AA@ 10002cac     oal_kitl:kitl.obj
 0001:00001ccc       ??_C@_0BP@GCIAPLEP@pArgs?9?$DOip4address?4?4?4?4?4?4?4?4?5?$CFs?$AN?6?$AA@ 10002ccc     oal_kitl:kitl.obj
 0001:00001cec       ??_C@_0BP@EDAFLEND@pArgs?9?$DOdevLoc?4Pin?4?4?4?4?4?4?4?4?5?$CFd?$AN?6?$AA@ 10002cec     oal_kitl:kitl.obj
 0001:00001d0c       ??_C@_0CB@ELNIEECP@pArgs?9?$DOdevLoc?4PhysicalLoc?50x?$CFx?$AN?6@ 10002d0c     oal_kitl:kitl.obj
 0001:00001d30       ??_C@_0CB@OOHPGPEK@pArgs?9?$DOdevLoc?4LogicalLoc?4?50x?$CFx?$AN?6@ 10002d30     oal_kitl:kitl.obj
 0001:00001d54       ??_C@_0BP@CLIEPDAL@pArgs?9?$DOdevLoc?4IfcType?4?4?4?4?5?$CFd?$AN?6?$AA@ 10002d54     oal_kitl:kitl.obj
 0001:00001d74       ??_C@_0CB@LJCIEGGC@pArgs?9?$DOflags?4?4?4?4?4?4?4?4?4?4?4?4?4?50x?$CFx?$AN?6@ 10002d74     oal_kitl:kitl.obj
 0001:00001d98       ??_C@_0BP@HJJCJHBD@DeviceId?4?4?4?4?4?4?4?4?4?4?4?4?4?4?4?4?4?5?$CFs?$AN?6?$AA@ 10002d98     oal_kitl:kitl.obj
 0001:00001db8       ??_C@_0DF@BBIFGKFF@?$CLOALKitlInit?$CI?8?$CFhs?8?0?50x?$CF08x?5?9?5?$CFd?1@ 10002db8     oal_kitl:kitl.obj
 0001:00001df0       ??_C@_0BD@GBONLPAN@?9OALKitlPowerOff?$AN?6?$AA@ 10002df0     oal_kitl:kitl.obj
 0001:00001e04       ??_C@_0BD@PMDBLEBO@?$CLOALKitlPowerOff?$AN?6?$AA@ 10002e04     oal_kitl:kitl.obj
 0001:00001e18       ??_C@_0BC@KIOCKNCJ@?9OALKitlPowerOn?$AN?6?$AA@ 10002e18     oal_kitl:kitl.obj
 0001:00001e2c       ??_C@_0BC@KGJOBBKM@?$CLOALKitlPowerOn?$AN?6?$AA@ 10002e2c     oal_kitl:kitl.obj
 0001:00001ed0       ??_C@_0CG@IHIMJOIA@?9OALKitlCreateName?$CIpBuffer?5?$DN?5?8?$CFh@ 10002ed0     oal_kitl:name.obj
 0001:00001ef8       ??_C@_0CM@BCMDHFLI@?$CLOALKitlCreateName?$CI?8?$CFhs?8?0?50x?$CF04x@ 10002ef8     oal_kitl:name.obj
 0001:00001fbc       ??_C@_0BO@KPIGKMGK@?9OALKitlSerialInit?$CIrc?5?$DN?5?$CFd?$CJ?$AN?6?$AA@ 10002fbc     oal_kitl:kitlserial.obj
 0001:00001fdc       ??_C@_0CG@IJDAEBCE@WARN?3?5KITL?5will?5run?5in?5polling?5m@ 10002fdc     oal_kitl:kitlserial.obj
 0001:00002004       ??_C@_0CN@MENCFIED@WARN?3?5KITL?5can?8t?5obtain?5SYSINTR?5@ 10003004     oal_kitl:kitlserial.obj
 0001:00002034       ??_C@_0CO@BPFMIJNH@WARN?3?5KITL?5can?8t?5obtain?5IRQ?5for?5@ 10003034     oal_kitl:kitlserial.obj
 0001:00002064       ??_C@_0CF@GMMNDEHJ@ERROR?3?5KITL?5call?5to?5pfnInit?5fail@ 10003064     oal_kitl:kitlserial.obj
 0001:0000208c       ??_C@_0CE@LGCGCDLA@ERROR?3?5KITL?5device?5driver?5is?5NUL@ 1000308c     oal_kitl:kitlserial.obj
 0001:000020b0       ??_C@_0DB@NNJFABKG@?$CLOALKitlSerialInit?$CI?8?$CFS?8?0?5?8?$CFs?8?0?50@ 100030b0     oal_kitl:kitlserial.obj
 0001:000020e4       ??_C@_0BG@PDHAIEPB@?9SerialSend?$CIrc?5?$DN?51?$CJ?$AN?6?$AA@ 100030e4     oal_kitl:kitlserial.obj
 0001:000020fc       ??_C@_0BK@FJBKAKDG@?$CLSerialSend?$CI0x?$CF08x?0?5?$CFd?$CJ?$AN?6?$AA@ 100030fc     oal_kitl:kitlserial.obj
 0001:00002118       ??_C@_0BN@FOGKPFOM@?9SerialRecv?$CI?$CKpLength?5?$DN?5?$CFd?$CJ?$AN?6?$AA@ 10003118     oal_kitl:kitlserial.obj
 0001:00002138       ??_C@_0DN@FPKOAPOO@ERROR?3?5SerialRecv?3?5Received?5pack@ 10003138     oal_kitl:kitlserial.obj
 0001:00002178       ??_C@_0DI@FBKFFAPI@WARN?3?5SerialRecv?3?5Packet?5checksu@ 10003178     oal_kitl:kitlserial.obj
 0001:000021b0       ??_C@_0FC@OLAMHMJA@WARN?3?5SerialRecv?3?5payload?5size?5e@ 100031b0     oal_kitl:kitlserial.obj
 0001:00002208       ??_C@_0FE@EPOLMELO@WARN?3?5SerialRecv?3?5Packet?5type?5wr@ 10003208     oal_kitl:kitlserial.obj
 0001:00002260       ??_C@_0FH@COFDJCJM@WARN?3?5SerialRecv?3?5Header?5checksu@ 10003260     oal_kitl:kitlserial.obj
 0001:000022b8       ??_C@_0BK@PNMBDCIB@?$CLSerialRecv?$CI0x?$CF08x?0?5?$CFd?$CJ?$AN?6?$AA@ 100032b8     oal_kitl:kitlserial.obj
 0001:00002368       ??_C@_0CJ@OFEHEAMD@KITL?3?5Connected?5host?5?5IP?3?5?$CFs?5?5Po@ 10003368     oal_kitl:kitleth.obj
 0001:00002394       ??_C@_0CB@GFLGAKPJ@KITL?3?5Start?5DHCP?5RENEW?5process?$AN?6@ 10003394     oal_kitl:kitleth.obj
 0001:000023b8       ??_C@_0BM@FALEIOIG@?9OALIoCtlVBridge?$CIrc?5?$DN?5?$CFd?$CJ?$AN?6?$AA@ 100033b8     oal_kitl:kitleth.obj
 0001:000023d4       ??_C@_0BP@BIAFCCDM@?$CLOALIoCtlVBridge?$CI0x?$CF08x?0?4?4?4?$CJ?$AN?6?$AA@ 100033d4     oal_kitl:kitleth.obj
 0001:000023f4       ??_C@_0BL@OCIIDPCB@?9OALKitlEthInit?$CIrc?5?$DN?5?$CFd?$CJ?$AN?6?$AA@ 100033f4     oal_kitl:kitleth.obj
 0001:00002410       ??_C@_0BL@EIDMIDBA@KITL?3?5using?5sysintr?50x?$CFx?$AN?6?$AA@ 10003410     oal_kitl:kitleth.obj
 0001:0000242c       ??_C@_0BP@ILGKAKAA@KITL?3?5?$CK?$CK?$CK?5Device?5Name?5?$CFs?5?$CK?$CK?$CK?$AN?6?$AA@ 1000342c     oal_kitl:kitleth.obj
 0001:0000244c       ??_C@_0CO@PDOCGCJP@ERROR?3?5KITL?5call?5to?5pfnInitDmaBu@ 1000344c     oal_kitl:kitleth.obj
 0001:0000247c       ??_C@_0CO@HIMCOMKP@?$CLOALKitlEthInit?$CI?8?$CFS?8?0?5?8?$CFs?8?0?50x?$CF0@ 1000347c     oal_kitl:kitleth.obj
 0001:000024ac       ??_C@_0CF@CNPGAGEH@KITL?3?5DHCP?5get?1renew?5device?5IP?3?5@ 100034ac     oal_kitl:kitleth.obj
 0001:000024d4       ??_C@_0CO@LIMJACDF@?9KitlEthDecode?$CIpData?5?$DN?50x?$CF08x?0?5l@ 100034d4     oal_kitl:kitleth.obj
 0001:00002504       ??_C@_0CF@DCHGBGAP@?$CLKitlEthDecode?$CI0x?$CF08x?0?50x?$CF08x?9?$DO?$CF@ 10003504     oal_kitl:kitleth.obj
 0001:0000252c       ??_C@_0BJ@BAFHPAIJ@?9KitlEthEncode?$CIrc?5?$DN?51?$CJ?$AN?6?$AA@ 1000352c     oal_kitl:kitleth.obj
 0001:00002548       ??_C@_0BL@NHDADPAH@?$CLKitlEthEncode?$CI?$CF08x?0?5?$CFd?$CJ?$AN?6?$AA@ 10003548     oal_kitl:kitleth.obj
 0001:00002564       ??_C@_0BN@OHPDCAJH@?9KitlEthGetDevCfg?$CIrc?5?$DN?5?$CFd?$CJ?$AN?6?$AA@ 10003564     oal_kitl:kitleth.obj
 0001:00002584       ??_C@_0CI@LLEHHLED@?$CLKitlEthGetDevCfg?$CI0x?$CF08x?0?50x?$CF08x@ 10003584     oal_kitl:kitleth.obj
 0001:000025ac       ??_C@_0BI@DJIGCCGG@?9KitlEthSend?$CIrc?5?$DN?5?$CFd?$CJ?$AN?6?$AA@ 100035ac     oal_kitl:kitleth.obj
 0001:000025c4       ??_C@_0CA@ELPHLPBP@?$CBDriver?5Send?5failure?0?5retry?5?$CFu?6?$AA@ 100035c4     oal_kitl:kitleth.obj
 0001:000025e4       ??_C@_0BL@MJDALEMH@?$CLKitlEthSend?$CI0x?$CF08x?0?5?$CFd?$CJ?$AN?6?$AA@ 100035e4     oal_kitl:kitleth.obj
 0001:00002600       ??_C@_0BI@PEEPNADN@?9KitlEthRecv?$CIrc?5?$DN?5?$CFd?$CJ?$AN?6?$AA@ 10003600     oal_kitl:kitleth.obj
 0001:00002618       ??_C@_0CD@HNBDALDE@?$CLKitlEthRecv?$CI0x?$CF08x?0?50x?$CF08x?9?$DO?$CFd?$CJ@ 10003618     oal_kitl:kitleth.obj
 0001:0000263c       ??_C@_0BE@NDAHGBJL@?9KitlEthEnableInt?$AN?6?$AA@ 1000363c     oal_kitl:kitleth.obj
 0001:00002650       ??_C@_0BI@OLDCGLHD@?$CLKitlEthEnableInt?$CI?$CFd?$CJ?$AN?6?$AA@ 10003650     oal_kitl:kitleth.obj
 0001:000026f8       ??_C@_0EB@BGCKLDE@?9OALKitlFindDevice?$CIpDevice?5?$DN?50x?$CF@ 100036f8     oal_kitl:device.obj
 0001:0000273c       ??_C@_11LOCGONAA@?$AA?$AA@ 1000373c     oal_kitl:device.obj
 0001:00002740       ??_C@_0CJ@GPDFFIKB@?$CLOALKitlFindDevice?$CI?$CFd?1?$CFd?1?$CF08x?0?50@ 10003740     oal_kitl:device.obj
 0001:0000276c       ??_C@_0CJ@MPHJDLPH@?9OALKitlDeviceName?$CIname?5?$DN?50x?$CF08x@ 1000376c     oal_kitl:device.obj
 0001:00002798       ??_C@_0CJ@OKPKABKG@?$CLOALKitlDeviceName?$CI?$CFd?1?$CFd?1?$CF08x?0?50@ 10003798     oal_kitl:device.obj
 0001:000027c4       ??_C@_0CA@ECNOOFDD@?9OALKitlDeviceType?$CItype?5?$DN?5?$CFd?$CJ?$AN?6?$AA@ 100037c4     oal_kitl:device.obj
 0001:000027e4       ??_C@_0CJ@HOEFFCBD@?$CLOALKitlDeviceType?$CI?$CFd?1?$CFd?1?$CF08x?0?50@ 100037e4     oal_kitl:device.obj
 0001:000028a0       ??_C@_1BI@FCMLLAGN@?$AA?$CF?$AAd?$AA?4?$AA?$CF?$AAd?$AA?4?$AA?$CF?$AAd?$AA?4?$AA?$CF?$AAd?$AA?$AA@ 100038a0     oal_kitl:format.obj
 0001:000028b8       ??_C@_1DM@BKFFFBIH@?$AA?$CF?$AA0?$AA2?$AAx?$AA?3?$AA?$CF?$AA0?$AA2?$AAx?$AA?3?$AA?$CF?$AA0?$AA2?$AAx?$AA?3?$AA?$CF?$AA0?$AA2?$AAx?$AA?3?$AA?$CF?$AA0?$AA2?$AAx?$AA?3?$AA?$CF?$AA0?$AA2?$AAx?$AA?$AA@ 100038b8     oal_kitl:format.obj
 0001:00002aa8       ??_C@_1CC@KBABDHEI@?$AA?9?$AAF?$AAE?$AAC?$AAE?$AAn?$AAa?$AAb?$AAl?$AAe?$AAI?$AAn?$AAt?$AAs?$AA?$AN?$AA?6?$AA?$AA@ 10003aa8     oal_ethdrv_fec_common_topaz_v1:fec.obj
 0001:00002acc       ??_C@_1CC@HKAMNBPM@?$AA?$CL?$AAF?$AAE?$AAC?$AAE?$AAn?$AAa?$AAb?$AAl?$AAe?$AAI?$AAn?$AAt?$AAs?$AA?$AN?$AA?6?$AA?$AA@ 10003acc     oal_ethdrv_fec_common_topaz_v1:fec.obj
 0001:00002af0       ??_C@_1CE@PAJNDNPH@?$AA?9?$AAF?$AAE?$AAC?$AAD?$AAi?$AAs?$AAa?$AAb?$AAl?$AAe?$AAI?$AAn?$AAt?$AAs?$AA?$AN?$AA?6?$AA?$AA@ 10003af0     oal_ethdrv_fec_common_topaz_v1:fec.obj
 0001:00002b14       ??_C@_1CE@DJFNMKAL@?$AA?$CL?$AAF?$AAE?$AAC?$AAD?$AAi?$AAs?$AAa?$AAb?$AAl?$AAe?$AAI?$AAn?$AAt?$AAs?$AA?$AN?$AA?6?$AA?$AA@ 10003b14     oal_ethdrv_fec_common_topaz_v1:fec.obj
 0001:00002b38       ??_C@_1DK@CHFIODGD@?$AA?9?$AAF?$AAE?$AAC?$AAI?$AAn?$AAi?$AAt?$AAD?$AAM?$AAA?$AAB?$AAu?$AAf?$AAf?$AAe?$AAr?$AA?$CI?$AAr?$AAc?$AA?5?$AA?$DN?$AA?5?$AA?$CF?$AAd?$AA?$CJ?$AA?$AN?$AA?6?$AA?$AA@ 10003b38     oal_ethdrv_fec_common_topaz_v1:fec.obj
 0001:00002b78       ??_C@_1GA@LFAILOCH@?$AAE?$AAR?$AAR?$AAO?$AAR?$AA?3?$AA?5?$AAF?$AAE?$AAC?$AAI?$AAn?$AAi?$AAt?$AAD?$AAM?$AAA?$AAB?$AAu?$AAf?$AAf?$AAe?$AAr?$AA?3?$AA?5?$AAD?$AAM?$AAA?$AA?5?$AAB?$AAu?$AAf@ 10003b78     oal_ethdrv_fec_common_topaz_v1:fec.obj
 0001:00002bd8       ??_C@_0CI@KMIJHHBB@FECInitDMABuffer?5DMA?5Buffer?5too?5@ 10003bd8     oal_ethdrv_fec_common_topaz_v1:fec.obj
 0001:00002c00       ??_C@_1EA@MDNGEOGF@?$AA?$CL?$AAF?$AAE?$AAC?$AAI?$AAn?$AAi?$AAt?$AAD?$AAM?$AAA?$AAB?$AAu?$AAf?$AAf?$AAe?$AAr?$AA?$CI?$AA0?$AAx?$AA?$CF?$AAX?$AA?0?$AA?5?$AA0?$AAx?$AA?$CF?$AAX?$AA?$CJ?$AA?$AN?$AA?6?$AA?$AA@ 10003c00     oal_ethdrv_fec_common_topaz_v1:fec.obj
 0001:00002c40       ??_C@_1CI@LLGKHLKN@?$AA?9?$AAF?$AAE?$AAC?$AAI?$AAn?$AAi?$AAt?$AA?$CI?$AAr?$AAc?$AA?5?$AA?$DN?$AA?5?$AA?$CF?$AAd?$AA?$CJ?$AA?$AN?$AA?6?$AA?$AA@ 10003c40     oal_ethdrv_fec_common_topaz_v1:fec.obj
 0001:00002c68       ??_C@_0CN@NECAPPEM@FEC?5is?5linked?0?5speed?510?5Mbps?0?5ha@ 10003c68     oal_ethdrv_fec_common_topaz_v1:fec.obj
 0001:00002c98       ??_C@_0CN@KMHKLMCP@FEC?5is?5linked?0?5speed?510?5Mbps?0?5fu@ 10003c98     oal_ethdrv_fec_common_topaz_v1:fec.obj
 0001:00002cc8       ??_C@_0CO@NCDNBHO@FEC?5is?5linked?0?5speed?5100?5Mbps?0?5h@ 10003cc8     oal_ethdrv_fec_common_topaz_v1:fec.obj
 0001:00002cf8       ??_C@_0CO@HFHJJCBN@FEC?5is?5linked?0?5speed?5100?5Mbps?0?5f@ 10003cf8     oal_ethdrv_fec_common_topaz_v1:fec.obj
 0001:00002d28       ??_C@_0BG@BPBIADDC@Waiting?5for?5link?4?4?4?$AN?6?$AA@ 10003d28     oal_ethdrv_fec_common_topaz_v1:fec.obj
 0001:00002d40       ??_C@_0CB@DFINIDFK@Failed?5to?5get?5the?5external?5PHY?$AN?6@ 10003d40     oal_ethdrv_fec_common_topaz_v1:fec.obj
 0001:00002d68       ??_C@_1EM@PFHKNHEN@?$AAT?$AAh?$AAe?$AA?5?$AAn?$AAa?$AAm?$AAe?$AA?5?$AAf?$AAo?$AAr?$AA?5?$AAt?$AAh?$AAe?$AA?5?$AAe?$AAx?$AAt?$AAe?$AAr?$AAn?$AAa?$AAl?$AA?5?$AAP?$AAH?$AAY?$AA?5?$AAi?$AAs@ 10003d68     oal_ethdrv_fec_common_topaz_v1:fec.obj
 0001:00002db4       ??_C@_1DM@PNEAGLBJ@?$AAM?$AAI?$AAI?$AA_?$AAR?$AAE?$AAG?$AA_?$AAP?$AAH?$AAY?$AAI?$AAR?$AA1?$AA?5?$AAR?$AAE?$AAA?$AAD?$AA?5?$AAF?$AAa?$AAi?$AAl?$AAe?$AAd?$AA?5?$AA?$AN?$AA?6?$AA?$AA@ 10003db4     oal_ethdrv_fec_common_topaz_v1:fec.obj
 0001:00002df0       ??_C@_1HC@KIHIPIBC@?$AAF?$AAE?$AAC?$AAI?$AAn?$AAi?$AAt?$AA?$CI?$AA0?$AAx?$AA?$CF?$AA0?$AA8?$AAx?$AA?0?$AA?5?$AA0?$AAx?$AA?$CF?$AA0?$AA8?$AAx?$AA?0?$AA?5?$AA?$CF?$AA0?$AA2?$AAx?$AA?3?$AA?$CF?$AA0?$AA2@ 10003df0     oal_ethdrv_fec_common_topaz_v1:fec.obj
 0001:00002e64       ??_C@_0BL@PCLOMCF@Initializing?5Ethernet?4?4?4?$AN?6?$AA@ 10003e64     oal_ethdrv_fec_common_topaz_v1:fec.obj
 0001:00002e80       ??_C@_1DC@PKJNHKDJ@?$AA?9?$AAF?$AAE?$AAC?$AAS?$AAe?$AAn?$AAd?$AAF?$AAr?$AAa?$AAm?$AAe?$AA?$CI?$AAr?$AAc?$AA?5?$AA?$DN?$AA?5?$AA?$CF?$AAd?$AA?$CJ?$AA?$AN?$AA?6?$AA?$AA@ 10003e80     oal_ethdrv_fec_common_topaz_v1:fec.obj
 0001:00002eb8       ??_C@_1EI@KKGEKELM@?$AAE?$AAR?$AAR?$AAO?$AAR?$AA?3?$AA?5?$AAF?$AAE?$AAC?$AAS?$AAe?$AAn?$AAd?$AAF?$AAr?$AAa?$AAm?$AAe?$AA?3?$AA?5?$AAS?$AAe?$AAn?$AAd?$AA?5?$AAt?$AAi?$AAm?$AAe?$AAo?$AAu@ 10003eb8     oal_ethdrv_fec_common_topaz_v1:fec.obj
 0001:00002f00       ??_C@_1CE@KCCCDJJH@?$AA?$CL?$AAS?$AA?5?$AA?$CI?$AA0?$AAx?$AA?$CF?$AA0?$AA8?$AAx?$AA?0?$AA?5?$AA?$CF?$AAd?$AA?$CJ?$AA?$AN?$AA?6?$AA?$AA@ 10003f00     oal_ethdrv_fec_common_topaz_v1:fec.obj
 0001:00002f28       ??_C@_1EA@BEFHLOEB@?$AA?9?$AAF?$AAE?$AAC?$AAG?$AAe?$AAt?$AAF?$AAr?$AAa?$AAm?$AAe?$AA?$CI?$AAP?$AAa?$AAc?$AAk?$AAe?$AAt?$AAS?$AAi?$AAz?$AAe?$AA?5?$AA?$DN?$AA?5?$AA?$CF?$AAd?$AA?$CJ?$AA?$AN?$AA?6?$AA?$AA@ 10003f28     oal_ethdrv_fec_common_topaz_v1:fec.obj
 0001:00002f68       ??_C@_1DG@LJFMBLGF@?$AA?$CL?$AAF?$AAE?$AAC?$AAG?$AAe?$AAt?$AAF?$AAr?$AAa?$AAm?$AAe?$AA?$CI?$AA0?$AAx?$AA?$CF?$AA0?$AA8?$AAx?$AA?0?$AA?5?$AA?$CF?$AAd?$AA?$CJ?$AA?$AN?$AA?6?$AA?$AA@ 10003f68     oal_ethdrv_fec_common_topaz_v1:fec.obj
 0001:00002fa0       ??_C@_1DE@NJHDJGOC@?$AA?9?$AAF?$AAE?$AAC?$AAC?$AAu?$AAr?$AAr?$AAe?$AAn?$AAt?$AAP?$AAa?$AAc?$AAk?$AAe?$AAt?$AAF?$AAi?$AAl?$AAt?$AAe?$AAr?$AA?$AN?$AA?6?$AA?$AA@ 10003fa0     oal_ethdrv_fec_common_topaz_v1:fec.obj
 0001:00002fd8       ??_C@_1EE@EDJFMPFC@?$AA?$CL?$AAF?$AAE?$AAC?$AAC?$AAu?$AAr?$AAr?$AAe?$AAn?$AAt?$AAP?$AAa?$AAc?$AAk?$AAe?$AAt?$AAF?$AAi?$AAl?$AAt?$AAe?$AAr?$AA?$CI?$AA0?$AAx?$AA?$CF?$AA0?$AA8?$AAx?$AA?$CJ?$AA?$AN@ 10003fd8     oal_ethdrv_fec_common_topaz_v1:fec.obj
 0001:0000301c       ??_C@_1DI@GJINCFOM@?$AA?9?$AAF?$AAE?$AAC?$AAM?$AAu?$AAl?$AAt?$AAi?$AAc?$AAa?$AAs?$AAt?$AAL?$AAi?$AAs?$AAt?$AA?$CI?$AAr?$AAc?$AA?5?$AA?$DN?$AA?5?$AA1?$AA?$CJ?$AA?$AN?$AA?6?$AA?$AA@ 1000401c     oal_ethdrv_fec_common_topaz_v1:fec.obj
 0001:00003058       ??_C@_1EA@CKJMHDOG@?$AA?$CL?$AAF?$AAE?$AAC?$AAM?$AAu?$AAl?$AAt?$AAi?$AAc?$AAa?$AAs?$AAt?$AAL?$AAi?$AAs?$AAt?$AA?$CI?$AA0?$AAx?$AA?$CF?$AA0?$AA8?$AAx?$AA?0?$AA?5?$AA?$CF?$AAd?$AA?$CJ?$AA?$AN?$AA?6?$AA?$AA@ 10004058     oal_ethdrv_fec_common_topaz_v1:fec.obj
 0001:00003128       ??_C@_05OHIIGEOJ@E?5?$CFx?6?$AA@ 10004128     oal_kitlserial_common_topaz_v1:kitlserial.obj
 0001:00003130       ??_C@_1DE@DAHNLBLJ@?$AA?9?$AAO?$AAA?$AAL?$AAP?$AAA?$AAt?$AAo?$AAV?$AAA?$AA?$CI?$AAv?$AAa?$AA?5?$AA?$DN?$AA?5?$AA0?$AAx?$AA?$CF?$AA0?$AA8?$AAx?$AA?$CJ?$AA?$AN?$AA?6?$AA?$AA@ 10004130     oal_memory_arm:memory.obj
 0001:00003164       ??_C@_1CO@JEIJEAKF@?$AA?$CL?$AAO?$AAA?$AAL?$AAP?$AAA?$AAt?$AAo?$AAV?$AAA?$AA?$CI?$AA0?$AAx?$AA?$CF?$AAx?$AA?0?$AA?5?$AA?$CF?$AAd?$AA?$CJ?$AA?$AN?$AA?6?$AA?$AA@ 10004164     oal_memory_arm:memory.obj
 0001:00003194       ??_C@_1DA@BBOHBBNH@?$AA?9?$AAO?$AAA?$AAL?$AAV?$AAA?$AAt?$AAo?$AAP?$AAA?$AA?$CI?$AAp?$AAa?$AA?5?$AA?$DN?$AA?5?$AA0?$AAx?$AA?$CF?$AAx?$AA?$CJ?$AA?$AN?$AA?6?$AA?$AA@ 10004194     oal_memory_arm:memory.obj
 0001:000031c4       ??_C@_1CK@LKNIEAFP@?$AA?$CL?$AAO?$AAA?$AAL?$AAV?$AAA?$AAt?$AAo?$AAP?$AAA?$AA?$CI?$AA0?$AAx?$AA?$CF?$AA0?$AA8?$AAx?$AA?$CJ?$AA?$AN?$AA?6?$AA?$AA@ 100041c4     oal_memory_arm:memory.obj
 0001:00003280       ??_C@_1EA@DJGHLELP@?$AA?9?$AAO?$AAA?$AAL?$AAA?$AAr?$AAg?$AAs?$AAQ?$AAu?$AAe?$AAr?$AAy?$AA?$CI?$AAp?$AAD?$AAa?$AAt?$AAa?$AA?5?$AA?$DN?$AA?5?$AA0?$AAx?$AA?$CF?$AA0?$AA8?$AAx?$AA?$CJ?$AA?$AN?$AA?6?$AA?$AA@ 10004280     args:args.obj
 0001:000032c0       ??_C@_1CI@CLMEBIJE@?$AA?$CL?$AAO?$AAA?$AAL?$AAA?$AAr?$AAg?$AAs?$AAQ?$AAu?$AAe?$AAr?$AAy?$AA?$CI?$AA?$CF?$AAd?$AA?$CJ?$AA?$AN?$AA?6?$AA?$AA@ 100042c0     args:args.obj
 0001:00003378       ??_C@_1FE@FFNPEPPH@?$AAH?$AAa?$AAr?$AAd?$AAw?$AAa?$AAr?$AAe?$AA?5?$AAf?$AAl?$AAo?$AAw?$AA?5?$AAc?$AAo?$AAn?$AAt?$AAr?$AAo?$AAl?$AA?5?$AAi?$AAs?$AA?5?$AAn?$AAo?$AAt?$AA?5?$AAs?$AAu?$AAp@ 10004378     serialutils:serialutils.obj
 0001:000033d0       ??_C@_1KG@BFMCBNEC@?$AAC?$AA?3?$AA?2?$AAW?$AAI?$AAN?$AAC?$AAE?$AAR?$AAO?$AAO?$AAT?$AAS?$AA?2?$AAT?$AAo?$AAp?$AAa?$AAz?$AA?2?$AAW?$AAI?$AAN?$AAC?$AAE?$AA6?$AA0?$AA0?$AA?2?$AAP?$AAL?$AAA@ 100043d0     serialutils:serialutils.obj
 0001:00003508       ??_C@_1FC@FNPBDIGP@?$AAO?$AAA?$AAL?$AAK?$AAi?$AAt?$AAl?$AAF?$AAE?$AAC?$AAB?$AAS?$AAP?$AAI?$AAn?$AAi?$AAt?$AA?3?$AA?5?$AAG?$AAP?$AAI?$AAO?$AA2?$AA?5?$AAn?$AAu?$AAl?$AAl?$AA?5?$AAp?$AAo@ 10004508     bspfec:bspfec.obj
 0001:00003560       ??_C@_1FC@MIIBOMPK@?$AAO?$AAA?$AAL?$AAK?$AAi?$AAt?$AAl?$AAF?$AAE?$AAC?$AAB?$AAS?$AAP?$AAI?$AAn?$AAi?$AAt?$AA?3?$AA?5?$AAG?$AAP?$AAI?$AAO?$AA3?$AA?5?$AAn?$AAu?$AAl?$AAl?$AA?5?$AAp?$AAo@ 10004560     bspfec:bspfec.obj
 0001:000035b8       ??_C@_1FC@JEDBMPJD@?$AAO?$AAA?$AAL?$AAK?$AAi?$AAt?$AAl?$AAF?$AAE?$AAC?$AAB?$AAS?$AAP?$AAI?$AAn?$AAi?$AAt?$AA?3?$AA?5?$AAG?$AAP?$AAI?$AAO?$AA4?$AA?5?$AAn?$AAu?$AAl?$AAl?$AA?5?$AAp?$AAo@ 100045b8     bspfec:bspfec.obj
 0001:00003610       ??_C@_1FI@GIMIACCK@?$AAO?$AAA?$AAL?$AAK?$AAi?$AAt?$AAl?$AAF?$AAE?$AAC?$AAB?$AAS?$AAP?$AAI?$AAn?$AAi?$AAt?$AA?3?$AA?5?$AAI?$AAO?$AAM?$AAU?$AAX?$AAC?$AA?5?$AAm?$AAa?$AAp?$AAp?$AAi?$AAn@ 10004610     bspfec:bspfec.obj
 0001:000036f8       ??_C@_03IGDBGCKF@?$CFx?5?$AA@ 100046f8     vbridge:vbridge.obj
 0001:000036fc       ??_C@_01GBGANLPD@0?$AA@    100046fc     vbridge:vbridge.obj
 0001:00003700       ??_C@_04FMMHFHOO@?$AN?6?$AN?6?$AA@ 10004700     vbridge:vbridge.obj
 0001:00003708       ??_C@_08CNLJFGND@?$AN?60x?$CFx?3?5?$AA@ 10004708     vbridge:vbridge.obj
 0001:00003714       ??_C@_06DGFDGGJM@0x?$CFx?3?5?$AA@ 10004714     vbridge:vbridge.obj
 0001:0000371c       ??_C@_0CB@CALJDEOO@?$CL?9?9?9?9?5MEM?5DUMP?5?$CI?$CFd?5bytes?$CJ?9?9?9?9?$CL?$AN?6@ 1000471c     vbridge:vbridge.obj
 0001:00003740       ??_C@_0EH@OHHLEIM@VBridge?3?5Error?$CB?5ProduceBufferDon@ 10004740     vbridge:vbridge.obj
 0001:00003788       ??_C@_0ED@LALCLDGC@VBridge?3?5Error?$CB?5ConsumeBuffer?$CI?$CJ?5@ 10004788     vbridge:vbridge.obj
 0001:000037d0       ??_C@_0EH@PDMAJMNN@VBridge?3?5Error?$CB?5ConsumeBufferDon@ 100047d0     vbridge:vbridge.obj
 0001:00003818       ??_C@_0GA@BIIJJCHI@VBridge?3?5Error?$CB?5ConsumeBufferDon@ 10004818     vbridge:vbridge.obj
 0001:00003878       ??_C@_0BO@DMIECOA@Rx?5buffer?5?$FL0x?$CFx?$FN?5to?5?$FL0x?$CFx?$FN?4?$AN?6?$AA@ 10004878     vbridge:vbridge.obj
 0001:00003898       ??_C@_0BO@IKIKAINA@Tx?5buffer?5?$FL0x?$CFx?$FN?5to?5?$FL0x?$CFx?$FN?4?$AN?6?$AA@ 10004898     vbridge:vbridge.obj
 0001:000038b8       ??_C@_0DF@FKGFCLPJ@VBridgeInit?$CI?$CJ?4?4?4TX?5?$DN?5?$FL?$CFd?$FN?5bytes?5@ 100048b8     vbridge:vbridge.obj
 0001:000038f0       ??_C@_0CE@JNBGKBJC@VBridge?3?3?5built?5on?5?$FL?$CFs?$FN?5time?5?$FL?$CFs@ 100048f0     vbridge:vbridge.obj
 0001:00003914       ??_C@_0M@CJCABMIH@Sep?5?56?52006?$AA@ 10004914     vbridge:vbridge.obj
 0001:00003920       ??_C@_08OLPOOGDN@19?325?301?$AA@ 10004920     vbridge:vbridge.obj
 0001:0000392c       ??_C@_0CO@ILLJABOE@VBridgeKGetOneTxBuffer?$CI?$CJ?5Err?$CB?5?$FL0@ 1000492c     vbridge:vbridge.obj
 0001:0000395c       ??_C@_0DE@LOPBMMHM@VBridgeKGetOneTxBufferComplete?$CI?$CJ@ 1000495c     vbridge:vbridge.obj
 0001:00003990       ??_C@_0DI@HEJDFJBF@?$CK?$CK?5WARNING?$CB?$CB?$CB?5?$CK?$CK?5Device?5MAC?5addr@ 10004990     vbridge:vbridge.obj
 0001:000039c8       ??_C@_0DJ@LKNKOIHJ@VBridgeKIndicateOneRxBuffer?$CI?$CJ?5Er@ 100049c8     vbridge:vbridge.obj
 0001:00003a04       ??_C@_0CM@PJABNFGI@VBridge?3?3?5NK?5add?5MAC?3?5?$FL?$CFx?9?$CFx?9?$CFx?9@ 10004a04     vbridge:vbridge.obj
 0001:00003a30       ??_C@_0DJ@JPHIEPAD@VBridgeKSetLocalMacAddress?$CI?$CJ?5Err@ 10004a30     vbridge:vbridge.obj
 0001:00003a6c       ??_C@_0DA@BNPLKEKM@VBridgeUGetOneTxPacket?$CI?$CJ?5Err?$CB?$CB?5?$FL@ 10004a6c     vbridge:vbridge.obj
 0001:00003a9c       ??_C@_0DI@MDDGKNHB@VBridgeUGetOneTxPacketComplete?$CI?$CJ@ 10004a9c     vbridge:vbridge.obj
 0001:00003ad4       ??_C@_0DA@MGPGECBI@VBridgeUGetOneRxPacket?$CI?$CJ?5Err?$CB?$CB?5?$FL@ 10004ad4     vbridge:vbridge.obj
 0001:00003b04       ??_C@_0DA@KIINIKAM@VBridgeUGetOneRxPacketComplete?$CI?$CJ@ 10004b04     vbridge:vbridge.obj
 0001:00003b34       ??_C@_0CI@BDPMFOMO@VBridge?3?3?5VB_INITIALIZED?5returns@ 10004b34     vbridge:vbridge.obj
 0001:00003b5c       ??_C@_0CD@KPODIJAL@VBridge?3?3?5RESET_BUFFER?5received?4@ 10004b5c     vbridge:vbridge.obj
 0001:00003b80       ??_C@_0DB@IMBKLANK@VBridgeUGetEDBGMac?$CI?$CJ?0?5ERR?$CB?5NULL?5@ 10004b80     vbridge:vbridge.obj
 0001:00003bb4       ??_C@_0DB@BMKDFNPB@VBridge?3?3?5Current?5VMini?5packet?5f@ 10004bb4     vbridge:vbridge.obj
 0001:00003be8       ??_C@_0DG@MKNLPBLF@VBridgeUCurrentPacketFilter?$CI?$CJ?0?5E@ 10004be8     vbridge:vbridge.obj
 0001:00003cb0       ??_C@_0BK@FGOBGFEM@RNDISMINI?5?9?9?9?5RESET?5?9?9?9?$AN?6?$AA@ 10004cb0     fsl_rne_mdd_common_topaz_v1:rndis.obj
 0001:00003ccc       ??_C@_0CK@HCFNMAPL@RNdis?3?3?5Too?5much?5outgoing?0?5baili@ 10004ccc     fsl_rne_mdd_common_topaz_v1:rndis.obj
 0001:00003cf8       ??_C@_0DK@LOJODLJL@ASSERT?$CB?5Rndis?3?3MddSendRndisMessa@ 10004cf8     fsl_rne_mdd_common_topaz_v1:rndis.obj
 0001:00003d34       ??_C@_0BN@MJFOLLBM@RNdis?3?3?5Should?5not?5happen?$CB?$AN?6?$AA@ 10004d34     fsl_rne_mdd_common_topaz_v1:rndis.obj
 0001:00003d54       ??_C@_0CK@BEACHKGH@RNdis?3?3?5No?5mem?5for?5INITIALIZE_CO@ 10004d54     fsl_rne_mdd_common_topaz_v1:rndis.obj
 0001:00003d80       ??_C@_0DI@ELIDGGNF@ASSERT?5Fail?5at?5uiMessageSize?$CI?$CFd?$CJ@ 10004d80     fsl_rne_mdd_common_topaz_v1:rndis.obj
 0001:00003db8       ??_C@_0DA@CMCBBBCA@RNdis?3?3?5Unknown?5RNDIS?5msg?0?5buff?$FL@ 10004db8     fsl_rne_mdd_common_topaz_v1:rndis.obj
 0001:00003de8       ??_C@_0DB@PAFHLFPB@RndisMini?5rcv?5REMOTE_NDIS_RESET_@ 10004de8     fsl_rne_mdd_common_topaz_v1:rndis.obj
 0001:00003e1c       ??_C@_0DB@NGCDHJGD@RndisMini?5recv?5REMOTE_NDIS_HALT_@ 10004e1c     fsl_rne_mdd_common_topaz_v1:rndis.obj
 0001:00003e50       ??_C@_0CP@HEPIJLKK@RndisMdd?3?3?5PDD?8s?5max?5RX?5buffer?5?$DN@ 10004e50     fsl_rne_mdd_common_topaz_v1:rndis.obj
 0001:00003e80       ??_C@_0BP@HHOMIKAO@ASSERT?5at?5File?$CI?$CFs?$CJ?5line?5?$CI?$CFd?$CJ?$AN?6?$AA@ 10004e80     fsl_rne_mdd_common_topaz_v1:rndis.obj
 0001:00003ea0       ??_C@_09JBPNJICM@rndis?4cpp?$AA@ 10004ea0     fsl_rne_mdd_common_topaz_v1:rndis.obj
 0001:00003eac       ??_C@_0CK@JCOPOCLM@ERROR?$CB?5RndisInitialize?5msg?5recei@ 10004eac     fsl_rne_mdd_common_topaz_v1:rndis.obj
 0001:00003ed8       ??_C@_0CO@JHJMPDCG@RNDISMINI?5Err?$CB?$CB?5unsupported?5RNDI@ 10004ed8     fsl_rne_mdd_common_topaz_v1:rndis.obj
 0001:00003f08       ??_C@_0P@BDJJIKDL@Overrun?$DN0x?$CFx?6?$AN?$AA@ 10004f08     fsl_rne_mdd_common_topaz_v1:rndis.obj
 0001:00003f18       ??_C@_0BJ@IJMDONAK@Buffer?5is?5too?5big?50x?$CFx?6?$AN?$AA@ 10004f18     fsl_rne_mdd_common_topaz_v1:rndis.obj
 0001:00003f34       ??_C@_0CK@LKMHPIGI@Wrong?5Data?5DataLength?5Msg?$DN0x?$CFx?0P@ 10004f34     fsl_rne_mdd_common_topaz_v1:rndis.obj
 0001:00003f60       ??_C@_0CN@OHNGADLJ@RNdis?3?3?5Invalid?5RndisPacket?5l?$FL?$CFd@ 10004f60     fsl_rne_mdd_common_topaz_v1:rndis.obj
 0001:00003f90       ??_C@_0BH@HBKBIINO@Wrong?5Data?5Type?50x?$CFx?$AN?6?$AA@ 10004f90     fsl_rne_mdd_common_topaz_v1:rndis.obj
 0001:00003fa8       ??_C@_0CA@IBGOHNCO@Rndis?3?3?5initialization?3?5Fail?$CB?$AN?6?$AA@ 10004fa8     fsl_rne_mdd_common_topaz_v1:rndis.obj
 0001:00003fc8       ??_C@_0CC@EELLDCCI@Rndis?3?3?5initialization?3?5Success?$AN@ 10004fc8     fsl_rne_mdd_common_topaz_v1:rndis.obj
 0001:00003fec       ??_C@_0CD@EOFHIDOL@Rndis?3?3?5Get?5MAC?5address?5?$CFx?0?$CFx?0?$CFx@ 10004fec     fsl_rne_mdd_common_topaz_v1:rndis.obj
 0001:00004010       ??_C@_0CM@KLOLOCDD@Rndis?3?3?5Err?5no?5MAC?5address?5read?5@ 10005010     fsl_rne_mdd_common_topaz_v1:rndis.obj
 0001:0000403c       ??_C@_0BL@EINAHMEI@Rndis?3?3?5PDDInit?5Success?$CB?$AN?6?$AA@ 1000503c     fsl_rne_mdd_common_topaz_v1:rndis.obj
 0001:00004058       ??_C@_0BK@BFGGBGMH@Rndis?3?3?5initialization?$CB?$AN?6?$AA@ 10005058     fsl_rne_mdd_common_topaz_v1:rndis.obj
 0001:00004074       ??_C@_0CI@PFDJABBD@Rndis?3?3?5Address?5static?5map?5to?5ad@ 10005074     fsl_rne_mdd_common_topaz_v1:rndis.obj
 0001:0000409c       ??_C@_0CH@LBCKJEJO@Rndis?3?3?5initialization?3?5with?5add@ 1000509c     fsl_rne_mdd_common_topaz_v1:rndis.obj
 0001:00004158       ??_C@_0BP@JDIDIKNB@OID?$FL?$CFx?$FN?5not?5yet?5implemented?$CB?$AN?6?$AA@ 10005158     fsl_rne_mdd_common_topaz_v1:hostmini.obj
 0001:00004178       ??_C@_0CP@MKNOHPIM@HostMini?3?3?5New?5filter?5set?3?5?$FL0x?$CFx@ 10005178     fsl_rne_mdd_common_topaz_v1:hostmini.obj
 0001:000041a8       ??_C@_1LK@IAMBGBAA@?$AAC?$AA?3?$AA?2?$AAW?$AAI?$AAN?$AAC?$AAE?$AAR?$AAO?$AAO?$AAT?$AAS?$AA?2?$AAT?$AAo?$AAp?$AAa?$AAz?$AA?2?$AAW?$AAI?$AAN?$AAC?$AAE?$AA6?$AA0?$AA0?$AA?2?$AAP?$AAL?$AAA@ 100051a8     fsl_rne_mdd_common_topaz_v1:hostmini.obj
 0001:00004264       ??_C@_0BN@DGLONFMO@HostMini?3?3?5MddDisconnect?$CB?$CB?$AN?6?$AA@ 10005264     fsl_rne_mdd_common_topaz_v1:hostmini.obj
 0001:00004284       ??_C@_0BE@LPGPNKBH@HostMiniInit?3?3?5?$CB?$CB?$AN?6?$AA@ 10005284     fsl_rne_mdd_common_topaz_v1:hostmini.obj
 0001:00004328       ??_C@_1O@NJEHEHHO@?$AAu?$AAt?$AAi?$AAl?$AA?4?$AAc?$AA?$AA@ 10005328     fsl_rne_mdd_common_topaz_v1:util.obj
 0001:00004338       ??_C@_1FA@PHGBNLGM@?$AAM?$AAi?$AAc?$AAr?$AAo?$AAs?$AAo?$AAf?$AAt?$AA?5?$AAR?$AAN?$AAD?$AAI?$AAS?$AA?5?$AAK?$AAI?$AAT?$AAL?$AA?5?$AAf?$AAo?$AAr?$AA?5?$AAF?$AAS?$AAL?$AA?5?$AAH?$AAS?$AA?5@ 10005338     fsl_rne_pdd_common_topaz_v1:rndis_pdd.obj
 0001:00004388       ??_C@_1BE@DEAPIJA@?$AAM?$AAi?$AAc?$AAr?$AAo?$AAs?$AAo?$AAf?$AAt?$AA?$AA@ 10005388     fsl_rne_pdd_common_topaz_v1:rndis_pdd.obj
 0001:00004444       DigitTable                 10005444     fsl_rne_pdd_common_topaz_v1:rndis_pdd.obj
 0001:00004468       ??_C@_1FE@MMFBADFF@?$AA?$CK?$AA?$CK?$AA?$CK?$AA?5?$AAU?$AAn?$AAk?$AAn?$AAo?$AAw?$AAn?$AA?5?$AAG?$AAE?$AAT?$AA_?$AAD?$AAE?$AAS?$AAC?$AAR?$AAI?$AAP?$AAT?$AAO?$AAR?$AA?5?$AAr?$AAe?$AAq?$AAu?$AAe@ 10005468     fsl_rne_pdd_common_topaz_v1:rndis_pdd.obj
 0001:000044bc       ??_C@_1DM@FCMMONGE@?$AA?$CK?$AA?$CK?$AA?$CK?$AA?5?$AAU?$AAn?$AAk?$AAn?$AAo?$AAw?$AAn?$AA?5?$AAS?$AAT?$AAR?$AAI?$AAN?$AAG?$AA?5?$AAi?$AAn?$AAd?$AAe?$AAx?$AA?5?$AA?$CF?$AAd?$AA?$AN?$AA?6?$AA?$AA@ 100054bc     fsl_rne_pdd_common_topaz_v1:rndis_pdd.obj
 0001:000044f8       ??_C@_1MI@GEAJABFB@?$AAC?$AA?3?$AA?2?$AAW?$AAI?$AAN?$AAC?$AAE?$AAR?$AAO?$AAO?$AAT?$AAS?$AA?2?$AAT?$AAo?$AAp?$AAa?$AAz?$AA?2?$AAW?$AAI?$AAN?$AAC?$AAE?$AA6?$AA0?$AA0?$AA?2?$AAP?$AAL?$AAA@ 100054f8     fsl_rne_pdd_common_topaz_v1:rndis_pdd.obj
 0001:000045c0       ??_C@_1CK@OLHEFDLK@?$AAN?$AAo?$AA?5?$AAm?$AAe?$AAm?$AA?5?$AAf?$AAo?$AAr?$AA?5?$AAR?$AAX?$AA?5?$AAd?$AAa?$AAt?$AAa?$AA?$AN?$AA?6?$AA?$AA@ 100055c0     fsl_rne_pdd_common_topaz_v1:rndis_pdd.obj
 0001:000045ec       ??_C@_1DI@FELDACDH@?$AAN?$AAo?$AA?5?$AAm?$AAe?$AAm?$AA?5?$AAf?$AAo?$AAr?$AA?5?$AAR?$AAX?$AA?5?$AAD?$AAa?$AAt?$AAa?$AAW?$AAr?$AAa?$AAp?$AAp?$AAe?$AAr?$AA?$AN?$AA?6?$AA?$AA@ 100055ec     fsl_rne_pdd_common_topaz_v1:rndis_pdd.obj
 0001:00004624       ??_C@_1DG@HDGBABFG@?$AA?$CK?$AA?$CK?$AA?$CK?$AA?5?$AAU?$AAn?$AAk?$AAn?$AAo?$AAw?$AAn?$AA?5?$AAr?$AAe?$AAq?$AAu?$AAe?$AAs?$AAt?$AA?5?$AA0?$AAx?$AA?$CF?$AAx?$AA?$AN?$AA?6?$AA?$AA@ 10005624     fsl_rne_pdd_common_topaz_v1:rndis_pdd.obj
 0001:00004660       ??_C@_1FI@GLILKAEG@?$AA?$CK?$AA?$CK?$AA?$CK?$AA?5?$AAU?$AAn?$AAH?$AAa?$AAn?$AAd?$AAl?$AAe?$AAd?$AA?5?$AAG?$AAE?$AAT?$AA_?$AAD?$AAE?$AAS?$AAC?$AAR?$AAI?$AAP?$AAT?$AAO?$AAR?$AA?5?$AAr?$AAe?$AAq@ 10005660     fsl_rne_pdd_common_topaz_v1:rndis_pdd.obj
 0001:000046b8       ??_C@_1CO@NANJHOKH@?$AA?$CK?$AA?$CK?$AA?$CK?$AAR?$AAe?$AAq?$AAu?$AAe?$AAs?$AAt?$AAT?$AAy?$AAp?$AAe?$AA?$DN?$AA?$DN?$AA0?$AAx?$AA0?$AA2?$AA?$AN?$AA?6?$AA?$AA@ 100056b8     fsl_rne_pdd_common_topaz_v1:rndis_pdd.obj
 0001:000046e8       ??_C@_1CO@MDAODOFD@?$AA?$CK?$AA?$CK?$AA?$CK?$AAR?$AAe?$AAq?$AAu?$AAe?$AAs?$AAt?$AAT?$AAy?$AAp?$AAe?$AA?$DN?$AA?$DN?$AA0?$AAx?$AA8?$AA2?$AA?$AN?$AA?6?$AA?$AA@ 100056e8     fsl_rne_pdd_common_topaz_v1:rndis_pdd.obj
 0001:00004718       ??_C@_1EM@PLFMLLKO@?$AA?$CK?$AA?$CK?$AA?$CK?$AA?$CK?$AA?5?$AAU?$AAn?$AAh?$AAa?$AAn?$AAd?$AAl?$AAe?$AAd?$AA?5?$AAv?$AAe?$AAr?$AAn?$AAd?$AAo?$AAr?$AA?5?$AAc?$AAo?$AAm?$AAm?$AAa?$AAn?$AAd?$AA?5?$AA0@ 10005718     fsl_rne_pdd_common_topaz_v1:rndis_pdd.obj
 0001:00004764       ??_C@_1O@KIJBGEAN@?$AAD?$AAo?$AAn?$AAe?$AA?$AN?$AA?6?$AA?$AA@ 10005764     fsl_rne_pdd_common_topaz_v1:rndis_pdd.obj
 0001:00004778       ??_C@_1FG@LFHLPLMG@?$AAS?$AAe?$AAn?$AAd?$AAP?$AAa?$AAc?$AAk?$AAe?$AAt?$AA?5?$AAr?$AAe?$AAq?$AAu?$AAe?$AAs?$AAt?$AA?5?$AAc?$AAo?$AAm?$AAp?$AAl?$AAe?$AAt?$AAe?$AAd?$AA?$CB?$AA?5?$AA?$FL?$AA?$CF@ 10005778     fsl_rne_pdd_common_topaz_v1:rndis_pdd.obj
 0001:000047d0       ??_C@_0CB@HAHFALKI@Unexpected?5Msg?5in?5NotifyHandler?$CB@ 100057d0     fsl_rne_pdd_common_topaz_v1:rndis_pdd.obj
 0001:000047f4       ??_C@_0BG@MPFHNHOK@Unexpected?5bus?5event?$CB?$AA@ 100057f4     fsl_rne_pdd_common_topaz_v1:rndis_pdd.obj
 0001:0000480c       ??_C@_1DO@PFNPIHHC@?$AAU?$AAn?$AAe?$AAx?$AAp?$AAe?$AAc?$AAt?$AAe?$AAd?$AA?5?$AAE?$AAP?$AA2?$AA?5?$AAt?$AAr?$AAa?$AAn?$AAs?$AAf?$AAe?$AAr?$AA?5?$AAs?$AAt?$AAa?$AAt?$AAe?$AA?$CB?$AA?$AA@ 1000580c     fsl_rne_pdd_common_topaz_v1:rndis_pdd.obj
 0001:00004850       ??_C@_1EG@NEPEKMDB@?$AAS?$AAe?$AAn?$AAd?$AAP?$AAa?$AAc?$AAk?$AAe?$AAt?$AA?5?$AAN?$AAU?$AAL?$AAL?$AA?5?$AAt?$AAe?$AAr?$AAm?$AAi?$AAn?$AAa?$AAt?$AAo?$AAr?$AA?5?$AAs?$AAe?$AAn?$AAt?$AA?$CB@ 10005850     fsl_rne_pdd_common_topaz_v1:rndis_pdd.obj
 0001:00004898       ??_C@_1FI@KOMJGPLF@?$AAS?$AAe?$AAn?$AAd?$AAi?$AAn?$AAg?$AA?5?$AAN?$AAU?$AAL?$AAL?$AA?5?$AAt?$AAe?$AAr?$AAm?$AAi?$AAn?$AAa?$AAt?$AAo?$AAr?$AA?5?$AAf?$AAo?$AAr?$AA?5?$AAt?$AAh?$AAe?$AA?5@ 10005898     fsl_rne_pdd_common_topaz_v1:rndis_pdd.obj
 0001:000048f0       ??_C@_1EA@ODINLGJJ@?$AAR?$AAe?$AAc?$AAe?$AAi?$AAv?$AAe?$AAd?$AA?5?$AAa?$AA?5?$AAp?$AAa?$AAc?$AAk?$AAe?$AAt?$AA?5?$AA?$FL?$AA?$CF?$AAd?$AA?5?$AAb?$AAy?$AAt?$AAe?$AAs?$AA?$FN?$AA?$CB?$AA?$AN?$AA?6?$AA?$AA@ 100058f0     fsl_rne_pdd_common_topaz_v1:rndis_pdd.obj
 0001:00004930       ??_C@_1EC@LJDGALBJ@?$AAS?$AAe?$AAn?$AAd?$AAM?$AAe?$AAs?$AAs?$AAa?$AAg?$AAe?$AA?5?$AAr?$AAe?$AAq?$AAu?$AAe?$AAs?$AAt?$AA?5?$AAc?$AAo?$AAm?$AAp?$AAl?$AAe?$AAt?$AAe?$AAd?$AA?$CB?$AA?$AN?$AA?6@ 10005930     fsl_rne_pdd_common_topaz_v1:rndis_pdd.obj
 0001:00004974       ??_C@_1CK@FEGGBLDE@?$AAD?$AAo?$AAn?$AAe?$AA?5?$AAs?$AAe?$AAn?$AAd?$AAi?$AAn?$AAg?$AA?5?$AAd?$AAa?$AAt?$AAa?$AA?4?$AA?$AN?$AA?6?$AA?$AA@ 10005974     fsl_rne_pdd_common_topaz_v1:rndis_pdd.obj
 0001:000049a0       ??_C@_1CM@FNJKEBIB@?$AAR?$AAe?$AAc?$AAe?$AAi?$AAv?$AAe?$AAd?$AA?5?$AAa?$AA?5?$AAm?$AAe?$AAs?$AAs?$AAa?$AAg?$AAe?$AA?$CB?$AA?$AN?$AA?6?$AA?$AA@ 100059a0     fsl_rne_pdd_common_topaz_v1:rndis_pdd.obj
 0001:000049cc       ??_C@_1CO@MJKBFNNP@?$AAD?$AAo?$AAn?$AAe?$AA?5?$AAr?$AAe?$AAc?$AAe?$AAi?$AAv?$AAi?$AAn?$AAg?$AA?5?$AAd?$AAa?$AAt?$AAa?$AA?4?$AA?$AN?$AA?6?$AA?$AA@ 100059cc     fsl_rne_pdd_common_topaz_v1:rndis_pdd.obj
 0001:00004a00       ??_C@_1FM@FDJOONCJ@?$AAG?$AAo?$AAt?$AA?5?$AAS?$AAE?$AAT?$AAU?$AAP?$AA?5?$AA?$DM?$AAN?$AAO?$AA?5?$AAD?$AAA?$AAT?$AAA?$AA?3?$AA?5?$AA?$CF?$AAx?$AA?5?$AA?$CF?$AAx?$AA?5?$AA?$CF?$AAx?$AA?5?$AA?$CF?$AAx?$AA?5@ 10005a00     fsl_rne_pdd_common_topaz_v1:rndis_pdd.obj
 0001:00004a5c       ??_C@_1DA@MJLPENBD@?$AAG?$AAo?$AAt?$AA?5?$AAS?$AAE?$AAT?$AAU?$AAP?$AA?5?$AAO?$AAU?$AAT?$AA?5?$AAp?$AAa?$AAc?$AAk?$AAe?$AAt?$AA?4?$AA?$AN?$AA?6?$AA?$AA@ 10005a5c     fsl_rne_pdd_common_topaz_v1:rndis_pdd.obj
 0001:00004a8c       ??_C@_1CM@NHNGDKFM@?$AAG?$AAo?$AAt?$AA?5?$AAS?$AAE?$AAT?$AAU?$AAP?$AA?5?$AAI?$AAN?$AA?5?$AAp?$AAa?$AAc?$AAk?$AAe?$AAt?$AA?$AN?$AA?6?$AA?$AA@ 10005a8c     fsl_rne_pdd_common_topaz_v1:rndis_pdd.obj
 0001:00004ab8       ??_C@_1DK@CJOHLCDF@?$AAE?$AAR?$AAR?$AAO?$AAR?$AA?5?$AAP?$AAA?$AAR?$AAS?$AAI?$AAN?$AAG?$AA?5?$AAS?$AAE?$AAT?$AAU?$AAP?$AA?5?$AAP?$AAA?$AAC?$AAK?$AAE?$AAT?$AA?$AN?$AA?6?$AA?$AA@ 10005ab8     fsl_rne_pdd_common_topaz_v1:rndis_pdd.obj
 0001:00004af4       ??_C@_1CO@MPAJKINN@?$AA?9?$AAR?$AAN?$AAD?$AAI?$AAS?$AA_?$AAU?$AAS?$AAB?$AAF?$AAN?$AA_?$AAP?$AAD?$AAD?$AAI?$AAn?$AAi?$AAt?$AA?$AN?$AA?6?$AA?$AA@ 10005af4     fsl_rne_pdd_common_topaz_v1:rndis_pdd.obj
 0001:00004b28       ??_C@_1GC@COEDNCDC@?$AA?5?$AAR?$AAN?$AAD?$AAI?$AAS?$AA_?$AAU?$AAS?$AAB?$AAF?$AAN?$AA_?$AAP?$AAD?$AAD?$AAI?$AAn?$AAi?$AAt?$AA?3?$AA?5?$AAi?$AAn?$AAi?$AAt?$AAi?$AAa?$AAl?$AAi?$AAz?$AAa@ 10005b28     fsl_rne_pdd_common_topaz_v1:rndis_pdd.obj
 0001:00004b8c       ??_C@_1CM@CGCNDLMD@?$AAU?$AAf?$AAn?$AAP?$AAd?$AAd?$AA_?$AAI?$AAn?$AAi?$AAt?$AA?5?$AAf?$AAa?$AAi?$AAl?$AAe?$AAd?$AA?$CB?$AA?$AN?$AA?6?$AA?$AA@ 10005b8c     fsl_rne_pdd_common_topaz_v1:rndis_pdd.obj
 0001:00004bb8       ??_C@_1DA@MNIGJPIF@?$AA?9?$AAR?$AAN?$AAD?$AAI?$AAS?$AA_?$AAU?$AAS?$AAB?$AAF?$AAN?$AA_?$AAP?$AAD?$AAD?$AAD?$AAe?$AAn?$AAi?$AAt?$AA?$AN?$AA?6?$AA?$AA@ 10005bb8     fsl_rne_pdd_common_topaz_v1:rndis_pdd.obj
 0001:00004be8       ??_C@_1DA@EACCPFEN@?$AA?$CL?$AAR?$AAN?$AAD?$AAI?$AAS?$AA_?$AAU?$AAS?$AAB?$AAF?$AAN?$AA_?$AAP?$AAD?$AAD?$AAD?$AAe?$AAn?$AAi?$AAt?$AA?$AN?$AA?6?$AA?$AA@ 10005be8     fsl_rne_pdd_common_topaz_v1:rndis_pdd.obj
 0001:00004c18       ??_C@_1EI@ONHOMNHJ@?$AA?9?$AAR?$AAN?$AAD?$AAI?$AAS?$AA_?$AAU?$AAS?$AAB?$AAF?$AAN?$AA_?$AAP?$AAD?$AAD?$AA_?$AAS?$AAe?$AAn?$AAd?$AAR?$AAn?$AAd?$AAi?$AAs?$AAM?$AAe?$AAs?$AAs?$AAa?$AAg@ 10005c18     fsl_rne_pdd_common_topaz_v1:rndis_pdd.obj
 0001:00004c60       ??_C@_1HE@PDJOEOPK@?$AA?$CL?$AAR?$AAN?$AAD?$AAI?$AAS?$AA_?$AAU?$AAS?$AAB?$AAF?$AAN?$AA_?$AAP?$AAD?$AAD?$AA_?$AAS?$AAe?$AAn?$AAd?$AAR?$AAn?$AAd?$AAi?$AAs?$AAM?$AAe?$AAs?$AAs?$AAa?$AAg@ 10005c60     fsl_rne_pdd_common_topaz_v1:rndis_pdd.obj
 0001:00004cd8       ??_C@_1GK@OCDDHLML@?$AA?$CL?$AAR?$AAN?$AAD?$AAI?$AAS?$AA_?$AAU?$AAS?$AAB?$AAF?$AAN?$AA_?$AAP?$AAD?$AAD?$AA_?$AAS?$AAe?$AAn?$AAd?$AAR?$AAn?$AAd?$AAi?$AAs?$AAM?$AAe?$AAs?$AAs?$AAa?$AAg@ 10005cd8     fsl_rne_pdd_common_topaz_v1:rndis_pdd.obj
 0001:00004d48       ??_C@_1EI@LPKHCIID@?$AA?$CL?$AAR?$AAN?$AAD?$AAI?$AAS?$AA_?$AAU?$AAS?$AAB?$AAF?$AAN?$AA_?$AAP?$AAD?$AAD?$AA_?$AAS?$AAe?$AAn?$AAd?$AAR?$AAn?$AAd?$AAi?$AAs?$AAM?$AAe?$AAs?$AAs?$AAa?$AAg@ 10005d48     fsl_rne_pdd_common_topaz_v1:rndis_pdd.obj
 0001:00004d90       ??_C@_1EG@FPFPIBJG@?$AA?9?$AAR?$AAN?$AAD?$AAI?$AAS?$AA_?$AAU?$AAS?$AAB?$AAF?$AAN?$AA_?$AAP?$AAD?$AAD?$AA_?$AAS?$AAe?$AAn?$AAd?$AAR?$AAn?$AAd?$AAi?$AAs?$AAP?$AAa?$AAc?$AAk?$AAe?$AAt@ 10005d90     fsl_rne_pdd_common_topaz_v1:rndis_pdd.obj
 0001:00004dd8       ??_C@_1FG@MIKLDILD@?$AA?$CK?$AA?$CK?$AA?$CK?$AA?$CK?$AAM?$AAu?$AAl?$AAt?$AAi?$AAp?$AAl?$AAe?$AA?5?$AAp?$AAe?$AAn?$AAd?$AAi?$AAn?$AAg?$AA?5?$AAs?$AAe?$AAn?$AAd?$AA?5?$AAr?$AAn?$AAd?$AAi?$AAs?$AA?5@ 10005dd8     fsl_rne_pdd_common_topaz_v1:rndis_pdd.obj
 0001:00004e30       ??_C@_1EI@PJCOBAOE@?$AAG?$AAo?$AAt?$AA?5?$AAS?$AAe?$AAn?$AAd?$AAP?$AAa?$AAc?$AAk?$AAe?$AAt?$AA?5?$AAR?$AAe?$AAq?$AAu?$AAe?$AAs?$AAt?$AA?5?$AA?$FL?$AA?$CF?$AAd?$AA?5?$AAb?$AAy?$AAt?$AAe?$AAs@ 10005e30     fsl_rne_pdd_common_topaz_v1:rndis_pdd.obj
 0001:00004e78       ??_C@_1EG@FDHKBGKN@?$AA?$CL?$AAR?$AAN?$AAD?$AAI?$AAS?$AA_?$AAU?$AAS?$AAB?$AAF?$AAN?$AA_?$AAP?$AAD?$AAD?$AA_?$AAS?$AAe?$AAn?$AAd?$AAR?$AAn?$AAd?$AAi?$AAs?$AAP?$AAa?$AAc?$AAk?$AAe?$AAt@ 10005e78     fsl_rne_pdd_common_topaz_v1:rndis_pdd.obj
 0001:00004ec0       ??_C@_1CO@MBMDAIGD@?$AA?9?$AAR?$AAN?$AAD?$AAI?$AAS?$AA_?$AAU?$AAS?$AAB?$AAF?$AAN?$AA_?$AAP?$AAD?$AAD?$AA_?$AAS?$AAe?$AAt?$AA?$AN?$AA?6?$AA?$AA@ 10005ec0     fsl_rne_pdd_common_topaz_v1:rndis_pdd.obj
 0001:00004ef0       ??_C@_1DO@PIKCPFME@?$AAP?$AAD?$AAD?$AA_?$AAS?$AAe?$AAt?$AA?3?$AAU?$AAn?$AAk?$AAn?$AAo?$AAw?$AAn?$AA?5?$AAr?$AAe?$AAq?$AAu?$AAe?$AAs?$AAt?$AA?3?$AA0?$AAx?$AA?$CF?$AAx?$AA?$AN?$AA?6?$AA?$AA@ 10005ef0     fsl_rne_pdd_common_topaz_v1:rndis_pdd.obj
 0001:00004f30       ??_C@_1DK@PGGKHLLK@?$AAP?$AAD?$AAD?$AA_?$AAS?$AAe?$AAt?$AA?3?$AAR?$AAE?$AAQ?$AA_?$AAI?$AAD?$AA_?$AAD?$AAI?$AAS?$AAA?$AAB?$AAL?$AAE?$AA_?$AAI?$AAN?$AAT?$AA?$AN?$AA?6?$AA?$AA@ 10005f30     fsl_rne_pdd_common_topaz_v1:rndis_pdd.obj
 0001:00004f6c       ??_C@_1DI@KFPGHMKG@?$AAP?$AAD?$AAD?$AA_?$AAS?$AAe?$AAt?$AA?3?$AAR?$AAE?$AAQ?$AA_?$AAI?$AAD?$AA_?$AAE?$AAN?$AAA?$AAB?$AAL?$AAE?$AA_?$AAI?$AAN?$AAT?$AA?$AN?$AA?6?$AA?$AA@ 10005f6c     fsl_rne_pdd_common_topaz_v1:rndis_pdd.obj
 0001:00004fa4       ??_C@_1DI@MFNCMIPE@?$AAP?$AAD?$AAD?$AA_?$AAS?$AAe?$AAt?$AA?3?$AAR?$AAE?$AAQ?$AA_?$AAI?$AAD?$AA_?$AAS?$AAO?$AAF?$AAT?$AA_?$AAR?$AAE?$AAS?$AAE?$AAT?$AA?$AN?$AA?6?$AA?$AA@ 10005fa4     fsl_rne_pdd_common_topaz_v1:rndis_pdd.obj
 0001:00004fdc       ??_C@_1DI@LPFOEPEC@?$AAP?$AAD?$AAD?$AA_?$AAS?$AAe?$AAt?$AA?3?$AAR?$AAE?$AAQ?$AA_?$AAI?$AAD?$AA_?$AAH?$AAA?$AAR?$AAD?$AA_?$AAR?$AAE?$AAS?$AAE?$AAT?$AA?$AN?$AA?6?$AA?$AA@ 10005fdc     fsl_rne_pdd_common_topaz_v1:rndis_pdd.obj
 0001:00005014       ??_C@_1CO@BKAHFHEI@?$AA?$CL?$AAR?$AAN?$AAD?$AAI?$AAS?$AA_?$AAU?$AAS?$AAB?$AAF?$AAN?$AA_?$AAP?$AAD?$AAD?$AA_?$AAS?$AAe?$AAt?$AA?$AN?$AA?6?$AA?$AA@ 10006014     fsl_rne_pdd_common_topaz_v1:rndis_pdd.obj
 0001:00005044       ??_C@_0BO@FJNCJEJP@Discard?5?$CFd?5Pending?5Messages?$AN?6?$AA@ 10006044     fsl_rne_pdd_common_topaz_v1:rndis_pdd.obj
 0001:00005064       ??_C@_1CO@MONNNOOA@?$AA?9?$AAR?$AAN?$AAD?$AAI?$AAS?$AA_?$AAU?$AAS?$AAB?$AAF?$AAN?$AA_?$AAP?$AAD?$AAD?$AA_?$AAG?$AAe?$AAt?$AA?$AN?$AA?6?$AA?$AA@ 10006064     fsl_rne_pdd_common_topaz_v1:rndis_pdd.obj
 0001:00005098       ??_C@_1EC@FCCAEHJA@?$AA?9?$AAP?$AAD?$AAD?$AA_?$AAG?$AAe?$AAt?$AA?3?$AA?5?$AAu?$AAn?$AAk?$AAn?$AAo?$AAw?$AAn?$AA?5?$AAr?$AAe?$AAq?$AAu?$AAe?$AAs?$AAt?$AA?5?$AA0?$AAx?$AA?$CF?$AAx?$AA?$AN?$AA?6@ 10006098     fsl_rne_pdd_common_topaz_v1:rndis_pdd.obj
 0001:000050dc       ??_C@_1CO@BFBJIBML@?$AA?$CL?$AAR?$AAN?$AAD?$AAI?$AAS?$AA_?$AAU?$AAS?$AAB?$AAF?$AAN?$AA_?$AAP?$AAD?$AAD?$AA_?$AAG?$AAe?$AAt?$AA?$AN?$AA?6?$AA?$AA@ 100060dc     fsl_rne_pdd_common_topaz_v1:rndis_pdd.obj
 0001:00005110       ??_C@_1FO@HIPGBBGN@?$AA?9?$AAR?$AAN?$AAD?$AAI?$AAS?$AA_?$AAU?$AAS?$AAB?$AAF?$AAN?$AA_?$AAP?$AAD?$AAD?$AA_?$AAI?$AAn?$AAd?$AAi?$AAc?$AAa?$AAt?$AAe?$AAR?$AAn?$AAd?$AAi?$AAs?$AAP?$AAa@ 10006110     fsl_rne_pdd_common_topaz_v1:rndis_pdd.obj
 0001:00005170       ??_C@_1FO@PLBKEBPA@?$AA?$CL?$AAR?$AAN?$AAD?$AAI?$AAS?$AA_?$AAU?$AAS?$AAB?$AAF?$AAN?$AA_?$AAP?$AAD?$AAD?$AA_?$AAI?$AAn?$AAd?$AAi?$AAc?$AAa?$AAt?$AAe?$AAR?$AAn?$AAd?$AAi?$AAs?$AAP?$AAa@ 10006170     fsl_rne_pdd_common_topaz_v1:rndis_pdd.obj
 0001:000051d0       ??_C@_1DG@LOIHLLKG@?$AAR?$AAN?$AAD?$AAI?$AAS?$AA?5?$AAS?$AAe?$AAr?$AAi?$AAa?$AAl?$AA?5?$AAN?$AAu?$AAm?$AAb?$AAe?$AAr?$AA?$DN?$AA?$FL?$AA?$CF?$AAs?$AA?$FN?$AA?$AN?$AA?6?$AA?$AA@ 100061d0     fsl_rne_pdd_common_topaz_v1:rndis_pdd.obj
 0001:00005208       ??_C@_1BC@GDFGLIEL@?$AAO?$AAT?$AAG?$AAG?$AAr?$AAo?$AAu?$AAp?$AA?$AA@ 10006208     usb_usbfn_mx25_topaz_v1:i_pdd.obj
 0001:0000521c       ??_C@_1BG@HHFAGDDC@?$AAO?$AAT?$AAG?$AAS?$AAu?$AAp?$AAp?$AAo?$AAr?$AAt?$AA?$AA@ 1000621c     usb_usbfn_mx25_topaz_v1:i_pdd.obj
 0001:00005234       ??_C@_1BI@BHLBGEOK@?$AAP?$AAr?$AAi?$AAo?$AAr?$AAi?$AAt?$AAy?$AA2?$AA5?$AA6?$AA?$AA@ 10006234     usb_usbfn_mx25_topaz_v1:i_pdd.obj
 0001:0000524c       ??_C@_17DJGGJCGD@?$AAI?$AAr?$AAq?$AA?$AA@ 1000624c     usb_usbfn_mx25_topaz_v1:i_pdd.obj
 0001:00005254       ??_C@_1O@LBBNFMDB@?$AAM?$AAe?$AAm?$AAL?$AAe?$AAn?$AA?$AA@ 10006254     usb_usbfn_mx25_topaz_v1:i_pdd.obj
 0001:00005264       ??_C@_1BA@INLDIDEN@?$AAM?$AAe?$AAm?$AAB?$AAa?$AAs?$AAe?$AA?$AA@ 10006264     usb_usbfn_mx25_topaz_v1:i_pdd.obj
 0001:00005398       ??_C@_1CM@IKIIJOLF@?$AAP?$AAo?$AAw?$AAe?$AAr?$AAD?$AAo?$AAw?$AAn?$AA?5?$AAc?$AAo?$AAm?$AAp?$AAl?$AAe?$AAt?$AAe?$AAd?$AA?$AN?$AA?6?$AA?$AA@ 10006398     usb_usbfn_mx25_topaz_v1:i_pdd.obj
 0001:000053c4       ??_C@_1CC@OEGDFOPI@?$AAU?$AAS?$AAB?$AA?5?$AAC?$AAl?$AAo?$AAc?$AAk?$AA?5?$AAs?$AAt?$AAo?$AAp?$AA?$AN?$AA?6?$AA?$AA@ 100063c4     usb_usbfn_mx25_topaz_v1:i_pdd.obj
 0001:000053e8       ??_C@_1DC@MJCJJIDL@?$AAP?$AAo?$AAw?$AAe?$AAr?$AAD?$AAo?$AAw?$AAn?$AA?5?$AAU?$AAS?$AAB?$AAC?$AAT?$AAR?$AAL?$AA?$DN?$AA0?$AAx?$AA?$CF?$AAx?$AA?$AN?$AA?6?$AA?$AA@ 100063e8     usb_usbfn_mx25_topaz_v1:i_pdd.obj
 0001:0000541c       ??_C@_1DC@NJODNJCA@?$AAP?$AAo?$AAw?$AAe?$AAr?$AAD?$AAo?$AAw?$AAn?$AA?5?$AAP?$AAO?$AAR?$AAT?$AAS?$AAC?$AA?$DN?$AA?5?$AA0?$AAx?$AA?$CF?$AAx?$AA?$AN?$AA?6?$AA?$AA@ 1000641c     usb_usbfn_mx25_topaz_v1:i_pdd.obj
 0001:00005450       ??_C@_1DG@NJOCHJMF@?$AAP?$AAo?$AAw?$AAe?$AAr?$AAD?$AAo?$AAw?$AAn?$AA?5?$AAU?$AAS?$AAB?$AAI?$AAN?$AAT?$AAR?$AA?5?$AA?$DN?$AA?5?$AA0?$AAx?$AA?$CF?$AAx?$AA?$AN?$AA?6?$AA?$AA@ 10006450     usb_usbfn_mx25_topaz_v1:i_pdd.obj
 0001:00005488       ??_C@_1DE@CFOAAIJP@?$AAP?$AAo?$AAw?$AAe?$AAr?$AAD?$AAo?$AAw?$AAn?$AA?5?$AAU?$AAS?$AAB?$AAC?$AAM?$AAD?$AA?5?$AA?$DN?$AA?5?$AA0?$AAx?$AA?$CF?$AAx?$AA?$AN?$AA?6?$AA?$AA@ 10006488     usb_usbfn_mx25_topaz_v1:i_pdd.obj
 0001:000054c0       ??_C@_1EM@IEDMFFDN@?$AAU?$AAf?$AAn?$AAP?$AAd?$AAd?$AA_?$AAP?$AAo?$AAw?$AAe?$AAr?$AAD?$AAo?$AAw?$AAn?$AA?5?$AAn?$AAo?$AA?5?$AAa?$AAc?$AAt?$AAi?$AAo?$AAn?$AA?5?$AAr?$AAe?$AAq?$AAu?$AAi@ 100064c0     usb_usbfn_mx25_topaz_v1:i_pdd.obj
 0001:0000550c       ??_C@_1CG@OIILOOGO@?$AAU?$AAs?$AAb?$AAP?$AAd?$AAd?$AA_?$AAP?$AAo?$AAw?$AAe?$AAr?$AAD?$AAo?$AAw?$AAn?$AA?$AN?$AA?6?$AA?$AA@ 1000650c     usb_usbfn_mx25_topaz_v1:i_pdd.obj
 0001:00005534       ??_C@_1DA@KMOKCFJD@?$AAP?$AAo?$AAw?$AAe?$AAr?$AAU?$AAp?$AA?5?$AAU?$AAS?$AAB?$AAC?$AAM?$AAD?$AA?5?$AA?$DN?$AA?5?$AA0?$AAx?$AA?$CF?$AAx?$AA?$AN?$AA?6?$AA?$AA@ 10006534     usb_usbfn_mx25_topaz_v1:i_pdd.obj
 0001:00005568       ??_C@_1EA@HIDFOGGD@?$AAW?$AAa?$AAk?$AAe?$AAu?$AAp?$AA?5?$AAI?$AAn?$AAt?$AAe?$AAr?$AAr?$AAu?$AAp?$AAt?$AA?5?$AAS?$AAe?$AAt?$AAt?$AAi?$AAn?$AAg?$AA?5?$AA0?$AAx?$AA?$CF?$AAx?$AA?$AN?$AA?6?$AA?$AA@ 10006568     usb_usbfn_mx25_topaz_v1:i_pdd.obj
 0001:000055a8       ??_C@_1DA@ODLPFKGM@?$AAP?$AAo?$AAw?$AAe?$AAr?$AAU?$AAp?$AA?5?$AAw?$AAa?$AAk?$AAe?$AAu?$AAp?$AA?5?$AA?$DN?$AA?5?$AA0?$AAx?$AA?$CF?$AAx?$AA?$AN?$AA?6?$AA?$AA@ 100065a8     usb_usbfn_mx25_topaz_v1:i_pdd.obj
 0001:000055d8       ??_C@_1BO@JBMLODEA@?$AAF?$AAo?$AAr?$AAc?$AAe?$AA?5?$AAr?$AAe?$AAs?$AAu?$AAm?$AAe?$AA?$AN?$AA?6?$AA?$AA@ 100065d8     usb_usbfn_mx25_topaz_v1:i_pdd.obj
 0001:000055f8       ??_C@_1EI@LEEJEJNJ@?$AAP?$AAo?$AAw?$AAe?$AAr?$AAU?$AAp?$AA?3?$AAU?$AAS?$AAB?$AAS?$AAT?$AAS?$AA?$CI?$AA0?$AAx?$AA?$CF?$AAx?$AA?$CJ?$AA?5?$AAP?$AAO?$AAR?$AAT?$AAS?$AAC?$AA?$CI?$AA0?$AAx?$AA?$CF?$AAx@ 100065f8     usb_usbfn_mx25_topaz_v1:i_pdd.obj
 0001:00005640       ??_C@_1CE@HMNFKKGB@?$AAU?$AAS?$AAB?$AA?5?$AAC?$AAl?$AAo?$AAc?$AAk?$AA?5?$AAs?$AAt?$AAa?$AAr?$AAt?$AA?$AN?$AA?6?$AA?$AA@ 10006640     usb_usbfn_mx25_topaz_v1:i_pdd.obj
 0001:00005668       ??_C@_1EE@FMEOMODP@?$AAU?$AAs?$AAb?$AAP?$AAd?$AAd?$AA_?$AAP?$AAo?$AAw?$AAe?$AAr?$AAU?$AAp?$AA?5?$AAw?$AAi?$AAt?$AAh?$AA?5?$AAb?$AAI?$AAn?$AAU?$AAS?$AAB?$AAF?$AAN?$AA?5?$AA?$CF?$AAd?$AA?$AN@ 10006668     usb_usbfn_mx25_topaz_v1:i_pdd.obj
 0001:000056b0       ??_C@_1EC@POPMIGGA@?$AAU?$AAp?$AAd?$AAa?$AAt?$AAe?$AAD?$AAe?$AAv?$AAi?$AAc?$AAe?$AAP?$AAo?$AAw?$AAe?$AAr?$AA?5?$AAt?$AAo?$AA?5?$AAp?$AAo?$AAw?$AAe?$AAr?$AAd?$AAo?$AAw?$AAn?$AA?$AN?$AA?6@ 100066b0     usb_usbfn_mx25_topaz_v1:i_pdd.obj
 0001:000056f4       ??_C@_1DO@CFDCODDO@?$AAU?$AAp?$AAd?$AAa?$AAt?$AAe?$AAD?$AAe?$AAv?$AAi?$AAc?$AAe?$AAP?$AAo?$AAw?$AAe?$AAr?$AA?5?$AAt?$AAo?$AA?5?$AAp?$AAo?$AAw?$AAe?$AAr?$AAu?$AAp?$AA?$AN?$AA?6?$AA?$AA@ 100066f4     usb_usbfn_mx25_topaz_v1:i_pdd.obj
 0001:00005738       ??_C@_1FE@DIHLBJLK@?$AAU?$AAp?$AAd?$AAa?$AAt?$AAe?$AAD?$AAe?$AAv?$AAi?$AAc?$AAe?$AAP?$AAo?$AAw?$AAe?$AAr?$AA?5?$AAG?$AAo?$AAi?$AAn?$AAg?$AA?5?$AAf?$AAr?$AAo?$AAm?$AA?5?$AAD?$AA?$CF?$AAd@ 10006738     usb_usbfn_mx25_topaz_v1:i_pdd.obj
 0001:00005790       ??_C@_1KO@LDNIEBB@?$AAC?$AA?3?$AA?2?$AAW?$AAI?$AAN?$AAC?$AAE?$AAR?$AAO?$AAO?$AAT?$AAS?$AA?2?$AAT?$AAo?$AAp?$AAa?$AAz?$AA?2?$AAW?$AAI?$AAN?$AAC?$AAE?$AA6?$AA0?$AA0?$AA?2?$AAp?$AAl?$AAa@ 10006790     usb_usbfn_mx25_topaz_v1:i_pdd.obj
 0001:00005840       ??_C@_1BO@LJJCCAKA@?$AAS?$AAe?$AAt?$AAu?$AAp?$AA?3?$AA?5?$AA?$CF?$AAx?$AA?5?$AA?$CF?$AAx?$AA?$AN?$AA?6?$AA?$AA@ 10006840     usb_usbfn_mx25_topaz_v1:i_pdd.obj
 0001:00005860       ??_C@_1CA@NAJOELH@?$AAD?$AAe?$AAv?$AAi?$AAc?$AAe?$AA?5?$AAA?$AAt?$AAt?$AAa?$AAc?$AAh?$AA?$AN?$AA?6?$AA?$AA@ 10006860     usb_usbfn_mx25_topaz_v1:i_pdd.obj
 0001:00005880       ??_C@_1IE@MBNKMJA@?$AA?$CD?$AA?$CD?$AA?$CD?$AA?$CD?$AA?$CD?$AA?$CD?$AA?$CD?$AA?5?$AAG?$AAe?$AAt?$AAS?$AAe?$AAt?$AAu?$AAp?$AAP?$AAa?$AAc?$AAk?$AAe?$AAt?$AA?3?$AA?5?$AAF?$AAl?$AAu?$AAs?$AAh?$AAi?$AAn?$AAg@ 10006880     usb_usbfn_mx25_topaz_v1:i_pdd.obj
 0001:00005908       ??_C@_1KK@KOKNNFID@?$AA?$CD?$AA?$CD?$AA?$CD?$AA?$CD?$AA?$CD?$AA?$CD?$AA?$CD?$AA?5?$AAG?$AAe?$AAt?$AAS?$AAe?$AAt?$AAu?$AAp?$AAP?$AAa?$AAc?$AAk?$AAe?$AAt?$AA?3?$AA?5?$AAT?$AAr?$AAa?$AAn?$AAs?$AAf?$AAe?$AAr@ 10006908     usb_usbfn_mx25_topaz_v1:i_pdd.obj
 0001:000059b4       ??_C@_1DM@JOKNMMI@?$AAG?$AAe?$AAt?$AAS?$AAe?$AAt?$AAu?$AAp?$AAP?$AAa?$AAc?$AAk?$AAe?$AAt?$AA?5?$AA?$CF?$AA8?$AA?4?$AA8?$AAl?$AAx?$AA?$CF?$AA8?$AA?4?$AA8?$AAl?$AAx?$AA?$AN?$AA?6?$AA?$AA@ 100069b4     usb_usbfn_mx25_topaz_v1:i_pdd.obj
 0001:000059f0       ??_C@_1DM@PINNGIJL@?$AA?7?$AA?7?$AA?7?$AAS?$AAe?$AAr?$AAi?$AAa?$AAl?$AA?1?$AA1?$AA?4?$AA1?$AA?5?$AAP?$AAH?$AAY?$AA?5?$AA?$CI?$AAF?$AAS?$AA?5?$AAO?$AAn?$AAl?$AAy?$AA?$CJ?$AA?$AN?$AA?6?$AA?$AA@ 100069f0     usb_usbfn_mx25_topaz_v1:i_pdd.obj
 0001:00005a2c       ??_C@_1BE@OHMKGMAA@?$AA?7?$AA?7?$AA?7?$AAU?$AAL?$AAP?$AAI?$AA?$AN?$AA?6?$AA?$AA@ 10006a2c     usb_usbfn_mx25_topaz_v1:i_pdd.obj
 0001:00005a40       ??_C@_1CK@JDCKMGFE@?$AA?7?$AA?7?$AA?7?$AAP?$AAh?$AAi?$AAl?$AAi?$AAp?$AAs?$AA?5?$AAC?$AAl?$AAa?$AAs?$AAs?$AAi?$AAc?$AA?$AN?$AA?6?$AA?$AA@ 10006a40     usb_usbfn_mx25_topaz_v1:i_pdd.obj
 0001:00005a6c       ??_C@_1CA@GIFIBBC@?$AA?7?$AA?7?$AA?7?$AAU?$AAT?$AAM?$AAI?$AA?1?$AAU?$AAT?$AAM?$AAI?$AA?$CL?$AA?$AN?$AA?6?$AA?$AA@ 10006a6c     usb_usbfn_mx25_topaz_v1:i_pdd.obj
 0001:00005a90       ??_C@_1EG@GEPPEHI@?$AA?7?$AA?7?$AAP?$AAa?$AAr?$AAa?$AAl?$AAl?$AAe?$AAl?$AA?5?$AAT?$AAr?$AAa?$AAn?$AAs?$AAc?$AAe?$AAi?$AAv?$AAe?$AAr?$AA?5?$AAS?$AAe?$AAl?$AAe?$AAc?$AAt?$AA?3?$AA?$CF?$AAx@ 10006a90     usb_usbfn_mx25_topaz_v1:i_pdd.obj
 0001:00005ad8       ??_C@_1DO@GOALHOBG@?$AA?7?$AA?7?$AAS?$AAe?$AAr?$AAi?$AAa?$AAl?$AA?5?$AAT?$AAr?$AAa?$AAn?$AAs?$AAc?$AAe?$AAi?$AAv?$AAe?$AAr?$AA?5?$AAS?$AAe?$AAl?$AAe?$AAc?$AAt?$AA?5?$AA?$AN?$AA?6?$AA?$AA@ 10006ad8     usb_usbfn_mx25_topaz_v1:i_pdd.obj
 0001:00005b18       ??_C@_1BI@PMFMKPBN@?$AA?7?$AA?7?$AA?7?$AA8?$AA?5?$AAb?$AAi?$AAt?$AAs?$AA?$AN?$AA?6?$AA?$AA@ 10006b18     usb_usbfn_mx25_topaz_v1:i_pdd.obj
 0001:00005b30       ??_C@_1BK@DMIJGPDB@?$AA?7?$AA?7?$AA?7?$AA1?$AA6?$AA?5?$AAb?$AAi?$AAt?$AAs?$AA?$AN?$AA?6?$AA?$AA@ 10006b30     usb_usbfn_mx25_topaz_v1:i_pdd.obj
 0001:00005b50       ??_C@_1EE@PJPHJMEN@?$AA?7?$AA?7?$AAP?$AAa?$AAr?$AAa?$AAl?$AAl?$AAe?$AAl?$AA?5?$AAT?$AAr?$AAa?$AAn?$AAs?$AAc?$AAe?$AAi?$AAv?$AAe?$AAr?$AA?5?$AAW?$AAi?$AAd?$AAt?$AAh?$AA?3?$AA?$CF?$AAx?$AA?9@ 10006b50     usb_usbfn_mx25_topaz_v1:i_pdd.obj
 0001:00005b94       ??_C@_1CA@CFDEDDEG@?$AA?7?$AA?7?$AA?7?$AAH?$AAi?$AAg?$AAh?$AA?5?$AAS?$AAp?$AAe?$AAe?$AAd?$AA?$AN?$AA?6?$AA?$AA@ 10006b94     usb_usbfn_mx25_topaz_v1:i_pdd.obj
 0001:00005bb4       ??_C@_1BO@DONMFABC@?$AA?7?$AA?7?$AA?7?$AAL?$AAo?$AAw?$AA?5?$AAS?$AAp?$AAe?$AAe?$AAd?$AA?$AN?$AA?6?$AA?$AA@ 10006bb4     usb_usbfn_mx25_topaz_v1:i_pdd.obj
 0001:00005bd4       ??_C@_1CA@EFHFHOIO@?$AA?7?$AA?7?$AA?7?$AAF?$AAu?$AAl?$AAl?$AA?5?$AAS?$AAp?$AAe?$AAe?$AAd?$AA?$AN?$AA?6?$AA?$AA@ 10006bd4     usb_usbfn_mx25_topaz_v1:i_pdd.obj
 0001:00005bf4       ??_C@_1CG@DLDJDNPN@?$AA?7?$AA?7?$AAP?$AAo?$AAr?$AAt?$AA?5?$AAS?$AAp?$AAe?$AAe?$AAd?$AA?3?$AA?5?$AA?$CF?$AAx?$AA?9?$AA?$DO?$AA?$AA@ 10006bf4     usb_usbfn_mx25_topaz_v1:i_pdd.obj
 0001:00005c20       ??_C@_1EG@FLKCNOK@?$AA?7?$AA?7?$AAP?$AAo?$AAr?$AAt?$AA?5?$AAF?$AAo?$AAr?$AAc?$AAe?$AA?5?$AAF?$AAu?$AAl?$AAl?$AA?5?$AAS?$AAp?$AAe?$AAe?$AAd?$AA?5?$AAC?$AAo?$AAn?$AAn?$AAe?$AAc?$AAt?$AA?5@ 10006c20     usb_usbfn_mx25_topaz_v1:i_pdd.obj
 0001:00005c68       ??_C@_1GI@HKEGLKNC@?$AA?7?$AA?7?$AAP?$AAH?$AAY?$AA?5?$AAL?$AAo?$AAw?$AA?5?$AAP?$AAo?$AAw?$AAe?$AAr?$AA?5?$AAS?$AAu?$AAs?$AAp?$AAe?$AAn?$AAd?$AA?5?$AA?9?$AA?5?$AAC?$AAl?$AAo?$AAc?$AAk?$AA?5@ 10006c68     usb_usbfn_mx25_topaz_v1:i_pdd.obj
 0001:00005cd0       ??_C@_1FE@PECIMICA@?$AA?7?$AA?7?$AAW?$AAa?$AAk?$AAe?$AA?5?$AAo?$AAn?$AA?5?$AAO?$AAv?$AAe?$AAr?$AA?9?$AAc?$AAu?$AAr?$AAr?$AAe?$AAn?$AAt?$AA?5?$AAE?$AAn?$AAa?$AAb?$AAl?$AAe?$AA?5?$AA?$CI?$AAW@ 10006cd0     usb_usbfn_mx25_topaz_v1:i_pdd.obj
 0001:00005d28       ??_C@_1FI@KPMEKFHG@?$AA?7?$AA?7?$AAW?$AAa?$AAk?$AAe?$AA?5?$AAo?$AAn?$AA?5?$AAD?$AAi?$AAs?$AAc?$AAo?$AAn?$AAn?$AAe?$AAc?$AAt?$AA?5?$AAE?$AAn?$AAa?$AAb?$AAl?$AAe?$AA?5?$AA?$CI?$AAW?$AAK?$AAD@ 10006d28     usb_usbfn_mx25_topaz_v1:i_pdd.obj
 0001:00005d80       ??_C@_1EM@HPIOFCNI@?$AA?7?$AA?7?$AAW?$AAa?$AAk?$AAe?$AA?5?$AAo?$AAn?$AA?5?$AAC?$AAo?$AAn?$AAn?$AAe?$AAc?$AAt?$AA?5?$AAE?$AAn?$AAa?$AAb?$AAl?$AAe?$AA?5?$AA?$CI?$AAW?$AAK?$AAC?$AAN?$AAN?$AAT@ 10006d80     usb_usbfn_mx25_topaz_v1:i_pdd.obj
 0001:00005dcc       ??_C@_1DE@NJCPBMGI@?$AA?7?$AA?7?$AAP?$AAo?$AAr?$AAt?$AA?5?$AAT?$AAe?$AAs?$AAt?$AA?5?$AAC?$AAo?$AAn?$AAt?$AAr?$AAo?$AAl?$AA?3?$AA?5?$AA?$CF?$AAx?$AA?$AN?$AA?6?$AA?$AA@ 10006dcc     usb_usbfn_mx25_topaz_v1:i_pdd.obj
 0001:00005e00       ??_C@_1BG@LAPJBFLO@?$AA?7?$AA?7?$AA?7?$AAG?$AAr?$AAe?$AAe?$AAn?$AA?$AN?$AA?6?$AA?$AA@ 10006e00     usb_usbfn_mx25_topaz_v1:i_pdd.obj
 0001:00005e18       ??_C@_1BG@IMMCDJCL@?$AA?7?$AA?7?$AA?7?$AAA?$AAm?$AAb?$AAe?$AAr?$AA?$AN?$AA?6?$AA?$AA@ 10006e18     usb_usbfn_mx25_topaz_v1:i_pdd.obj
 0001:00005e30       ??_C@_1DC@IPGABND@?$AA?7?$AA?7?$AAP?$AAo?$AAr?$AAt?$AA?5?$AAI?$AAn?$AAd?$AAi?$AAc?$AAa?$AAt?$AAo?$AAr?$AA?5?$AAC?$AAo?$AAn?$AAt?$AAr?$AAo?$AAl?$AA?$AA@ 10006e30     usb_usbfn_mx25_topaz_v1:i_pdd.obj
 0001:00005e64       ??_C@_1BO@FPLCLNEP@?$AA?7?$AA?7?$AAP?$AAo?$AAr?$AAt?$AA?5?$AAO?$AAw?$AAn?$AAe?$AAr?$AA?$AN?$AA?6?$AA?$AA@ 10006e64     usb_usbfn_mx25_topaz_v1:i_pdd.obj
 0001:00005e84       ??_C@_1DO@MCLJLJA@?$AA?7?$AA?7?$AA?$DP?$AA?$DP?$AA?$DP?$AA?5?$AAS?$AAh?$AAo?$AAu?$AAl?$AAd?$AA?5?$AAb?$AAe?$AA?5?$AA0?$AA?5?$AAf?$AAo?$AAr?$AA?5?$AAd?$AAe?$AAv?$AAi?$AAc?$AAe?$AA?$AN?$AA?6?$AA?$AA@ 10006e84     usb_usbfn_mx25_topaz_v1:i_pdd.obj
 0001:00005ec4       ??_C@_1BO@CGJIBKMJ@?$AA?7?$AA?7?$AA?7?$AAU?$AAn?$AAd?$AAe?$AAf?$AAi?$AAn?$AAe?$AAd?$AA?$AN?$AA?6?$AA?$AA@ 10006ec4     usb_usbfn_mx25_topaz_v1:i_pdd.obj
 0001:00005ee4       ??_C@_1BK@LEBDPOFP@?$AA?7?$AA?7?$AA?7?$AAK?$AA?9?$AAs?$AAt?$AAa?$AAt?$AAe?$AA?$AN?$AA?6?$AA?$AA@ 10006ee4     usb_usbfn_mx25_topaz_v1:i_pdd.obj
 0001:00005f00       ??_C@_1BK@NBHEMFBJ@?$AA?7?$AA?7?$AA?7?$AAJ?$AA?9?$AAs?$AAt?$AAa?$AAt?$AAe?$AA?$AN?$AA?6?$AA?$AA@ 10006f00     usb_usbfn_mx25_topaz_v1:i_pdd.obj
 0001:00005f1c       ??_C@_1BC@HGFCDNBO@?$AA?7?$AA?7?$AA?7?$AAS?$AAE?$AA0?$AA?$AN?$AA?6?$AA?$AA@ 10006f1c     usb_usbfn_mx25_topaz_v1:i_pdd.obj
 0001:00005f30       ??_C@_1CE@HKBMNK@?$AA?7?$AA?7?$AAL?$AAi?$AAn?$AAe?$AA?5?$AAS?$AAt?$AAa?$AAt?$AAu?$AAs?$AA?3?$AA?5?$AA?$CF?$AAx?$AA?$AA@ 10006f30     usb_usbfn_mx25_topaz_v1:i_pdd.obj
 0001:00005f54       ??_C@_1CK@KAKGINHH@?$AA?7?$AA?7?$AAH?$AAi?$AAg?$AAh?$AA?9?$AAS?$AAp?$AAe?$AAe?$AAd?$AA?5?$AAP?$AAo?$AAr?$AAt?$AA?5?$AA?$AN?$AA?6?$AA?$AA@ 10006f54     usb_usbfn_mx25_topaz_v1:i_pdd.obj
 0001:00005f80       ??_C@_1BO@GDNLNMNM@?$AA?7?$AA?7?$AAP?$AAo?$AAr?$AAt?$AA?5?$AAR?$AAe?$AAs?$AAe?$AAt?$AA?$AN?$AA?6?$AA?$AA@ 10006f80     usb_usbfn_mx25_topaz_v1:i_pdd.obj
 0001:00005fa0       ??_C@_1BI@BCOEFLFO@?$AA?7?$AA?7?$AAS?$AAu?$AAs?$AAp?$AAe?$AAn?$AAd?$AA?$AN?$AA?6?$AA?$AA@ 10006fa0     usb_usbfn_mx25_topaz_v1:i_pdd.obj
 0001:00005fb8       ??_C@_1CM@LOGLIGHF@?$AA?7?$AA?7?$AAF?$AAo?$AAr?$AAc?$AAe?$AA?5?$AAP?$AAo?$AAr?$AAt?$AA?5?$AAR?$AAe?$AAs?$AAu?$AAm?$AAe?$AA?$AN?$AA?6?$AA?$AA@ 10006fb8     usb_usbfn_mx25_topaz_v1:i_pdd.obj
 0001:00005fe4       ??_C@_1DA@IPBKEGAM@?$AA?7?$AA?7?$AAO?$AAv?$AAe?$AAr?$AA?9?$AAc?$AAu?$AAr?$AAr?$AAe?$AAn?$AAt?$AA?5?$AAC?$AAh?$AAa?$AAn?$AAg?$AAe?$AA?$AN?$AA?6?$AA?$AA@ 10006fe4     usb_usbfn_mx25_topaz_v1:i_pdd.obj
 0001:00006014       ??_C@_1DA@IOPAFHGK@?$AA?7?$AA?7?$AAO?$AAv?$AAe?$AAr?$AA?9?$AAc?$AAu?$AAr?$AAr?$AAe?$AAn?$AAt?$AA?5?$AAA?$AAc?$AAt?$AAi?$AAv?$AAe?$AA?$AN?$AA?6?$AA?$AA@ 10007014     usb_usbfn_mx25_topaz_v1:i_pdd.obj
 0001:00006044       ??_C@_1DO@IDEEGAC@?$AA?7?$AA?7?$AAP?$AAo?$AAr?$AAt?$AA?5?$AAE?$AAn?$AAa?$AAb?$AAl?$AAe?$AA?1?$AAD?$AAi?$AAs?$AAa?$AAb?$AAl?$AAe?$AA?5?$AAC?$AAh?$AAa?$AAn?$AAg?$AAe?$AA?$AN?$AA?6?$AA?$AA@ 10007044     usb_usbfn_mx25_topaz_v1:i_pdd.obj
 0001:00006084       ??_C@_1CC@HIBPLHBD@?$AA?7?$AA?7?$AAP?$AAo?$AAr?$AAt?$AA?5?$AAE?$AAn?$AAa?$AAb?$AAl?$AAe?$AAd?$AA?$AN?$AA?6?$AA?$AA@ 10007084     usb_usbfn_mx25_topaz_v1:i_pdd.obj
 0001:000060a8       ??_C@_1EG@CHIFACHN@?$AA?7?$AA?7?$AAC?$AAo?$AAn?$AAn?$AAe?$AAc?$AAt?$AA?5?$AAS?$AAt?$AAa?$AAt?$AAu?$AAs?$AA?5?$AAC?$AAh?$AAa?$AAn?$AAg?$AAe?$AA?3?$AA?5?$AAC?$AAh?$AAa?$AAn?$AAg?$AAe?$AAd@ 100070a8     usb_usbfn_mx25_topaz_v1:i_pdd.obj
 0001:000060f0       ??_C@_1EK@CIGPBIFB@?$AA?7?$AA?7?$AAC?$AAu?$AAr?$AAr?$AAe?$AAn?$AAt?$AA?5?$AAC?$AAo?$AAn?$AAn?$AAe?$AAc?$AAt?$AA?5?$AAS?$AAt?$AAa?$AAt?$AAu?$AAs?$AA?3?$AA?5?$AAA?$AAt?$AAt?$AAa?$AAc?$AAh@ 100070f0     usb_usbfn_mx25_topaz_v1:i_pdd.obj
 0001:00006140       ??_C@_1EE@NKEDAIOG@?$AA?7?$AAA?$AAs?$AAy?$AAn?$AAc?$AAh?$AAr?$AAo?$AAn?$AAo?$AAu?$AAs?$AA?5?$AAS?$AAc?$AAh?$AAe?$AAd?$AAu?$AAl?$AAe?$AA?5?$AAS?$AAt?$AAa?$AAt?$AAu?$AAs?$AA?4?$AA?5?$AA?$AN@ 10007140     usb_usbfn_mx25_topaz_v1:i_pdd.obj
 0001:00006184       ??_C@_1DM@OLIDMOLB@?$AA?7?$AAP?$AAe?$AAr?$AAi?$AAo?$AAd?$AAi?$AAc?$AA?5?$AAS?$AAc?$AAh?$AAe?$AAd?$AAu?$AAl?$AAe?$AA?5?$AAS?$AAt?$AAa?$AAt?$AAu?$AAs?$AA?4?$AA?5?$AA?$AN?$AA?6?$AA?$AA@ 10007184     usb_usbfn_mx25_topaz_v1:i_pdd.obj
 0001:000061c0       ??_C@_1GE@JMEHEIAD@?$AA?7?$AAR?$AAe?$AAc?$AAl?$AAa?$AAm?$AAa?$AAt?$AAi?$AAo?$AAn?$AA?0?$AAO?$AAn?$AAl?$AAy?$AA?5?$AAu?$AAs?$AAe?$AAd?$AA?5?$AAb?$AAy?$AA?5?$AAt?$AAh?$AAe?$AA?5?$AAh?$AAo@ 100071c0     usb_usbfn_mx25_topaz_v1:i_pdd.obj
 0001:00006224       ??_C@_1BK@HBEGAPL@?$AA?7?$AAH?$AAC?$AAH?$AAa?$AAI?$AAt?$AAe?$AAd?$AA?5?$AA?$AN?$AA?6?$AA?$AA@ 10007224     usb_usbfn_mx25_topaz_v1:i_pdd.obj
 0001:00006240       ??_C@_1CE@IIMNHGIF@?$AA?7?$AAU?$AAL?$AAP?$AAI?$AA?5?$AAI?$AAn?$AAt?$AAe?$AAr?$AAr?$AAu?$AAp?$AAt?$AA?$AN?$AA?6?$AA?$AA@ 10007240     usb_usbfn_mx25_topaz_v1:i_pdd.obj
 0001:00006264       ??_C@_1BM@JKFMOBOF@?$AA?7?$AAD?$AAC?$AAS?$AAu?$AAs?$AAp?$AAe?$AAn?$AAd?$AA?5?$AA?$AN?$AA?6?$AA?$AA@ 10007264     usb_usbfn_mx25_topaz_v1:i_pdd.obj
 0001:00006280       ??_C@_1CC@ILIGGFI@?$AA?7?$AAS?$AAO?$AAF?$AA?5?$AAR?$AAe?$AAc?$AAe?$AAi?$AAv?$AAe?$AAd?$AA?5?$AA?$AN?$AA?6?$AA?$AA@ 10007280     usb_usbfn_mx25_topaz_v1:i_pdd.obj
 0001:000062a4       ??_C@_1CO@KLBBIGDH@?$AA?7?$AAU?$AAS?$AAB?$AA?5?$AAR?$AAe?$AAs?$AAe?$AAt?$AA?5?$AAR?$AAe?$AAc?$AAe?$AAi?$AAv?$AAe?$AAd?$AA?5?$AA?$AN?$AA?6?$AA?$AA@ 100072a4     usb_usbfn_mx25_topaz_v1:i_pdd.obj
 0001:000062d4       ??_C@_1DM@GMIDHHHN@?$AA?7?$AAI?$AAn?$AAt?$AAe?$AAr?$AAr?$AAu?$AAp?$AAt?$AA?5?$AAo?$AAn?$AA?5?$AAA?$AAs?$AAy?$AAn?$AAc?$AA?5?$AAA?$AAd?$AAv?$AAa?$AAn?$AAc?$AAe?$AA?$AN?$AA?6?$AA?$AA@ 100072d4     usb_usbfn_mx25_topaz_v1:i_pdd.obj
 0001:00006310       ??_C@_1CA@OPJKBAE@?$AA?7?$AAS?$AAy?$AAs?$AAt?$AAe?$AAm?$AA?5?$AAE?$AAr?$AAr?$AAo?$AAr?$AA?$AN?$AA?6?$AA?$AA@ 10007310     usb_usbfn_mx25_topaz_v1:i_pdd.obj
 0001:00006330       ??_C@_1CO@ONBPMBE@?$AA?7?$AAF?$AAr?$AAa?$AAm?$AAe?$AA?5?$AAL?$AAi?$AAs?$AAt?$AA?5?$AAR?$AAo?$AAl?$AAl?$AAo?$AAv?$AAe?$AAr?$AA?$AN?$AA?6?$AA?$AA@ 10007330     usb_usbfn_mx25_topaz_v1:i_pdd.obj
 0001:00006360       ??_C@_1CM@BOJMIELL@?$AA?7?$AAP?$AAo?$AAr?$AAt?$AA?5?$AAC?$AAh?$AAa?$AAn?$AAg?$AAe?$AA?5?$AAD?$AAe?$AAt?$AAe?$AAc?$AAt?$AA?$AN?$AA?6?$AA?$AA@ 10007360     usb_usbfn_mx25_topaz_v1:i_pdd.obj
 0001:00006390       ??_C@_1EG@JNFJCNAA@?$AA?7?$AAU?$AAS?$AAB?$AA?5?$AAE?$AAr?$AAr?$AAo?$AAr?$AA?5?$AAI?$AAn?$AAt?$AAe?$AAr?$AAr?$AAu?$AAp?$AAt?$AA?5?$AA?$CI?$AAU?$AAS?$AAB?$AAE?$AAR?$AAR?$AAI?$AAN?$AAT?$AA?$CJ@ 10007390     usb_usbfn_mx25_topaz_v1:i_pdd.obj
 0001:000063d8       ??_C@_1DE@KHLIMFPA@?$AA?7?$AAU?$AAS?$AAB?$AA?5?$AAI?$AAn?$AAt?$AAe?$AAr?$AAr?$AAu?$AAp?$AAt?$AA?5?$AA?$CI?$AAU?$AAS?$AAB?$AAI?$AAN?$AAT?$AA?$CJ?$AA?$AN?$AA?6?$AA?$AA@ 100073d8     usb_usbfn_mx25_topaz_v1:i_pdd.obj
 0001:0000640c       ??_C@_1DG@EIGILMMI@?$AAI?$AAN?$AA?5?$AA?$CF?$AAs?$AA?5?$AAC?$AAo?$AAm?$AAp?$AAl?$AAe?$AAt?$AAe?$AAd?$AA?5?$AAa?$AAt?$AA?5?$AAe?$AAp?$AA?5?$AA?$CF?$AAd?$AA?$AN?$AA?6?$AA?$AA@ 1000740c     usb_usbfn_mx25_topaz_v1:i_pdd.obj
 0001:00006448       ??_C@_1FA@KBGDHCDA@?$AAS?$AAe?$AAn?$AAd?$AA?5?$AAe?$AAr?$AAr?$AAo?$AAr?$AA?$DP?$AA?$DP?$AA?5?$AAl?$AAe?$AAn?$AA?$DN?$AA?$CF?$AAx?$AA?0?$AA?5?$AAs?$AAt?$AAa?$AAt?$AAu?$AAs?$AA?$DN?$AA?$CF?$AAx?$AA?0?$AA?5@ 10007448     usb_usbfn_mx25_topaz_v1:i_pdd.obj
 0001:00006498       ??_C@_1EC@ONAPCMHH@?$AAS?$AAt?$AAa?$AAt?$AAu?$AAs?$AA?5?$AAi?$AAs?$AA?5?$AAn?$AAo?$AAt?$AA?5?$AA0?$AA?5?$AAo?$AAn?$AA?5?$AAs?$AAe?$AAn?$AAt?$AA?5?$AA?$CF?$AAx?$AA?5?$AA?$DN?$AA?$CF?$AAx?$AA?$AN?$AA?6@ 10007498     usb_usbfn_mx25_topaz_v1:i_pdd.obj
 0001:000064e0       ??_C@_1GI@DMJOJCJK@?$AAC?$AAh?$AAe?$AAc?$AAk?$AAE?$AAn?$AAd?$AAp?$AAo?$AAi?$AAn?$AAt?$AA?3?$AAS?$AAe?$AAt?$AA?5?$AAA?$AAd?$AAd?$AAr?$AAe?$AAs?$AAs?$AA?3?$AA?5?$AA?$CF?$AAx?$AA?$CI?$AA?$CF?$AAx@ 100074e0     usb_usbfn_mx25_topaz_v1:i_pdd.obj
 0001:00006548       ??_C@_1FO@LDFIJMJF@?$AAC?$AAh?$AAe?$AAc?$AAk?$AAE?$AAn?$AAd?$AAp?$AAo?$AAi?$AAn?$AAt?$AA?3?$AAE?$AAP?$AA0?$AA?5?$AAO?$AAU?$AAT?$AA?5?$AAN?$AAU?$AAL?$AAL?$AA?5?$AAt?$AAr?$AAa?$AAn?$AAs@ 10007548     usb_usbfn_mx25_topaz_v1:i_pdd.obj
 0001:000065a8       ??_C@_1FG@MIJKNENI@?$AAC?$AAh?$AAe?$AAc?$AAk?$AAE?$AAn?$AAd?$AAp?$AAo?$AAi?$AAn?$AAt?$AA?3?$AAE?$AAP?$AA0?$AA?5?$AAO?$AAU?$AAT?$AA?5?$AA?$CF?$AAd?$AA?5?$AAb?$AAy?$AAt?$AAe?$AAs?$AA?5?$AAc@ 100075a8     usb_usbfn_mx25_topaz_v1:i_pdd.obj
 0001:00006600       ??_C@_1FK@DOJLLFPC@?$AAC?$AAh?$AAe?$AAc?$AAk?$AAE?$AAn?$AAd?$AAp?$AAo?$AAi?$AAn?$AAt?$AA?3?$AAE?$AAP?$AA0?$AA?5?$AAO?$AAU?$AAT?$AA?5?$AA?$CF?$AAd?$AA?5?$AAb?$AAy?$AAt?$AAe?$AAs?$AA?5?$AAn@ 10007600     usb_usbfn_mx25_topaz_v1:i_pdd.obj
 0001:00006660       ??_C@_1GA@IAMKOKAN@?$AA?$CD?$AA?$CD?$AA?$CD?$AA?$CD?$AA?$CD?$AA?5?$AAm?$AAo?$AAr?$AAe?$AA?5?$AAd?$AAa?$AAt?$AAa?$AA?5?$AAt?$AAo?$AA?5?$AAr?$AAe?$AAc?$AAe?$AAi?$AAv?$AAe?$AA?5?$AAo?$AAn?$AA?5?$AAE?$AAP@ 10007660     usb_usbfn_mx25_topaz_v1:i_pdd.obj
 0001:000066c0       ??_C@_1IM@GIGJCFIB@?$AA?$CD?$AA?$CD?$AA?$CD?$AA?$CD?$AA?$CD?$AA?$CD?$AA?$CD?$AA?$CD?$AA?$CD?$AA?$CD?$AA?$CD?$AA?$CD?$AA?$CD?$AA?5?$AAE?$AAN?$AAD?$AAP?$AAT?$AAC?$AAO?$AAM?$AAP?$AAL?$AAE?$AAT?$AAE?$AA?5?$AA?$CF?$AAx?$AA?5?$AAN@ 100076c0     usb_usbfn_mx25_topaz_v1:i_pdd.obj
 0001:00006750       ??_C@_1EG@NDHBBAAH@?$AAO?$AAU?$AAT?$AA?5?$AA?$CF?$AAs?$AA?5?$AAC?$AAo?$AAm?$AAp?$AAl?$AAe?$AAt?$AAe?$AAd?$AA?5?$AAf?$AAo?$AAr?$AA?5?$AAe?$AAn?$AAd?$AAp?$AAo?$AAi?$AAn?$AAt?$AA?5?$AA?$CF?$AAd@ 10007750     usb_usbfn_mx25_topaz_v1:i_pdd.obj
 0001:00006798       ??_C@_1O@BIOIDBLM@?$AAC?$AAa?$AAn?$AAc?$AAe?$AAl?$AA?$AA@ 10007798     usb_usbfn_mx25_topaz_v1:i_pdd.obj
 0001:000067a8       ??_C@_1O@PFKKKDLL@?$AAN?$AAo?$AAr?$AAm?$AAa?$AAl?$AA?$AA@ 100077a8     usb_usbfn_mx25_topaz_v1:i_pdd.obj
 0001:000067b8       ??_C@_1EK@JNBLLHDF@?$AAC?$AAh?$AAe?$AAc?$AAk?$AAE?$AAn?$AAd?$AAp?$AAo?$AAi?$AAn?$AAt?$AA?$CI?$AAe?$AAp?$AA?$DN?$AA?$CF?$AAd?$AA?$CJ?$AA?3?$AA?5?$AAB?$AAU?$AAF?$AAF?$AAE?$AAR?$AA_?$AAE?$AAR?$AAR@ 100077b8     usb_usbfn_mx25_topaz_v1:i_pdd.obj
 0001:00006804       ??_C@_1CG@FAGAAPBN@?$AAE?$AAN?$AAD?$AAP?$AAT?$AAC?$AAO?$AAM?$AAP?$AAL?$AAE?$AAT?$AAE?$AA?5?$AA?$CF?$AAx?$AA?$AN?$AA?6?$AA?$AA@ 10007804     usb_usbfn_mx25_topaz_v1:i_pdd.obj
 0001:0000682c       ??_C@_1DO@LDKDDFPP@?$AAS?$AAt?$AAa?$AAt?$AAu?$AAs?$AA?5?$AAi?$AAs?$AA?5?$AAn?$AAo?$AAt?$AA?5?$AA0?$AA?5?$AAo?$AAn?$AA?5?$AAr?$AAe?$AAc?$AAv?$AA?5?$AA?$CF?$AAx?$AA?5?$AA?$DN?$AA?$CF?$AAx?$AA?$AA@ 1000782c     usb_usbfn_mx25_topaz_v1:i_pdd.obj
 0001:00006870       ??_C@_1EO@FDNJCHA@?$AAD?$AAe?$AAv?$AAi?$AAc?$AAe?$AA?5?$AAD?$AAe?$AAt?$AAa?$AAc?$AAh?$AA?0?$AA?5?$AAw?$AAi?$AAt?$AAh?$AA?5?$AAs?$AAu?$AAs?$AAp?$AA?$CI?$AA?$CF?$AAd?$AA?$CJ?$AA?0?$AA?5?$AAi?$AAd@ 10007870     usb_usbfn_mx25_topaz_v1:i_pdd.obj
 0001:000068c0       ??_C@_1BO@PIPKGBKA@?$AA?$CK?$AAt?$AAe?$AAm?$AAp?$AA3?$AA?5?$AA0?$AAx?$AA?$CF?$AAx?$AA?5?$AA?$AN?$AA?6?$AA?$AA@ 100078c0     usb_usbfn_mx25_topaz_v1:i_pdd.obj
 0001:000068e0       ??_C@_1CI@HKDMKLGF@?$AAD?$AAe?$AAt?$AAa?$AAc?$AAh?$AA?3?$AA?5?$AAP?$AAO?$AAR?$AAT?$AAS?$AAC?$AA?5?$AA0?$AAx?$AA?$CF?$AAx?$AA?$AA@ 100078e0     usb_usbfn_mx25_topaz_v1:i_pdd.obj
 0001:00006908       ??_C@_1CK@LPGMAHKL@?$AA?9?$AAU?$AAF?$AAN?$AA_?$AAD?$AAE?$AAT?$AAA?$AAC?$AAH?$AA?5?$AAc?$AAa?$AAl?$AAl?$AAe?$AAd?$AA?$AN?$AA?6?$AA?$AA@ 10007908     usb_usbfn_mx25_topaz_v1:i_pdd.obj
 0001:00006934       ??_C@_1CK@MPBLBBEN@?$AA?$CL?$AAU?$AAF?$AAN?$AA_?$AAD?$AAE?$AAT?$AAA?$AAC?$AAH?$AA?5?$AAc?$AAa?$AAl?$AAl?$AAe?$AAd?$AA?$AN?$AA?6?$AA?$AA@ 10007934     usb_usbfn_mx25_topaz_v1:i_pdd.obj
 0001:00006960       ??_C@_1O@BJIMCIMK@?$AAR?$AAe?$AAs?$AAu?$AAm?$AAe?$AA?$AA@ 10007960     usb_usbfn_mx25_topaz_v1:i_pdd.obj
 0001:00006970       ??_C@_1BC@MHKABCGD@?$AAB?$AAr?$AAe?$AAa?$AAk?$AA?5?$AA?$AN?$AA?6?$AA?$AA@ 10007970     usb_usbfn_mx25_topaz_v1:i_pdd.obj
 0001:00006984       ??_C@_1BE@JNFMNJIM@?$AAI?$AAn?$AAt?$AAr?$AA?3?$AAD?$AAo?$AAn?$AAe?$AA?$AA@ 10007984     usb_usbfn_mx25_topaz_v1:i_pdd.obj
 0001:00006998       ??_C@_1CC@IFAPINEE@?$AAS?$AAe?$AAt?$AAu?$AAp?$AAE?$AAv?$AAe?$AAn?$AAt?$AA?5?$AA?4?$AA?4?$AA?4?$AA?$AN?$AA?6?$AA?$AA@ 10007998     usb_usbfn_mx25_topaz_v1:i_pdd.obj
 0001:000069c0       ??_C@_1EE@JAFGGGNF@?$AAI?$AAn?$AAt?$AAr?$AA?3?$AAU?$AAI?$AA?5?$AAS?$AAE?$AAT?$AAU?$AAP?$AAS?$AAT?$AAA?$AAT?$AA?5?$AA?$CF?$AAx?$AA?5?$AAE?$AAN?$AAD?$AAP?$AAT?$AAC?$AAO?$AAM?$AAP?$AA?5?$AA?$CF@ 100079c0     usb_usbfn_mx25_topaz_v1:i_pdd.obj
 0001:00006a04       ??_C@_1BC@MCOFDLFC@?$AAI?$AAn?$AAt?$AAr?$AA?3?$AAS?$AAL?$AAI?$AA?$AA@ 10007a04     usb_usbfn_mx25_topaz_v1:i_pdd.obj
 0001:00006a18       ??_C@_1BO@EGKDOEEI@?$AAI?$AAn?$AAt?$AAr?$AA?3?$AAS?$AAi?$AAg?$AAn?$AAa?$AAl?$AAl?$AAe?$AAd?$AA?$AA@ 10007a18     usb_usbfn_mx25_topaz_v1:i_pdd.obj
 0001:00006a38       ??_C@_1CA@FFAPNJLP@?$AAP?$AAD?$AAD?$AA?5?$AA?9?$AA?5?$AAS?$AAU?$AAS?$AAP?$AAE?$AAN?$AAD?$AA?$AN?$AA?6?$AA?$AA@ 10007a38     usb_usbfn_mx25_topaz_v1:i_pdd.obj
 0001:00006a58       ??_C@_1CC@NCLEKMLF@?$AA?5?$AAs?$AAt?$AAa?$AAt?$AAe?$AA?4?$AAP?$AAS?$AAP?$AAD?$AA?5?$AA?$CF?$AAx?$AA?$AN?$AA?6?$AA?$AA@ 10007a58     usb_usbfn_mx25_topaz_v1:i_pdd.obj
 0001:00006a7c       ??_C@_1CM@GCFNPFKO@?$AA?5?$AAB?$AAS?$AA_?$AAF?$AAU?$AAL?$AAL?$AA_?$AAS?$AAP?$AAE?$AAE?$AAD?$AA?5?$AA?5?$AA?5?$AA?$CF?$AAx?$AA?$AN?$AA?6?$AA?$AA@ 10007a7c     usb_usbfn_mx25_topaz_v1:i_pdd.obj
 0001:00006aa8       ??_C@_1CM@EIGJNBDN@?$AA?5?$AAB?$AAS?$AA_?$AAH?$AAI?$AAG?$AAH?$AA_?$AAS?$AAP?$AAE?$AAE?$AAD?$AA?5?$AA?5?$AA?5?$AA?$CF?$AAx?$AA?$AN?$AA?6?$AA?$AA@ 10007aa8     usb_usbfn_mx25_topaz_v1:i_pdd.obj
 0001:00006ad8       ??_C@_1JI@KKCMHPHI@?$AAH?$AAa?$AAn?$AAd?$AAl?$AAe?$AAU?$AAS?$AAB?$AAR?$AAe?$AAs?$AAe?$AAt?$AA?3?$AA?5?$AAN?$AAo?$AAt?$AA?5?$AAs?$AAt?$AAi?$AAl?$AAl?$AA?5?$AAi?$AAn?$AA?5?$AAr?$AAe?$AAs@ 10007ad8     usb_usbfn_mx25_topaz_v1:i_pdd.obj
 0001:00006b70       ??_C@_1CA@KBLMCKFP@?$AAD?$AAe?$AAv?$AAi?$AAc?$AAe?$AA?5?$AAD?$AAe?$AAt?$AAa?$AAc?$AAh?$AA?$AN?$AA?6?$AA?$AA@ 10007b70     usb_usbfn_mx25_topaz_v1:i_pdd.obj
 0001:00006b90       ??_C@_1FO@DFNLJIPA@?$AAU?$AAS?$AAB?$AAC?$AAo?$AAn?$AAt?$AAr?$AAo?$AAl?$AAl?$AAe?$AAr?$AAR?$AAu?$AAn?$AA?$CI?$AA?$CF?$AAd?$AA?$CJ?$AA?3?$AA?5?$AAf?$AAa?$AAi?$AAl?$AAe?$AAd?$AA?5?$AAt?$AAo?$AA?5@ 10007b90     usb_usbfn_mx25_topaz_v1:i_pdd.obj
 0001:00006bf0       ??_C@_1HI@FMJPDAIJ@?$AAU?$AAS?$AAB?$AAC?$AAo?$AAn?$AAt?$AAr?$AAo?$AAl?$AAl?$AAe?$AAr?$AAR?$AAu?$AAn?$AA?$CI?$AA1?$AA?$CJ?$AA?3?$AA?5?$AAE?$AAR?$AAR?$AAO?$AAR?$AA?5?$AA?$CD?$AA?$CD?$AA?$CD?$AA?$CD?$AA?$CD@ 10007bf0     usb_usbfn_mx25_topaz_v1:i_pdd.obj
 0001:00006c68       ??_C@_1EM@BBPKMFPI@?$AAS?$AAt?$AAo?$AAp?$AA?5?$AAU?$AAS?$AAB?$AA?5?$AAc?$AAo?$AAn?$AAt?$AAr?$AAo?$AAl?$AAl?$AAe?$AAr?$AA?5?$AA?$CI?$AAR?$AAS?$AA?$DN?$AA?$CF?$AAd?$AA?5?$AA?9?$AA?$DO?$AA?5?$AAR?$AAS@ 10007c68     usb_usbfn_mx25_topaz_v1:i_pdd.obj
 0001:00006cb8       ??_C@_1EO@GGMICPAJ@?$AAS?$AAt?$AAa?$AAr?$AAt?$AA?5?$AAU?$AAS?$AAB?$AA?5?$AAc?$AAo?$AAn?$AAt?$AAr?$AAo?$AAl?$AAl?$AAe?$AAr?$AA?5?$AA?$CI?$AAR?$AAS?$AA?$DN?$AA?$CF?$AAd?$AA?5?$AA?9?$AA?$DO?$AA?5?$AAR@ 10007cb8     usb_usbfn_mx25_topaz_v1:i_pdd.obj
 0001:00006d08       ??_C@_1IO@CBIPFBFK@?$AA?$CD?$AA?$CD?$AA?$CD?$AA?$CD?$AA?$CD?$AA?$CD?$AA?$CD?$AA?$CD?$AA?$CD?$AA?$CD?$AA?$CD?$AA?$CD?$AA?$CD?$AA?5?$AAP?$AAr?$AAi?$AAm?$AAe?$AA?5?$AAF?$AAa?$AAi?$AAl?$AAe?$AAd?$AA?5?$AAf?$AAo?$AAr?$AA?5?$AAe@ 10007d08     usb_usbfn_mx25_topaz_v1:i_pdd.obj
 0001:00006d98       ??_C@_1FO@BKKPAEJB@?$AAI?$AAs?$AAs?$AAu?$AAe?$AAT?$AAr?$AAa?$AAn?$AAs?$AAf?$AAe?$AAr?$AA?5?$AAS?$AAE?$AAT?$AAU?$AAP?$AAS?$AAT?$AAA?$AAT?$AA?5?$AAr?$AAe?$AAc?$AAe?$AAi?$AAv?$AAe?$AAd@ 10007d98     usb_usbfn_mx25_topaz_v1:i_pdd.obj
 0001:00006df8       ??_C@_1EK@PGGCKEHJ@?$AAU?$AAf?$AAn?$AAP?$AAd?$AAd?$AA?3?$AA?5?$AAn?$AAe?$AAw?$AA?5?$AAs?$AAe?$AAt?$AAu?$AAp?$AA?5?$AAr?$AAe?$AAq?$AAu?$AAe?$AAs?$AAt?$AA?5?$AAd?$AAe?$AAt?$AAe?$AAc?$AAt@ 10007df8     usb_usbfn_mx25_topaz_v1:i_pdd.obj
 0001:00006e48       ??_C@_1HI@CDKGKFCF@?$AAE?$AAR?$AAR?$AAO?$AAR?$AA?3?$AA?5?$AAU?$AAf?$AAn?$AAP?$AAd?$AAd?$AA_?$AAI?$AAs?$AAs?$AAu?$AAe?$AAT?$AAr?$AAa?$AAn?$AAs?$AAf?$AAe?$AAr?$AA?3?$AA?5?$AAC?$AAe?$AAC@ 10007e48     usb_usbfn_mx25_topaz_v1:i_pdd.obj
 0001:00006ec0       ??_C@_1FK@CELBMJI@?$AAU?$AAf?$AAn?$AAP?$AAd?$AAd?$AA?3?$AA?5?$AAP?$AAa?$AAg?$AAe?$AA?5?$AAt?$AAr?$AAa?$AAn?$AAs?$AAl?$AAa?$AAt?$AAi?$AAo?$AAn?$AA?5?$AAf?$AAa?$AAi?$AAl?$AAe?$AAd?$AA?4@ 10007ec0     usb_usbfn_mx25_topaz_v1:i_pdd.obj
 0001:00006f20       ??_C@_1HA@DFAMLEOB@?$AAU?$AAf?$AAn?$AAP?$AAd?$AAd?$AA_?$AAI?$AAs?$AAs?$AAu?$AAe?$AAT?$AAr?$AAa?$AAn?$AAs?$AAf?$AAe?$AAr?$AA?3?$AA?5?$AAB?$AAu?$AAf?$AAf?$AAe?$AAr?$AA?5?$AAP?$AAa?$AAg@ 10007f20     usb_usbfn_mx25_topaz_v1:i_pdd.obj
 0001:00006f90       ??_C@_1KA@JGAAJONG@?$AAU?$AAf?$AAn?$AAP?$AAd?$AAd?$AA_?$AAI?$AAs?$AAs?$AAu?$AAe?$AAT?$AAr?$AAa?$AAn?$AAs?$AAf?$AAe?$AAr?$AA?3?$AA?5?$AAF?$AAa?$AAi?$AAl?$AAe?$AAd?$AA?5?$AAt?$AAo?$AA?5@ 10007f90     usb_usbfn_mx25_topaz_v1:i_pdd.obj
 0001:00007030       ??_C@_1HG@OBGGAFFH@?$AAE?$AAR?$AAR?$AAO?$AAR?$AA?3?$AA?5?$AAU?$AAf?$AAn?$AAP?$AAd?$AAd?$AA_?$AAI?$AAs?$AAs?$AAu?$AAe?$AAT?$AAr?$AAa?$AAn?$AAs?$AAf?$AAe?$AAr?$AA?3?$AA?5?$AAC?$AAe?$AAO@ 10008030     usb_usbfn_mx25_topaz_v1:i_pdd.obj
 0001:000070a8       ??_C@_1FA@PGOEGLMA@?$AAU?$AAf?$AAn?$AAP?$AAd?$AAd?$AA_?$AAI?$AAs?$AAs?$AAu?$AAe?$AAT?$AAr?$AAa?$AAn?$AAs?$AAf?$AAe?$AAr?$AA?5?$AAf?$AAi?$AAr?$AAs?$AAt?$AA?5?$AAt?$AAi?$AAm?$AAe?$AA?$CI@ 100080a8     usb_usbfn_mx25_topaz_v1:i_pdd.obj
 0001:000070f8       ??_C@_1JO@PEEOMCDL@?$AAI?$AAs?$AAs?$AAT?$AAr?$AAa?$AAn?$AA?5?$AA?$CI?$AA?$CF?$AAd?$AA?$CJ?$AA?3?$AA?5?$AA?$CF?$AAs?$AA?5?$AA?$CI?$AAp?$AAT?$AAr?$AAa?$AAn?$AAs?$AAf?$AAe?$AAr?$AA?$DN?$AA0?$AAx?$AA?$CF?$AAx@ 100080f8     usb_usbfn_mx25_topaz_v1:i_pdd.obj
 0001:00007198       ??_C@_1EA@GOCNCOIC@?$AAI?$AAs?$AAs?$AAu?$AAe?$AAT?$AAr?$AAa?$AAn?$AAs?$AAf?$AAe?$AAr?$AA?3?$AA?5?$AA?$CF?$AAs?$AA?5?$AAw?$AAi?$AAt?$AAh?$AA?5?$AA?$CF?$AAd?$AA?5?$AAb?$AAy?$AAt?$AAe?$AAs?$AA?$AA@ 10008198     usb_usbfn_mx25_topaz_v1:i_pdd.obj
 0001:000071d8       ??_C@_19CIJIHAKK@?$AAN?$AAU?$AAL?$AAL?$AA?$AA@ 100081d8     usb_usbfn_mx25_topaz_v1:i_pdd.obj
 0001:000071e4       ??_C@_17HCEMPBGG@?$AAO?$AAU?$AAT?$AA?$AA@ 100081e4     usb_usbfn_mx25_topaz_v1:i_pdd.obj
 0001:000071ec       ??_C@_15BNKBCKPG@?$AAI?$AAN?$AA?$AA@ 100081ec     usb_usbfn_mx25_topaz_v1:i_pdd.obj
 0001:000071f8       ??_C@_1EG@CKENHIMK@?$AAU?$AAs?$AAb?$AAF?$AAn?$AAP?$AAd?$AAd?$AA_?$AAA?$AAb?$AAo?$AAr?$AAt?$AAT?$AAr?$AAa?$AAn?$AAs?$AAf?$AAe?$AAr?$AA?9?$AA?5?$AA?$CI?$AAE?$AAP?$AA?$DN?$AA?5?$AA?$CF?$AAd?$AA?$CJ@ 100081f8     usb_usbfn_mx25_topaz_v1:i_pdd.obj
 0001:00007240       ??_C@_1FA@PHGGDELL@?$AAA?$AAb?$AAo?$AAr?$AAt?$AA?$CI?$AA?$CF?$AAd?$AA?$CJ?$AA?5?$AAs?$AAk?$AAi?$AAp?$AAp?$AAe?$AAd?$AA?5?$AA?$CI?$AAT?$AAr?$AAa?$AAn?$AA?5?$AA0?$AAx?$AA?$CF?$AAx?$AA?5?$AA?$CB?$AA?$DN?$AA?5@ 10008240     usb_usbfn_mx25_topaz_v1:i_pdd.obj
 0001:00007290       ??_C@_1FK@ENKBNDBL@?$AA?$CD?$AA?$CD?$AA?$CD?$AA?$CD?$AA?$CD?$AA?$CD?$AA?$CD?$AA?$CD?$AA?$CD?$AA?$CD?$AA?$CD?$AA?5?$AAA?$AAb?$AAo?$AAr?$AAt?$AAT?$AAr?$AAa?$AAn?$AAs?$AAf?$AAe?$AAr?$AA?$CI?$AA?$CF?$AAd?$AA?$CJ?$AA?5?$AAD?$AAe@ 10008290     usb_usbfn_mx25_topaz_v1:i_pdd.obj
 0001:000072f0       ??_C@_1GK@BJNDOLBF@?$AAU?$AAs?$AAb?$AAF?$AAn?$AAP?$AAd?$AAd?$AA_?$AAA?$AAb?$AAo?$AAr?$AAt?$AAT?$AAr?$AAa?$AAn?$AAs?$AAf?$AAe?$AAr?$AA?3?$AA?5?$AAp?$AAT?$AAr?$AAa?$AAn?$AAs?$AAf?$AAe@ 100082f0     usb_usbfn_mx25_topaz_v1:i_pdd.obj
 0001:0000735c       ??_C@_1DA@JMEFNML@?$AAA?$AAb?$AAo?$AAr?$AAt?$AAT?$AAr?$AAa?$AAn?$AAs?$AAf?$AAe?$AAr?$AA?5?$AA?$CI?$AA?$CF?$AAs?$AA?5?$AAE?$AAP?$AA?$CF?$AAd?$AA?$CJ?$AA?$AA@ 1000835c     usb_usbfn_mx25_topaz_v1:i_pdd.obj
 0001:00007390       ??_C@_1EG@BFJDKFHL@?$AAU?$AAs?$AAb?$AAF?$AAn?$AAP?$AAd?$AAd?$AA_?$AAA?$AAb?$AAo?$AAr?$AAt?$AAT?$AAr?$AAa?$AAn?$AAs?$AAf?$AAe?$AAr?$AA?$CL?$AA?5?$AA?$CI?$AAE?$AAP?$AA?$DN?$AA?5?$AA?$CF?$AAd?$AA?$CJ@ 10008390     usb_usbfn_mx25_topaz_v1:i_pdd.obj
 0001:000073d8       ??_C@_1DI@FFFNHHBF@?$AAU?$AAs?$AAb?$AAF?$AAn?$AAP?$AAd?$AAd?$AA_?$AAS?$AAt?$AAa?$AAl?$AAl?$AAE?$AAn?$AAd?$AAp?$AAo?$AAi?$AAn?$AAt?$AA?5?$AA?$CF?$AAd?$AA?$AN?$AA?6?$AA?$AA@ 100083d8     usb_usbfn_mx25_topaz_v1:i_pdd.obj
 0001:00007410       ??_C@_1DI@EBJLFADF@?$AAU?$AAs?$AAb?$AAF?$AAn?$AAP?$AAd?$AAd?$AA_?$AAC?$AAl?$AAe?$AAa?$AAr?$AAE?$AAn?$AAd?$AAp?$AAo?$AAi?$AAn?$AAt?$AA?5?$AA?$CF?$AAd?$AA?$AN?$AA?6?$AA?$AA@ 10008410     usb_usbfn_mx25_topaz_v1:i_pdd.obj
 0001:00007448       ??_C@_1EA@DIDLDIBI@?$AA?9?$AAU?$AAs?$AAb?$AAF?$AAn?$AAP?$AAd?$AAd?$AA_?$AAI?$AAs?$AAE?$AAn?$AAd?$AAp?$AAo?$AAi?$AAn?$AAt?$AAH?$AAa?$AAl?$AAt?$AAe?$AAd?$AA?5?$AA?$CF?$AAd?$AA?$AN?$AA?6?$AA?$AA@ 10008448     usb_usbfn_mx25_topaz_v1:i_pdd.obj
 0001:00007488       ??_C@_1DO@MLIBPKBI@?$AAU?$AAs?$AAb?$AAF?$AAn?$AAP?$AAd?$AAd?$AA_?$AAI?$AAs?$AAE?$AAn?$AAd?$AAp?$AAo?$AAi?$AAn?$AAt?$AAH?$AAa?$AAl?$AAt?$AAe?$AAd?$AA?5?$AA?$CF?$AAd?$AA?$AN?$AA?6?$AA?$AA@ 10008488     usb_usbfn_mx25_topaz_v1:i_pdd.obj
 0001:000074c8       ??_C@_1CA@HMLLGPGC@?$AA?9?$AAS?$AAe?$AAn?$AAd?$AAC?$AAS?$AAH?$AA?5?$AA?$CI?$AAE?$AAP?$AA?$CF?$AAd?$AA?$CJ?$AA?$AA@ 100084c8     usb_usbfn_mx25_topaz_v1:i_pdd.obj
 0001:000074e8       ??_C@_1CE@MAHEKDJP@?$AAS?$AAe?$AAn?$AAd?$AAC?$AAS?$AAH?$AA?5?$AAI?$AAN?$AA?5?$AA?$CI?$AA?$CF?$AAd?$AA?$CJ?$AA?$AN?$AA?6?$AA?$AA@ 100084e8     usb_usbfn_mx25_topaz_v1:i_pdd.obj
 0001:0000750c       ??_C@_1CG@NAGMKJIL@?$AAS?$AAe?$AAn?$AAd?$AAC?$AAS?$AAH?$AA?5?$AAO?$AAU?$AAT?$AA?5?$AA?$CI?$AA?$CF?$AAd?$AA?$CJ?$AA?$AN?$AA?6?$AA?$AA@ 1000850c     usb_usbfn_mx25_topaz_v1:i_pdd.obj
 0001:00007534       ??_C@_1CA@DFPEHIFN@?$AA?$CL?$AAS?$AAe?$AAn?$AAd?$AAC?$AAS?$AAH?$AA?5?$AA?$CI?$AAE?$AAP?$AA?$CF?$AAd?$AA?$CJ?$AA?$AA@ 10008534     usb_usbfn_mx25_topaz_v1:i_pdd.obj
 0001:00007558       ??_C@_1FM@FGGEPKIB@?$AA?$CD?$AA?$CD?$AA?$CD?$AA?$CD?$AA?$CD?$AA?$CD?$AA?$CD?$AA?$CD?$AA?$CD?$AA?$CD?$AA?$CD?$AA?$CD?$AA?$CD?$AA?$CD?$AA?$CD?$AA?$CD?$AA?5?$AAF?$AAa?$AAi?$AAl?$AAe?$AAd?$AA?5?$AAt?$AAo?$AA?5?$AAp?$AAr?$AAi?$AAm?$AAe@ 10008558     usb_usbfn_mx25_topaz_v1:i_pdd.obj
 0001:000075b8       ??_C@_1EG@KGILPPEC@?$AAC?$AAa?$AAn?$AA?5?$AAn?$AAo?$AAt?$AA?5?$AAp?$AAr?$AAi?$AAm?$AAe?$AA?5?$AAf?$AAo?$AAr?$AA?5?$AAZ?$AAL?$AAT?$AA?5?$AA?$CI?$AA?$CF?$AAs?$AA?$CJ?$AA?3?$AA?5?$AAb?$AAu?$AAs?$AAy@ 100085b8     usb_usbfn_mx25_topaz_v1:i_pdd.obj
 0001:00007600       ??_C@_1BM@LGGJJGMB@?$AAP?$AAr?$AAi?$AAm?$AAe?$AAF?$AAZ?$AAL?$AAT?$AA?3?$AA?5?$AA?$CF?$AAs?$AA?$AA@ 10008600     usb_usbfn_mx25_topaz_v1:i_pdd.obj
 0001:00007620       ??_C@_1EA@KNMJPPBI@?$AAU?$AAs?$AAb?$AAF?$AAn?$AAP?$AAd?$AAd?$AA_?$AAI?$AAn?$AAi?$AAt?$AAi?$AAa?$AAt?$AAe?$AAR?$AAe?$AAm?$AAo?$AAt?$AAe?$AAW?$AAa?$AAk?$AAe?$AAu?$AAp?$AA?$AN?$AA?6?$AA?$AA@ 10008620     usb_usbfn_mx25_topaz_v1:i_pdd.obj
 0001:00007660       ??_C@_1CO@LFIHBCKN@?$AAS?$AAe?$AAt?$AAP?$AAo?$AAw?$AAe?$AAr?$AAS?$AAt?$AAa?$AAt?$AAe?$AA?5?$AA?$DN?$AA?5?$AA0?$AAx?$AA?$CF?$AAx?$AA?$AN?$AA?6?$AA?$AA@ 10008660     usb_usbfn_mx25_topaz_v1:i_pdd.obj
 0001:00007690       ??_C@_1HC@FEAKGGLP@?$AAP?$AAD?$AAD?$AA?3?$AA?5?$AAS?$AAe?$AAt?$AA?5?$AAF?$AAe?$AAa?$AAt?$AAu?$AAr?$AAe?$AA?5?$AA?$CI?$AAT?$AAE?$AAS?$AAT?$AA?5?$AAM?$AAO?$AAD?$AAE?$AA?$CJ?$AA?5?$AAO?$AAT?$AAG@ 10008690     usb_usbfn_mx25_topaz_v1:i_pdd.obj
 0001:00007708       ??_C@_1HC@GBFNHNAG@?$AAI?$AAO?$AAC?$AAT?$AAL?$AA_?$AAB?$AAU?$AAS?$AA_?$AAS?$AAE?$AAT?$AA_?$AAP?$AAO?$AAW?$AAE?$AAR?$AA_?$AAS?$AAT?$AAA?$AAT?$AAE?$AA?3?$AA?5?$AAC?$AAe?$AAO?$AAp?$AAe@ 10008708     usb_usbfn_mx25_topaz_v1:i_pdd.obj
 0001:00007780       ??_C@_1HE@NONILAAF@?$AAI?$AAO?$AAC?$AAT?$AAL?$AA_?$AAB?$AAU?$AAS?$AA_?$AAS?$AAE?$AAT?$AA_?$AAP?$AAO?$AAW?$AAE?$AAR?$AA_?$AAS?$AAT?$AAA?$AAT?$AAE?$AA?3?$AA?5?$AAC?$AAe?$AAC?$AAl?$AAo@ 10008780     usb_usbfn_mx25_topaz_v1:i_pdd.obj
 0001:000077f8       ??_C@_1EG@GJIKGHF@?$AAI?$AAO?$AAC?$AAT?$AAL?$AA_?$AAB?$AAU?$AAS?$AA_?$AAS?$AAE?$AAT?$AA_?$AAP?$AAO?$AAW?$AAE?$AAR?$AA_?$AAS?$AAT?$AAA?$AAT?$AAE?$AA?5?$AAc?$AAa?$AAl?$AAl?$AAe?$AAd@ 100087f8     usb_usbfn_mx25_topaz_v1:i_pdd.obj
 0001:00007840       ??_C@_1HC@NPNGJCMK@?$AAI?$AAO?$AAC?$AAT?$AAL?$AA_?$AAB?$AAU?$AAS?$AA_?$AAG?$AAE?$AAT?$AA_?$AAP?$AAO?$AAW?$AAE?$AAR?$AA_?$AAS?$AAT?$AAA?$AAT?$AAE?$AA?3?$AA?5?$AAC?$AAe?$AAO?$AAp?$AAe@ 10008840     usb_usbfn_mx25_topaz_v1:i_pdd.obj
 0001:000078b8       ??_C@_1HE@IJCCGJCF@?$AAI?$AAO?$AAC?$AAT?$AAL?$AA_?$AAB?$AAU?$AAS?$AA_?$AAG?$AAE?$AAT?$AA_?$AAP?$AAO?$AAW?$AAE?$AAR?$AA_?$AAS?$AAT?$AAA?$AAT?$AAE?$AA?3?$AA?5?$AAC?$AAe?$AAC?$AAl?$AAo@ 100088b8     usb_usbfn_mx25_topaz_v1:i_pdd.obj
 0001:00007930       ??_C@_1EG@FFODHJCP@?$AAI?$AAO?$AAC?$AAT?$AAL?$AA_?$AAB?$AAU?$AAS?$AA_?$AAG?$AAE?$AAT?$AA_?$AAP?$AAO?$AAW?$AAE?$AAR?$AA_?$AAS?$AAT?$AAA?$AAT?$AAE?$AA?5?$AAc?$AAa?$AAl?$AAl?$AAe?$AAd@ 10008930     usb_usbfn_mx25_topaz_v1:i_pdd.obj
 0001:00007978       ??_C@_1BM@ELBPNMDN@?$AAU?$AAf?$AAn?$AAP?$AAd?$AAd?$AA_?$AAS?$AAt?$AAo?$AAp?$AA?$AN?$AA?6?$AA?$AA@ 10008978     usb_usbfn_mx25_topaz_v1:i_pdd.obj
 0001:00007994       ??_C@_1DK@CCAICBIP@?$AA?$CL?$AAU?$AAf?$AAn?$AAP?$AAd?$AAd?$AA_?$AAD?$AAe?$AAi?$AAn?$AAi?$AAt?$AAE?$AAn?$AAd?$AAp?$AAo?$AAi?$AAn?$AAt?$AA?3?$AA?5?$AA?$CF?$AAd?$AA?$AN?$AA?6?$AA?$AA@ 10008994     usb_usbfn_mx25_topaz_v1:i_pdd.obj
 0001:000079d0       ??_C@_1DK@MHIAFBPJ@?$AAI?$AAn?$AAi?$AAt?$AA?5?$AAE?$AAn?$AAd?$AAp?$AAo?$AAi?$AAn?$AAt?$AA?3?$AA?5?$AA?$CF?$AAx?$AA?0?$AA?5?$AAc?$AAt?$AAr?$AAl?$AA?$DN?$AA?$CF?$AAx?$AA?$AN?$AA?6?$AA?$AA@ 100089d0     usb_usbfn_mx25_topaz_v1:i_pdd.obj
 0001:00007a10       ??_C@_1EK@HMBFBNAN@?$AAU?$AAf?$AAn?$AAP?$AAd?$AAd?$AA_?$AAI?$AAn?$AAi?$AAt?$AAE?$AAn?$AAd?$AAp?$AAo?$AAi?$AAn?$AAt?$AA?3?$AA?5?$AA?$CF?$AAd?$AA?5?$AAA?$AAt?$AAt?$AAr?$AAi?$AAb?$AA?$CI?$AA?$CF@ 10008a10     usb_usbfn_mx25_topaz_v1:i_pdd.obj
 0001:00007a5c       ??_C@_1CA@IJBGFJAE@?$AA?9?$AAU?$AAf?$AAn?$AAP?$AAd?$AAd?$AA_?$AAS?$AAt?$AAa?$AAr?$AAt?$AA?$AN?$AA?6?$AA?$AA@ 10008a5c     usb_usbfn_mx25_topaz_v1:i_pdd.obj
 0001:00007a7c       ??_C@_1CA@MAFJEODL@?$AA?$CL?$AAU?$AAf?$AAn?$AAP?$AAd?$AAd?$AA_?$AAS?$AAt?$AAa?$AAr?$AAt?$AA?$AN?$AA?6?$AA?$AA@ 10008a7c     usb_usbfn_mx25_topaz_v1:i_pdd.obj
 0001:00007a9c       ??_C@_1DG@EEIHMJOF@?$AAS?$AAt?$AAa?$AAt?$AAu?$AAs?$AA?5?$AAf?$AAo?$AAr?$AA?5?$AAt?$AAd?$AA0?$AA?$DN?$AA?$CF?$AAx?$AA?0?$AA?5?$AAt?$AAb?$AA?$DN?$AA?$CF?$AAx?$AA?$AN?$AA?6?$AA?$AA@ 10008a9c     usb_usbfn_mx25_topaz_v1:i_pdd.obj
 0001:00007ad4       ??_C@_1CM@FGGAHLIL@?$AAP?$AAR?$AAI?$AAM?$AAE?$AA?5?$AAf?$AAa?$AAi?$AAl?$AAe?$AAd?$AA?5?$AAo?$AAn?$AA?5?$AAE?$AAP?$AA0?$AA?$AN?$AA?6?$AA?$AA@ 10008ad4     usb_usbfn_mx25_topaz_v1:i_pdd.obj
 0001:00007b00       ??_C@_1FC@FLIFOJB@?$AAN?$AAe?$AAw?$AA?5?$AAs?$AAe?$AAt?$AAu?$AAp?$AA?5?$AAr?$AAe?$AAc?$AAe?$AAi?$AAv?$AAe?$AAd?$AA?5?$AAw?$AAh?$AAe?$AAn?$AA?5?$AAp?$AAr?$AAi?$AAm?$AAi?$AAn?$AAg?$AA?$DN@ 10008b00     usb_usbfn_mx25_topaz_v1:i_pdd.obj
 0001:00007b58       ??_C@_1GC@FCEGAELL@?$AAS?$AAe?$AAt?$AAu?$AAp?$AA?5?$AAn?$AAo?$AAt?$AA?5?$AAp?$AAr?$AAo?$AAc?$AAe?$AAs?$AAs?$AAe?$AAd?$AA?5?$AA?$CI?$AAS?$AAE?$AAT?$AAU?$AAP?$AAS?$AAT?$AAA?$AAT?$AA?$DN?$AA0@ 10008b58     usb_usbfn_mx25_topaz_v1:i_pdd.obj
 0001:00007bbc       ??_C@_1BI@DKIPBNLN@?$AAI?$AAn?$AAi?$AAt?$AAq?$AAh?$AA0?$AA?0?$AA?5?$AA?$CF?$AAx?$AA?$AA@ 10008bbc     usb_usbfn_mx25_topaz_v1:i_pdd.obj
 0001:00007bd4       ??_C@_1BK@PALAPBNH@?$AA?4?$AA?4?$AAc?$AAo?$AAu?$AAn?$AAt?$AA?5?$AA?$CF?$AAd?$AA?$AN?$AA?6?$AA?$AA@ 10008bd4     usb_usbfn_mx25_topaz_v1:i_pdd.obj
 0001:00007bf0       ??_C@_1HA@BIGHAGHK@?$AAD?$AAi?$AAs?$AAa?$AAb?$AAl?$AAe?$AA?5?$AAI?$AAn?$AAt?$AAe?$AAr?$AAr?$AAu?$AAp?$AAt?$AA?5?$AAa?$AAn?$AAd?$AA?5?$AAl?$AAe?$AAt?$AA?5?$AAt?$AAh?$AAe?$AA?5?$AAT?$AAr@ 10008bf0     usb_usbfn_mx25_topaz_v1:i_pdd.obj
 0001:00007c60       ??_C@_1DC@LGPAELOO@?$AAS?$AAi?$AAz?$AAe?$AAo?$AAf?$AA?5?$AAq?$AAh?$AAb?$AAu?$AAf?$AAf?$AAe?$AAr?$AA?5?$AA?$DN?$AA?5?$AA0?$AAx?$AA?$CF?$AAx?$AA?$AN?$AA?6?$AA?$AA@ 10008c60     usb_usbfn_mx25_topaz_v1:i_pdd.obj
 0001:00007c98       ??_C@_1HE@JFIJHLAK@?$AAE?$AAR?$AAR?$AAO?$AAR?$AA?3?$AA?5?$AAU?$AAf?$AAn?$AAP?$AAd?$AAd?$AA_?$AAI?$AAn?$AAi?$AAt?$AA?3?$AA?5?$AAC?$AAo?$AAn?$AAt?$AAr?$AAo?$AAl?$AAl?$AAe?$AAr?$AA?5?$AAr@ 10008c98     usb_usbfn_mx25_topaz_v1:i_pdd.obj
 0001:00007d10       ??_C@_1FK@EMBOCJKF@?$AAE?$AAR?$AAR?$AAO?$AAR?$AA?3?$AA?5?$AAU?$AAf?$AAn?$AAP?$AAd?$AAd?$AA_?$AAI?$AAn?$AAi?$AAt?$AA?3?$AA?5?$AAF?$AAa?$AAi?$AAl?$AAe?$AAd?$AA?5?$AAo?$AAp?$AAe?$AAn?$AA?5@ 10008d10     usb_usbfn_mx25_topaz_v1:i_pdd.obj
 0001:00007d70       ??_C@_1GM@LIECJJPD@?$AAE?$AAR?$AAR?$AAO?$AAR?$AA?3?$AA?5?$AAU?$AAf?$AAn?$AAP?$AAd?$AAd?$AA_?$AAI?$AAn?$AAi?$AAt?$AA?3?$AA?5?$AAF?$AAa?$AAi?$AAl?$AAe?$AAd?$AA?5?$AAr?$AAe?$AAa?$AAd?$AA?5@ 10008d70     usb_usbfn_mx25_topaz_v1:i_pdd.obj
 0001:00007de0       ??_C@_1EG@BDFMMKKK@?$AAU?$AAf?$AAn?$AAP?$AAd?$AAd?$AA_?$AAI?$AAn?$AAi?$AAt?$AA?5?$AAp?$AAP?$AAd?$AAd?$AA?5?$AAa?$AAl?$AAl?$AAo?$AAc?$AAa?$AAt?$AAe?$AA?5?$AAf?$AAa?$AAi?$AAl?$AAe?$AAd@ 10008de0     usb_usbfn_mx25_topaz_v1:i_pdd.obj
 0001:00007e28       ??_C@_1GG@IILKAMAB@?$AAU?$AAS?$AAB?$AA?5?$AAD?$AAr?$AAi?$AAv?$AAe?$AAr?$AA?5?$AAl?$AAo?$AAa?$AAd?$AA?5?$AAf?$AAa?$AAi?$AAl?$AAu?$AAr?$AAe?$AA?5?$AAb?$AAe?$AAc?$AAa?$AAu?$AAs?$AAe?$AA?5@ 10008e28     usb_usbfn_mx25_topaz_v1:i_pdd.obj
 0001:00007f20       ??_C@_0CC@BCDLLINN@Host?5sent?5unhandled?5request?5type@ 10008f20     fsl_serial_pdd_common_topaz_v1:serial_dl.obj
 0001:00007f48       ??_C@_1NC@OGLLDPIP@?$AAC?$AA?3?$AA?2?$AAW?$AAI?$AAN?$AAC?$AAE?$AAR?$AAO?$AAO?$AAT?$AAS?$AA?2?$AAT?$AAo?$AAp?$AAa?$AAz?$AA?2?$AAW?$AAI?$AAN?$AAC?$AAE?$AA6?$AA0?$AA0?$AA?2?$AAP?$AAL?$AAA@ 10008f48     fsl_serial_pdd_common_topaz_v1:serial_dl.obj
 0001:0000801c       ??_C@_0DA@KIPOMLGH@Host?5indicated?5an?5unsupported?5SE@ 1000901c     fsl_serial_pdd_common_topaz_v1:serial_dl.obj
 0001:0000804c       ??_C@_0BP@ONENEGJJ@Unhandled?5Get?5DESCRIPTOR_TYPE?$CB?$AA@ 1000904c     fsl_serial_pdd_common_topaz_v1:serial_dl.obj
 0001:0000806c       ??_C@_0CG@MDLKJKHE@PDD?5Signaled?5bogus?5transfer?5comp@ 1000906c     fsl_serial_pdd_common_topaz_v1:serial_dl.obj
 0001:00008094       ??_C@_0CN@LOCOBGOP@Endpoint?52?5has?5entered?5an?5unsupp@ 10009094     fsl_serial_pdd_common_topaz_v1:serial_dl.obj
 0001:000080c8       ??_C@_1IK@NBNIIDPB@?$AAE?$AAR?$AAR?$AAO?$AAR?$AA?3?$AA?5?$AAP?$AAD?$AAD?$AA?5?$AAI?$AAn?$AAd?$AAi?$AAc?$AAa?$AAt?$AAe?$AAd?$AA?5?$AAt?$AAh?$AAe?$AAr?$AAe?$AA?5?$AAw?$AAa?$AAs?$AA?5?$AAa@ 100090c8     fsl_serial_pdd_common_topaz_v1:serial_dl.obj
 0001:00008158       ??_C@_1HE@HCMHOHD@?$AAE?$AAR?$AAR?$AAO?$AAR?$AA?3?$AA?5?$AAP?$AAD?$AAD?$AA?5?$AAI?$AAn?$AAd?$AAi?$AAc?$AAa?$AAt?$AAe?$AAd?$AA?5?$AAt?$AAh?$AAe?$AAr?$AAe?$AA?5?$AAw?$AAa?$AAs?$AA?5?$AAa@ 10009158     fsl_serial_pdd_common_topaz_v1:serial_dl.obj
 0001:000081d0       ??_C@_1GC@EHFCFLNO@?$AAE?$AAR?$AAR?$AAO?$AAR?$AA?3?$AA?5?$AAS?$AAe?$AAn?$AAt?$AA?5?$AAd?$AAa?$AAt?$AAa?$AA?5?$AAd?$AAo?$AAe?$AAs?$AA?5?$AAn?$AAo?$AAt?$AA?5?$AAm?$AAa?$AAt?$AAc?$AAh?$AA?5@ 100091d0     fsl_serial_pdd_common_topaz_v1:serial_dl.obj
 0001:00008238       ??_C@_1JG@LFGGGOHE@?$AAE?$AAR?$AAR?$AAO?$AAR?$AA?3?$AA?5?$AAP?$AAD?$AAD?$AA?5?$AAI?$AAn?$AAd?$AAi?$AAc?$AAa?$AAt?$AAe?$AAd?$AA?5?$AAR?$AAE?$AAC?$AAV?$AA?5?$AAc?$AAo?$AAm?$AAp?$AAl?$AAe@ 10009238     fsl_serial_pdd_common_topaz_v1:serial_dl.obj
 0001:000082d0       ??_C@_1HE@OMBLMFHA@?$AAE?$AAR?$AAR?$AAO?$AAR?$AA?3?$AA?5?$AAP?$AAD?$AAD?$AA?5?$AAI?$AAn?$AAd?$AAi?$AAc?$AAa?$AAt?$AAe?$AAd?$AA?5?$AAt?$AAh?$AAe?$AAr?$AAe?$AA?5?$AAw?$AAa?$AAs?$AA?5?$AAa@ 100092d0     fsl_serial_pdd_common_topaz_v1:serial_dl.obj
 0001:00008344       ??_C@_1CI@OLENNHLD@?$AAU?$AAf?$AAn?$AAP?$AAd?$AAd?$AA_?$AAI?$AAn?$AAi?$AAt?$AA?5?$AAf?$AAa?$AAi?$AAl?$AAe?$AAd?$AA?$CB?$AA?$AA@ 10009344     fsl_serial_pdd_common_topaz_v1:serial_dl.obj
 0001:00008370       ??_C@_1HG@HALKJNKP@?$AAE?$AAR?$AAR?$AAO?$AAR?$AA?3?$AA?5?$AAU?$AAS?$AAB?$AAS?$AAe?$AAr?$AAi?$AAa?$AAl?$AAI?$AAn?$AAi?$AAt?$AA?5?$AAc?$AAa?$AAl?$AAl?$AAe?$AAd?$AA?5?$AAa?$AAg?$AAa?$AAi@ 10009370     fsl_serial_pdd_common_topaz_v1:serial_dl.obj
 0001:000083e8       ??_C@_1GA@DBGLAADC@?$AAE?$AAR?$AAR?$AAO?$AAR?$AA?3?$AA?5?$AAP?$AAD?$AAD?$AA?5?$AAc?$AAa?$AAn?$AAn?$AAo?$AAt?$AA?5?$AAs?$AAu?$AAp?$AAp?$AAo?$AAr?$AAt?$AA?5?$AAl?$AAo?$AAg?$AAi?$AAc?$AAa@ 100093e8     fsl_serial_pdd_common_topaz_v1:serial_dl.obj
 0001:00008448       ??_C@_1CG@HDEJOBAB@?$AAM?$AAa?$AAp?$AAp?$AAi?$AAn?$AAg?$AA?5?$AA?$CF?$AAd?$AA?5?$AAt?$AAo?$AA?5?$AA?$CF?$AAd?$AA?$AN?$AA?6?$AA?$AA@ 10009448     fsl_serial_pdd_common_topaz_v1:serial_dl.obj
 0001:00008470       ??_C@_1EO@JLDEGKNA@?$AAE?$AAR?$AAR?$AAO?$AAR?$AA?3?$AA?5?$AAP?$AAD?$AAD?$AA?5?$AAc?$AAa?$AAn?$AAn?$AAo?$AAt?$AA?5?$AAs?$AAu?$AAp?$AAp?$AAo?$AAr?$AAt?$AA?5?$AAe?$AAn?$AAd?$AAp?$AAo?$AAi@ 10009470     fsl_serial_pdd_common_topaz_v1:serial_dl.obj
 0001:000084c0       ??_C@_0CJ@BBDJGCGB@Unexpected?5Msg?5in?5HandlePDDNotif@ 100094c0     fsl_serial_pdd_common_topaz_v1:serial_dl.obj
 0001:000084ec       ??_C@_1CO@ONOPPKFD@?$AAG?$AAo?$AAt?$AA?5?$AAS?$AAE?$AAT?$AAU?$AAP?$AA?5?$AAO?$AAU?$AAT?$AA?5?$AAp?$AAa?$AAc?$AAk?$AAe?$AAt?$AA?$AN?$AA?6?$AA?$AA@ 100094ec     fsl_serial_pdd_common_topaz_v1:serial_dl.obj
 0001:0000851c       ??_C@_0CI@BHALHJPB@Only?5GET_DESC?5and?5SET_CONFIG?5sup@ 1000951c     fsl_serial_pdd_common_topaz_v1:serial_dl.obj
 0001:00008548       ??_C@_1GM@JEDJFMFC@?$AAE?$AAR?$AAR?$AAO?$AAR?$AA?3?$AA?5?$AAO?$AAE?$AAM?$AAS?$AAe?$AAr?$AAi?$AAa?$AAl?$AAS?$AAe?$AAn?$AAd?$AAR?$AAa?$AAw?$AA?5?$AAc?$AAa?$AAl?$AAl?$AAe?$AAd?$AA?5?$AAb@ 10009548     fsl_serial_pdd_common_topaz_v1:serial_dl.obj
 0001:000085b4       ??_C@_0DB@LKOJLGG@Serial?5Wrapper?5Circular?5Buffer?5O@ 100095b4     fsl_serial_pdd_common_topaz_v1:serial_dl.obj
 0001:000085e8       ??_C@_0EA@FIJCBODK@Amount?5of?5transferred?5data?5in?5DW@ 100095e8     fsl_serial_pdd_common_topaz_v1:serial_dl.obj
 0001:00008628       ??_C@_1DO@JIIKDGOP@?$AAE?$AAx?$AAi?$AAt?$AAi?$AAn?$AAg?$AA?5?$AAO?$AAE?$AAM?$AAS?$AAe?$AAr?$AAi?$AAa?$AAl?$AAR?$AAe?$AAc?$AAv?$AAR?$AAa?$AAw?$AA?4?$AA?4?$AA?4?$AA?4?$AA?$AN?$AA?6?$AA?$AA@ 10009628     fsl_serial_pdd_common_topaz_v1:serial_dl.obj
 0001:00008668       ??_C@_1HA@FEDIMNNJ@?$AAM?$AAu?$AAs?$AAt?$AA?5?$AAi?$AAn?$AAc?$AAr?$AAe?$AAa?$AAs?$AAe?$AA?5?$AAR?$AAE?$AAC?$AAV?$AA_?$AAB?$AAU?$AAF?$AAF?$AAE?$AAR?$AA_?$AAS?$AAI?$AAZ?$AAE?$AA?5?$AAt@ 10009668     fsl_serial_pdd_common_topaz_v1:serial_dl.obj
 0001:000086d8       ??_C@_1GO@BNOBJNLF@?$AAE?$AAR?$AAR?$AAO?$AAR?$AA?3?$AA?5?$AAO?$AAE?$AAM?$AAS?$AAe?$AAr?$AAi?$AAa?$AAl?$AAR?$AAe?$AAc?$AAv?$AAR?$AAa?$AAw?$AA?5?$AAc?$AAa?$AAl?$AAl?$AAe?$AAr?$AA?5?$AAa@ 100096d8     fsl_serial_pdd_common_topaz_v1:serial_dl.obj
 0001:00008748       ??_C@_1GM@DFDLJAKN@?$AAE?$AAR?$AAR?$AAO?$AAR?$AA?3?$AA?5?$AAO?$AAE?$AAM?$AAS?$AAe?$AAr?$AAi?$AAa?$AAl?$AAR?$AAe?$AAc?$AAv?$AAR?$AAa?$AAw?$AA?5?$AAc?$AAa?$AAl?$AAl?$AAe?$AAd?$AA?5?$AAb@ 10009748     fsl_serial_pdd_common_topaz_v1:serial_dl.obj
 0001:000087b4       ??_C@_0DG@ODLBGEPM@ERROR?3?5OEMSerialRecvRaw?5called?5b@ 100097b4     fsl_serial_pdd_common_topaz_v1:serial_dl.obj
 0001:00008880       ??_C@_0CB@KKLHFGEJ@OALStall?3?5EPIT?5mapping?5failed?$CB?$AN?6@ 10009880     ethdrv:ethdrv.obj
 0001:000089ec       OALTimerGetClkSrc          100099ec f   kitl.obj
 0001:00008a04       OALTimerGetClkFreq         10009a04 f   kitl.obj
 0001:00008b18       OEMKitlStartup             10009b18 f   kitl.obj
 0001:00008eac       OALSerialInit              10009eac f   kitl.obj
 0001:00008f58       OEMKitlSerialInit          10009f58 f   kitl.obj
 0001:00008fb4       OALGetTickCount            10009fb4 f   kitl.obj
 0001:0000900c       OALClockSetGatingMode      1000a00c f   kitl.obj
 0001:000090d0       KITLSetDebug               1000a0d0 f   kitlcore:ethdbg.obj
 0001:00009104       IsDesktopDbgrExist         1000a104 f   kitlcore:ethdbg.obj
 0001:00009128       ChkDfltSvc                 1000a128 f   kitlcore:ethdbg.obj
 0001:000091b8       KITLRegisterDfltClient     1000a1b8 f   kitlcore:ethdbg.obj
 0001:00009464       KITLRegisterClient         1000a464 f   kitlcore:ethdbg.obj
 0001:0000a034       KITLDeregisterClient       1000b034 f   kitlcore:ethdbg.obj
 0001:0000a408       KITLInitializeInterrupt    1000b408 f   kitlcore:ethdbg.obj
 0001:0000a664       KITLWriteDebugString       1000b664 f   kitlcore:ethdbg.obj
 0001:0000acb0       ExtKITLIoctl               1000bcb0 f   kitlcore:ethdbg.obj
 0001:0000b338       KITLIoctl                  1000c338 f   kitlcore:ethdbg.obj
 0001:0000b714       KitlInit                   1000c714 f   kitlcore:ethdbg.obj
 0001:0000bbac       KitlDllMain                1000cbac f   kitlcore:ethdbg.obj
 0001:0000bcc0       GetObjPtr                  1000ccc0 f i kitlcore:ethdbg.obj
 0001:0000bd10       IsValidUsrPtr              1000cd10 f i kitlcore:ethdbg.obj
 0001:0000bd9c       KITLOutputDebugString      1000cd9c f   kitlcore:debug.obj
 0001:0000c2c8       inet_ntoa                  1000d2c8 f   kitlcore:debug.obj
 0001:0000c3b8       inet_addr                  1000d3b8 f   kitlcore:debug.obj
 0001:0000c4bc       DoDebugBreak               1000d4bc f   kitlcore:edbgprot.obj
 0001:0000c4c4       ResetClientState           1000d4c4 f   kitlcore:edbgprot.obj
 0001:0000c5e4       ExchangeConfig             1000d5e4 f   kitlcore:edbgprot.obj
 0001:0000c8e4       SendConfig                 1000d8e4 f   kitlcore:edbgprot.obj
 0001:0000cb48       KITLPollResponse           1000db48 f   kitlcore:edbgprot.obj
 0001:0000ce24       KITLSend                   1000de24 f   kitlcore:edbgprot.obj
 0001:0000dd50       RetransmitFrame            1000ed50 f   kitlcore:edbgprot.obj
 0001:0000e084       KITLRecv                   1000f084 f   kitlcore:edbgprot.obj
 0001:0000eb84       HandleRecvInterrupt        1000fb84 f   kitlcore:edbgprot.obj
 0001:000108e0       KitlSendRawData            100118e0 f   kitlcore:edbgprot.obj
 0001:000109e8       KitlSendFrame              100119e8 f   kitlcore:edbgprot.obj
 0001:00010a88       DumpTimerList              10011a88 f   kitlcore:timer.obj
 0001:00010af0       InitTimerList              10011af0 f   kitlcore:timer.obj
 0001:00010b84       FreeTimerEntry             10011b84 f   kitlcore:timer.obj
 0001:00010cbc       TimerCallback              10011cbc f   kitlcore:timer.obj
 0001:00010ebc       TimerThread                10011ebc f   kitlcore:timer.obj
 0001:00011448       TimerStart                 10012448 f   kitlcore:timer.obj
 0001:0001162c       TimerStop                  1001262c f   kitlcore:timer.obj
 0001:00011844       CancelTimersForClient      10012844 f   kitlcore:timer.obj
 0001:0001190c       KitlSetTimerCallback       1001290c f   kitlcore:timer.obj
 0001:000119f4       KitlStopTimerCallback      100129f4 f   kitlcore:timer.obj
 0001:00011a98       NKOutputDebugString        10012a98 f   nkstub:nkstub.obj
 0001:00011acc       NKvDbgPrintfW              10012acc f   nkstub:nkstub.obj
 0001:00011b04       NKDbgPrintfW               10012b04 f   nkstub:nkstub.obj
 0001:00011b58       NKwvsprintfW               10012b58 f   nkstub:nkstub.obj
 0001:00011bb0       NKSetLastError             10012bb0 f   nkstub:nkstub.obj
 0001:00011be4       NKGetLastError             10012be4 f   nkstub:nkstub.obj
 0001:00011c24       EnterCriticalSection       10012c24 f   nkstub:nkstub.obj
 0001:00011c58       LeaveCriticalSection       10012c58 f   nkstub:nkstub.obj
 0001:00011c8c       InitializeCriticalSection  10012c8c f   nkstub:nkstub.obj
 0001:00011cc0       DeleteCriticalSection      10012cc0 f   nkstub:nkstub.obj
 0001:00011cf4       INTERRUPTS_OFF             10012cf4 f   nkstub:nkstub.obj
 0001:00011d1c       INTERRUPTS_ON              10012d1c f   nkstub:nkstub.obj
 0001:00011d44       INTERRUPTS_ENABLE          10012d44 f   nkstub:nkstub.obj
 0001:00011d90       HookInterrupt              10012d90 f   nkstub:nkstub.obj
 0001:00011de0       UnhookInterrupt            10012de0 f   nkstub:nkstub.obj
 0001:00011e30       NKCallIntChain             10012e30 f   nkstub:nkstub.obj
 0001:00011e7c       NKIsSysIntrValid           10012e7c f   nkstub:nkstub.obj
 0001:00011ec8       NKSetInterruptEvent        10012ec8 f   nkstub:nkstub.obj
 0001:00011f14       NKSleep                    10012f14 f   nkstub:nkstub.obj
 0001:00011f48       NKVirtualSetAttributes     10012f48 f   nkstub:nkstub.obj
 0001:00011fa8       NKCreateStaticMapping      10012fa8 f   nkstub:nkstub.obj
 0001:00011ff8       NKDeleteStaticMapping      10012ff8 f   nkstub:nkstub.obj
 0001:00012048       NKRegCloseKey              10013048 f   nkstub:nkstub.obj
 0001:00012094       NKRegFlushKey              10013094 f   nkstub:nkstub.obj
 0001:000120e0       NKRegCreateKeyExW          100130e0 f   nkstub:nkstub.obj
 0001:00012160       NKRegOpenKeyExW            10013160 f   nkstub:nkstub.obj
 0001:000121c0       NKRegQueryValueExW         100131c0 f   nkstub:nkstub.obj
 0001:00012228       NKRegSetValueExW           10013228 f   nkstub:nkstub.obj
 0001:00012290       NKForceCleanBoot           10013290 f   nkstub:nkstub.obj
 0001:000122b8       NKReboot                   100132b8 f   nkstub:nkstub.obj
 0001:00012304       NKwcslen                   10013304 f   nkstub:nkstub.obj
 0001:00012350       NKwcscmp                   10013350 f   nkstub:nkstub.obj
 0001:000123a0       NKwcsicmp                  100133a0 f   nkstub:nkstub.obj
 0001:000123f0       NKwcsnicmp                 100133f0 f   nkstub:nkstub.obj
 0001:00012444       NKwcscpy                   10013444 f   nkstub:nkstub.obj
 0001:0001247c       NKwcsncpy                  1001347c f   nkstub:nkstub.obj
 0001:000124d0       NKstrcmpiAandW             100134d0 f   nkstub:nkstub.obj
 0001:00012520       NKUnicodeToAscii           10013520 f   nkstub:nkstub.obj
 0001:0001255c       NKAsciiToUnicode           1001355c f   nkstub:nkstub.obj
 0001:00012598       NKSystemTimeToFileTime     10013598 f   nkstub:nkstub.obj
 0001:000125e8       NKFileTimeToSystemTime     100135e8 f   nkstub:nkstub.obj
 0001:00012638       NKCompareFileTime          10013638 f   nkstub:nkstub.obj
 0001:00012690       ProfilerHit                10013690 f   nkstub:nkstub.obj
 0001:000126f4       ProfilerHitEx              100136f4 f   nkstub:nkstub.obj
 0001:00012728       GetEPC                     10013728 f   nkstub:nkstub.obj
 0001:00012768       NKPhysToVirt               10013768 f   nkstub:nkstub.obj
 0001:000127b8       NKVirtToPhys               100137b8 f   nkstub:nkstub.obj
 0001:00012804       __GetUserKData             10013804 f   nkstub:nkstub.obj
 0001:00012834       __report_gsfailure         10013834 f   nkstub:nkstub.obj
 0001:0001285c       GetOriginalDAbortHandlerAddress 1001385c f   nkstub:nkstub.obj
 0001:0001288c       NKSetDataAbortHandler      1001388c f   nkstub:nkstub.obj
 0001:00012918       OEMInitDebugSerial         10013918 f   oemstub:oemstub.obj
 0001:00012940       OEMInit                    10013940 f   oemstub:oemstub.obj
 0001:00012968       OEMWriteDebugByte          10013968 f   oemstub:oemstub.obj
 0001:0001299c       OEMWriteDebugString        1001399c f   oemstub:oemstub.obj
 0001:000129d0       OEMWriteDebugLED           100139d0 f   oemstub:oemstub.obj
 0001:00012a08       OEMReadDebugByte           10013a08 f   oemstub:oemstub.obj
 0001:00012a48       OEMCacheRangeFlush         10013a48 f   oemstub:oemstub.obj
 0001:00012a84       OEMInitClock               10013a84 f   oemstub:oemstub.obj
 0001:00012aac       OEMGetRealTime             10013aac f   oemstub:oemstub.obj
 0001:00012af8       OEMSetRealTime             10013af8 f   oemstub:oemstub.obj
 0001:00012b44       OEMSetAlarmTime            10013b44 f   oemstub:oemstub.obj
 0001:00012b90       OEMGetTickCount            10013b90 f   oemstub:oemstub.obj
 0001:00012bd0       OEMIdle                    10013bd0 f   oemstub:oemstub.obj
 0001:00012c04       OEMPowerOff                10013c04 f   oemstub:oemstub.obj
 0001:00012c2c       OEMGetExtensionDRAM        10013c2c f   oemstub:oemstub.obj
 0001:00012c7c       OEMInterruptDisable        10013c7c f   oemstub:oemstub.obj
 0001:00012cb0       OEMInterruptEnable         10013cb0 f   oemstub:oemstub.obj
 0001:00012d04       OEMInterruptDone           10013d04 f   oemstub:oemstub.obj
 0001:00012d38       OEMInterruptMask           10013d38 f   oemstub:oemstub.obj
 0001:00012d70       OEMNotifyIntrOccurs        10013d70 f   oemstub:oemstub.obj
 0001:00012dbc       OEMIoControl               10013dbc f   oemstub:oemstub.obj
 0001:00012ed8       OEMProfileTimerDisable     10013ed8 f   oemstub:oemstub.obj
 0001:00012f18       OEMProfileTimerEnable      10013f18 f   oemstub:oemstub.obj
 0001:00012f8c       OEMInterruptHandler        10013f8c f   oemstub:oemstub.obj
 0001:00012fd8       OEMInterruptHandlerFIQ     10013fd8 f   oemstub:oemstub.obj
 0001:00013000       OALKitlGetDevLoc           10014000 f   oal_kitl:kitl.obj
 0001:0001305c       OALKitlGetFlags            1001405c f   oal_kitl:kitl.obj
 0001:000130a8       OEMKitlInit                100140a8 f   oal_kitl:kitl.obj
 0001:00013224       OALKitlInit                10014224 f   oal_kitl:kitl.obj
 0001:00013778       OALKitlPowerOff            10014778 f   oal_kitl:kitl.obj
 0001:000138b8       OALKitlPowerOn             100148b8 f   oal_kitl:kitl.obj
 0001:000139e0       OALKitlCreateName          100149e0 f   oal_kitl:name.obj
 0001:00013c18       OEMKitlIoctl               10014c18 f   oal_kitl:kitlioctl.obj
 0001:00013c78       OALKitlSerialInit          10014c78 f   oal_kitl:kitlserial.obj
 0001:00014b04       DecodeIP                   10015b04 f   oal_kitl:kitleth.obj
 0001:00015f54       OALIoCtlVBridge            10016f54 f   oal_kitl:kitleth.obj
 0001:00016208       OALKitlEthInit             10017208 f   oal_kitl:kitleth.obj
 0001:00017a14       OALKitlFindDevice          10018a14 f   oal_kitl:device.obj
 0001:00017df8       OALKitlDeviceName          10018df8 f   oal_kitl:device.obj
 0001:00017f7c       OALKitlDeviceType          10018f7c f   oal_kitl:device.obj
 0001:00018100       OALKitlIPtoString          10019100 f   oal_kitl:format.obj
 0001:00018178       OALKitlMACtoString         10019178 f   oal_kitl:format.obj
 0001:00018224       OALKitlStringToIP          10019224 f   oal_kitl:format.obj
 0001:00018378       OALKitlStringToMAC         10019378 f   oal_kitl:format.obj
 0001:00018600       OALLogSerial               10019600 f   kitl_log:log.obj
 0001:0001865c       OALLogPrintf               1001965c f   kitl_log:log.obj
 0001:00018698       MIIREAD                    10019698 f   oal_ethdrv_fec_common_topaz_v1:fec.obj
 0001:000187ac       MIIWRITE                   100197ac f   oal_ethdrv_fec_common_topaz_v1:fec.obj
 0001:00018838       CalculateHashValue         10019838 f   oal_ethdrv_fec_common_topaz_v1:fec.obj
 0001:00018938       FECEnableInts              10019938 f   oal_ethdrv_fec_common_topaz_v1:fec.obj
 0001:000189e8       FECDisableInts             100199e8 f   oal_ethdrv_fec_common_topaz_v1:fec.obj
 0001:00018a98       FECInitDMABuffer           10019a98 f   oal_ethdrv_fec_common_topaz_v1:fec.obj
 0001:00018e78       FECInit                    10019e78 f   oal_ethdrv_fec_common_topaz_v1:fec.obj
 0001:0001995c       FECSendFrame               1001a95c f   oal_ethdrv_fec_common_topaz_v1:fec.obj
 0001:00019c14       FECGetFrame                1001ac14 f   oal_ethdrv_fec_common_topaz_v1:fec.obj
 0001:00019eac       FECCurrentPacketFilter     1001aeac f   oal_ethdrv_fec_common_topaz_v1:fec.obj
 0001:00019fe0       FECMulticastList           1001afe0 f   oal_ethdrv_fec_common_topaz_v1:fec.obj
 0001:0001a1e4       SerialInit                 1001b1e4 f   oal_kitlserial_common_topaz_v1:kitlserial.obj
 0001:0001a250       SerialDeinit               1001b250 f   oal_kitlserial_common_topaz_v1:kitlserial.obj
 0001:0001a254       SerialRecv                 1001b254 f   oal_kitlserial_common_topaz_v1:kitlserial.obj
 0001:0001a32c       SerialSend                 1001b32c f   oal_kitlserial_common_topaz_v1:kitlserial.obj
 0001:0001a3d0       SerialSendComplete         1001b3d0 f   oal_kitlserial_common_topaz_v1:kitlserial.obj
 0001:0001a3e4       SerialEnableInts           1001b3e4 f   oal_kitlserial_common_topaz_v1:kitlserial.obj
 0001:0001a3e8       SerialDisableInts          1001b3e8 f   oal_kitlserial_common_topaz_v1:kitlserial.obj
 0001:0001a3ec       SerialFlowControl          1001b3ec f   oal_kitlserial_common_topaz_v1:kitlserial.obj
 0001:0001a468       OALPAtoVA                  1001b468 f   oal_memory_arm:memory.obj
 0001:0001a590       OALVAtoPA                  1001b590 f   oal_memory_arm:memory.obj
 0001:0001a6c8       OALArgsQuery               1001b6c8 f   args:args.obj
 0001:0001aa04       OALConfigSerialUART        1001ba04 f   serialutils:serialutils.obj
 0001:0001ae48       OALConfigSerialIOMUX       1001be48 f   serialutils:serialutils.obj
 0001:0001af48       OALKitlGetFECDmaBuffer     1001bf48 f   bspfec:bspfec.obj
 0001:0001af64       OALKitlFECBSPInit          1001bf64 f   bspfec:bspfec.obj
 0001:0001b318       BSPFECusesRMII             1001c318 f   bspfec:bspfec.obj
 0001:0001b330       VBridgeDisplayHex          1001c330 f   vbridge:vbridge.obj
 0001:0001b36c       VBridgeDumpMemory          1001c36c f   vbridge:vbridge.obj
 0001:0001b428       ProduceBuffer              1001c428 f   vbridge:vbridge.obj
 0001:0001b68c       ProduceBufferDone          1001c68c f   vbridge:vbridge.obj
 0001:0001b6f4       ConsumeBuffer              1001c6f4 f   vbridge:vbridge.obj
 0001:0001b8d4       ConsumeBufferDone          1001c8d4 f   vbridge:vbridge.obj
 0001:0001b9ac       VBridgeInit                1001c9ac f   vbridge:vbridge.obj
 0001:0001bb14       VBridgeKGetOneTxBuffer     1001cb14 f   vbridge:vbridge.obj
 0001:0001bbc8       VBridgeKGetOneTxBufferComplete 1001cbc8 f   vbridge:vbridge.obj
 0001:0001bc1c       VBridgeKIndicateOneRxBuffer 1001cc1c f   vbridge:vbridge.obj
 0001:0001bd84       VBridgeKSetLocalMacAddress 1001cd84 f   vbridge:vbridge.obj
 0001:0001be3c       VBridgeUGetOneTxPacket     1001ce3c f   vbridge:vbridge.obj
 0001:0001bee0       VBridgeUGetOneTxPacketComplete 1001cee0 f   vbridge:vbridge.obj
 0001:0001bf38       VBridgeUGetOneRxPacket     1001cf38 f   vbridge:vbridge.obj
 0001:0001bfd4       VBridgeUGetOneRxPacketComplete 1001cfd4 f   vbridge:vbridge.obj
 0001:0001c02c       VBridgeUWildCard           1001d02c f   vbridge:vbridge.obj
 0001:0001c104       VBridgeUGetEDBGMac         1001d104 f   vbridge:vbridge.obj
 0001:0001c158       VBridgeUCurrentPacketFilter 1001d158 f   vbridge:vbridge.obj
 0001:0001c1b0       memset                     1001d1b0 f   fulllibc:memset.obj
 0001:0001c238       __GSHandlerCheck           1001d238 f   fulllibc:gshandler.obj
 0001:0001c280       __GSHandlerCheckCommon     1001d280 f   fulllibc:gshandler.obj
 0001:0001c328       __rt_udiv                  1001d328 f   fulllibc:__udiv.obj
 0001:0001c3ec       __security_check_cookie    1001d3ec f   fulllibc:armsecgs.obj
 0001:0001c400       __gsfailure                1001d400 f   fulllibc:armsecgs.obj
 0001:0001c444       strcmp                     1001d444 f   fulllibc:mdsstrcmp.obj
 0001:0001c534       strcpy                     1001d534 f   fulllibc:strcpy.obj
 0001:0001c5b8       strlen                     1001d5b8 f   fulllibc:mdsstrlen.obj
 0001:0001c61c       __rt_sdiv                  1001d61c f   fulllibc:__div.obj
 0001:0001c6f8       memcpy                     1001d6f8 f   fulllibc:memcpy.obj
 0001:0001caa4       memcpybigblk               1001daa4 f   fulllibc:memcpy.obj
 0001:0001d458       __GSHandlerCheck_SEH       1001e458 f   fulllibc:gshandlerseh.obj
 0001:0001d4e0       __C_specific_handler       1001e4e0 f   fulllibc:chandler.obj
 0001:0001d850       atol                       1001e850 f   fulllibc:atox.obj
 0001:0001da04       atoi                       1001ea04 f   fulllibc:atox.obj
 0001:0001da38       memcmp                     1001ea38 f   fulllibc:memcmp.obj
 0001:0001db04       __raise_int_divide_by_zero 1001eb04 f   fulllibc:diverr.obj
 0001:0001db28       __raise_int_overflow       1001eb28 f   fulllibc:diverr.obj
 0001:0001db4c       __C_ExecuteExceptionFilter 1001eb4c f   fulllibc:jmpuwind.obj
 0001:0001db4c       __C_ExecuteTerminationHandler 1001eb4c f   fulllibc:jmpuwind.obj
 0001:0001db8c       __crtRaiseException        1001eb8c f   fulllibc:raiseexc.obj
 0001:0001dbc0       RndisRestart               1001ebc0 f   fsl_rne_mdd_common_topaz_v1:rndis.obj
 0001:0001dc58       RndisPrepareRndisPacket    1001ec58 f   fsl_rne_mdd_common_topaz_v1:rndis.obj
 0001:0001ddcc       PDD_IsPacketSend           1001edcc f   fsl_rne_mdd_common_topaz_v1:rndis.obj
 0001:0001ddec       MddSendRndisPacketComplete 1001edec f   fsl_rne_mdd_common_topaz_v1:rndis.obj
 0001:0001de10       RndisEDbgSendFrame         1001ee10 f   fsl_rne_mdd_common_topaz_v1:rndis.obj
 0001:0001e028       MddSendRndisMessageComplete 1001f028 f   fsl_rne_mdd_common_topaz_v1:rndis.obj
 0001:0001e070       RndisSendRndisMessage      1001f070 f   fsl_rne_mdd_common_topaz_v1:rndis.obj
 0001:0001e554       RndisProcessMessage        1001f554 f   fsl_rne_mdd_common_topaz_v1:rndis.obj
 0001:0001ea6c       RndisEDbgGetFrame          1001fa6c f   fsl_rne_mdd_common_topaz_v1:rndis.obj
 0001:0001ec5c       RndisProcessPacket         1001fc5c f   fsl_rne_mdd_common_topaz_v1:rndis.obj
 0001:0001eecc       RndisInit                  1001fecc f   fsl_rne_mdd_common_topaz_v1:rndis.obj
 0001:0001f194       RndisGetIrq                10020194 f   fsl_rne_mdd_common_topaz_v1:rndis.obj
 0001:0001f1b4       RndisGetPCICard            100201b4 f   fsl_rne_mdd_common_topaz_v1:rndis.obj
 0001:0001f1f0       RndisDeInit                100201f0 f   fsl_rne_mdd_common_topaz_v1:rndis.obj
 0001:0001f1f4       RndisCurrentPacketFilter   100201f4 f   fsl_rne_mdd_common_topaz_v1:rndis.obj
 0001:0001f208       RndisMulticastList         10020208 f   fsl_rne_mdd_common_topaz_v1:rndis.obj
 0001:0001f230       RndisEnableInts            10020230 f   fsl_rne_mdd_common_topaz_v1:rndis.obj
 0001:0001f25c       RndisDisableInts           1002025c f   fsl_rne_mdd_common_topaz_v1:rndis.obj
 0001:0001f288       RndisSetOptions            10020288 f   fsl_rne_mdd_common_topaz_v1:rndis.obj
 0001:0001f2b0       MddInitializeCriticalSection 100202b0 f   fsl_rne_mdd_common_topaz_v1:rndis.obj
 0001:0001f2c4       MddDeleteCriticalSection   100202c4 f   fsl_rne_mdd_common_topaz_v1:rndis.obj
 0001:0001f2d8       MddEnterCriticalSection    100202d8 f   fsl_rne_mdd_common_topaz_v1:rndis.obj
 0001:0001f2ec       MddLeaveCriticalSection    100202ec f   fsl_rne_mdd_common_topaz_v1:rndis.obj
 0001:0001f300       RndisMiniCeLogMsg          10020300 f   fsl_rne_mdd_common_topaz_v1:rndis.obj
 0001:0001f314       HostMiniQueryInformation   10020314 f   fsl_rne_mdd_common_topaz_v1:hostmini.obj
 0001:0001f78c       HostMiniSetInformation     1002078c f   fsl_rne_mdd_common_topaz_v1:hostmini.obj
 0001:0001f994       MddIndicateRndisMessage    10020994 f   fsl_rne_mdd_common_topaz_v1:hostmini.obj
 0001:0001f9b0       MddIndicateRndisPacket     100209b0 f   fsl_rne_mdd_common_topaz_v1:hostmini.obj
 0001:0001f9dc       MDDAllocDataWrapper        100209dc f   fsl_rne_mdd_common_topaz_v1:hostmini.obj
 0001:0001fa58       MDDAllocMem                10020a58 f   fsl_rne_mdd_common_topaz_v1:hostmini.obj
 0001:0001fa74       MDDFreeMem                 10020a74 f   fsl_rne_mdd_common_topaz_v1:hostmini.obj
 0001:0001fa88       MDDFreeDataWrapper         10020a88 f   fsl_rne_mdd_common_topaz_v1:hostmini.obj
 0001:0001faac       MddDisconnect              10020aac f   fsl_rne_mdd_common_topaz_v1:hostmini.obj
 0001:0001facc       HostMiniInit               10020acc f   fsl_rne_mdd_common_topaz_v1:hostmini.obj
 0001:0001fb2c       HostMiniDeInit             10020b2c f   fsl_rne_mdd_common_topaz_v1:hostmini.obj
 0001:0001fb4c       InitBuffer                 10020b4c f   fsl_rne_mdd_common_topaz_v1:util.obj
 0001:0001fc4c       AvaiableBufferSize         10020c4c f   fsl_rne_mdd_common_topaz_v1:util.obj
 0001:0001fd2c       AllocBuffer                10020d2c f   fsl_rne_mdd_common_topaz_v1:util.obj
 0001:0001ffac       FreeBuffer                 10020fac f   fsl_rne_mdd_common_topaz_v1:util.obj
 0001:000202f4       GetFirstUsedBuffer         100212f4 f   fsl_rne_mdd_common_topaz_v1:util.obj
 0001:00020408       PDD_GetDescriptor          10021408 f   fsl_rne_pdd_common_topaz_v1:rndis_pdd.obj
 0001:00020788       PDD_DoVendorCommand        10021788 f   fsl_rne_pdd_common_topaz_v1:rndis_pdd.obj
 0001:00020b48       setupDataOutTransfer       10021b48 f   fsl_rne_pdd_common_topaz_v1:rndis_pdd.obj
 0001:00020cec       HandleSetupPacket          10021cec f   fsl_rne_pdd_common_topaz_v1:rndis_pdd.obj
 0001:00021188       TxComplete                 10022188 f   fsl_rne_pdd_common_topaz_v1:rndis_pdd.obj
 0001:00021260       NotifyHandler              10022260 f   fsl_rne_pdd_common_topaz_v1:rndis_pdd.obj
 0001:00021fc4       PDDInit                    10022fc4 f   fsl_rne_pdd_common_topaz_v1:rndis_pdd.obj
 0001:00022300       PDDDeinit                  10023300 f   fsl_rne_pdd_common_topaz_v1:rndis_pdd.obj
 0001:00022398       PDD_SendRndisMessage       10023398 f   fsl_rne_pdd_common_topaz_v1:rndis_pdd.obj
 0001:00022598       PDD_SendRndisPacket        10023598 f   fsl_rne_pdd_common_topaz_v1:rndis_pdd.obj
 0001:000227a0       PDD_Set                    100237a0 f   fsl_rne_pdd_common_topaz_v1:rndis_pdd.obj
 0001:00022acc       PDD_Get                    10023acc f   fsl_rne_pdd_common_topaz_v1:rndis_pdd.obj
 0001:00022d0c       PDD_ISR                    10023d0c f   fsl_rne_pdd_common_topaz_v1:rndis_pdd.obj
 0001:00022d44       PDD_IndicateRndisPacketComplete 10023d44 f   fsl_rne_pdd_common_topaz_v1:rndis_pdd.obj
 0001:00022dfc       SetRNDISMACAddress         10023dfc f   fsl_rne_pdd_common_topaz_v1:rndis_pdd.obj
 0001:00022e1c       SetRNDISSerialNumber       10023e1c f   fsl_rne_pdd_common_topaz_v1:rndis_pdd.obj
 0001:00022fa8       DescriptorPhy              10023fa8 f   usb_usbfn_mx25_topaz_v1:i_pdd.obj
 0001:00023000       DescriptorVirtual          10024000 f   usb_usbfn_mx25_topaz_v1:i_pdd.obj
 0001:00023058       ClearUsbstsUI              10024058 f   usb_usbfn_mx25_topaz_v1:i_pdd.obj
 0001:000230d8       UfnPdd_PowerDown           100240d8 f   usb_usbfn_mx25_topaz_v1:i_pdd.obj
 0001:0002380c       UfnPdd_PowerUp             1002480c f   usb_usbfn_mx25_topaz_v1:i_pdd.obj
 0001:00023d60       UpdateDevicePower          10024d60 f   usb_usbfn_mx25_topaz_v1:i_pdd.obj
 0001:0002406c       SetupEvent                 1002506c f   usb_usbfn_mx25_topaz_v1:i_pdd.obj
 0001:000247d4       DumpDeviceState            100257d4 f   usb_usbfn_mx25_topaz_v1:i_pdd.obj
 0001:00024c9c       DumpInterruptSource        10025c9c f   usb_usbfn_mx25_topaz_v1:i_pdd.obj
 0001:00024e38       CopyFromUncachedBuffer     10025e38 f   usb_usbfn_mx25_topaz_v1:i_pdd.obj
 0001:000250c8       CheckEndpoint              100260c8 f   usb_usbfn_mx25_topaz_v1:i_pdd.obj
 0001:00026654       InterruptHandle            10027654 f   usb_usbfn_mx25_topaz_v1:i_pdd.obj
 0001:00027b98       UfnPdd_IssueTransfer       10028b98 f   usb_usbfn_mx25_topaz_v1:i_pdd.obj
 0001:00029990       UfnPdd_AbortTransfer       1002a990 f   usb_usbfn_mx25_topaz_v1:i_pdd.obj
 0001:0002a068       UfnPdd_StallEndpoint       1002b068 f   usb_usbfn_mx25_topaz_v1:i_pdd.obj
 0001:0002a224       UfnPdd_ClearEndpointStall  1002b224 f   usb_usbfn_mx25_topaz_v1:i_pdd.obj
 0001:0002a428       UfnPdd_IsEndpointHalted    1002b428 f   usb_usbfn_mx25_topaz_v1:i_pdd.obj
 0001:0002a5f8       UfnPdd_SendControlStatusHandshake 1002b5f8 f   usb_usbfn_mx25_topaz_v1:i_pdd.obj
 0001:0002afc8       UfnPdd_InitiateRemoteWakeup 1002bfc8 f   usb_usbfn_mx25_topaz_v1:i_pdd.obj
 0001:0002b050       SetPowerState              1002c050 f   usb_usbfn_mx25_topaz_v1:i_pdd.obj
 0001:0002b40c       UfnPdd_IOControl           1002c40c f   usb_usbfn_mx25_topaz_v1:i_pdd.obj
 0001:0002b994       UfnPdd_Deinit              1002c994 f   usb_usbfn_mx25_topaz_v1:i_pdd.obj
 0001:0002b9c4       UfnPdd_DeregisterDevice    1002c9c4 f   usb_usbfn_mx25_topaz_v1:i_pdd.obj
 0001:0002b9ec       UfnPdd_Stop                1002c9ec f   usb_usbfn_mx25_topaz_v1:i_pdd.obj
 0001:0002bb1c       UfnPdd_DeinitEndpoint      1002cb1c f   usb_usbfn_mx25_topaz_v1:i_pdd.obj
 0001:0002bd78       UfnPdd_InitEndpoint        1002cd78 f   usb_usbfn_mx25_topaz_v1:i_pdd.obj
 0001:0002c200       UfnPdd_SetAddress          1002d200 f   usb_usbfn_mx25_topaz_v1:i_pdd.obj
 0001:0002c274       UfnPdd_Start               1002d274 f   usb_usbfn_mx25_topaz_v1:i_pdd.obj
 0001:0002cf58       UfnPdd_RegisterDevice      1002df58 f   usb_usbfn_mx25_topaz_v1:i_pdd.obj
 0001:0002d42c       UfnPdd_IsEndpointSupportable 1002e42c f   usb_usbfn_mx25_topaz_v1:i_pdd.obj
 0001:0002d4c8       UfnPdd_IsConfigurationSupportable 1002e4c8 f   usb_usbfn_mx25_topaz_v1:i_pdd.obj
 0001:0002d7f4       UfnPdd_Init                1002e7f4 f   usb_usbfn_mx25_topaz_v1:i_pdd.obj
 0001:0002e048       UfnPdd_DllEntry            1002f048 f   usb_usbfn_mx25_topaz_v1:i_pdd.obj
 0001:0002e070       FslUfnGetUsbFnPdd          1002f070 f   usb_usbfn_eboot_mx25_topaz_v1:i_stub.obj
 0001:0002e08c       FslUfnRequestIrq           1002f08c f   usb_usbfn_eboot_mx25_topaz_v1:i_stub.obj
 0001:0002e0b4       FslUfnIsUSBKitlEnable      1002f0b4 f   usb_usbfn_eboot_mx25_topaz_v1:i_stub.obj
 0001:0002e0cc       FslUfnCreateThread         1002f0cc f   usb_usbfn_eboot_mx25_topaz_v1:i_stub.obj
 0001:0002e0f4       UsbFnInterruptThread       1002f0f4 f   usb_usbfn_eboot_mx25_topaz_v1:i_stub.obj
 0001:0002e138       FslUfnTrigIrq              1002f138 f   usb_usbfn_eboot_mx25_topaz_v1:i_stub.obj
 0001:0002e154       FslUfnDeinit               1002f154 f   usb_usbfn_eboot_mx25_topaz_v1:i_stub.obj
 0001:0002e168       FslUfnGetDMABuffer         1002f168 f   usb_usbfn_eboot_mx25_topaz_v1:i_stub.obj
 0001:0002e294       BSPUSBClockSwitch          1002f294 f   usb_usbfn_eboot_mx25_topaz_v1:i_stub.obj
 0001:0002e2bc       BSPUSBClockCreateFileMapping 1002f2bc f   usb_usbfn_eboot_mx25_topaz_v1:i_stub.obj
 0001:0002e2d4       GetDeviceRegistryParams    1002f2d4 f   usb_usbfn_eboot_mx25_topaz_v1:i_stub.obj
 0001:0002e328       SetInterruptEvent          1002f328 f   usb_usbfn_eboot_mx25_topaz_v1:i_stub.obj
 0001:0002e35c       FslUfnGetPageNumber        1002f35c f   usb_usbfn_eboot_mx25_topaz_v1:i_stub.obj
 0001:0002e3a4       FslUfnGetPageSize          1002f3a4 f   usb_usbfn_eboot_mx25_topaz_v1:i_stub.obj
 0001:0002e3bc       FslUfnGetPageShift         1002f3bc f   usb_usbfn_eboot_mx25_topaz_v1:i_stub.obj
 0001:0002e3d4       FslInitializeCriticalSection 1002f3d4 f   usb_usbfn_eboot_mx25_topaz_v1:i_stub.obj
 0001:0002e3e8       FslEnterCriticalSection    1002f3e8 f   usb_usbfn_eboot_mx25_topaz_v1:i_stub.obj
 0001:0002e3fc       FslLeaveCriticalSection    1002f3fc f   usb_usbfn_eboot_mx25_topaz_v1:i_stub.obj
 0001:0002e410       LocalFree                  1002f410 f   usb_usbfn_eboot_mx25_topaz_v1:i_stub.obj
 0001:0002e438       CreateBusAccessHandle      1002f438 f   usb_usbfn_eboot_mx25_topaz_v1:i_stub.obj
 0001:0002e460       CloseBusAccessHandle       1002f460 f   usb_usbfn_eboot_mx25_topaz_v1:i_stub.obj
 0001:0002e474       CloseHandle                1002f474 f   usb_usbfn_eboot_mx25_topaz_v1:i_stub.obj
 0001:0002e49c       MmUnmapIoSpace             1002f49c f   usb_usbfn_eboot_mx25_topaz_v1:i_stub.obj
 0001:0002e4b0       CeLogData                  1002f4b0 f   usb_usbfn_eboot_mx25_topaz_v1:i_stub.obj
 0001:0002e4c4       InterruptInitialize        1002f4c4 f   usb_usbfn_eboot_mx25_topaz_v1:i_stub.obj
 0001:0002e4ec       InterruptDone              1002f4ec f   usb_usbfn_eboot_mx25_topaz_v1:i_stub.obj
 0001:0002e500       MmMapIoSpace               1002f500 f   usb_usbfn_eboot_mx25_topaz_v1:i_stub.obj
 0001:0002e53c       InterruptDisable           1002f53c f   usb_usbfn_eboot_mx25_topaz_v1:i_stub.obj
 0001:0002e550       CacheSync                  1002f550 f   usb_usbfn_eboot_mx25_topaz_v1:i_stub.obj
 0001:0002e56c       LockPages                  1002f56c f   usb_usbfn_eboot_mx25_topaz_v1:i_stub.obj
 0001:0002e5ac       GetLastError               1002f5ac f   usb_usbfn_eboot_mx25_topaz_v1:i_stub.obj
 0001:0002e5c4       UnlockPages                1002f5c4 f   usb_usbfn_eboot_mx25_topaz_v1:i_stub.obj
 0001:0002e5ec       CeOpenCallerBuffer         1002f5ec f   usb_usbfn_eboot_mx25_topaz_v1:i_stub.obj
 0001:0002e620       CeCloseCallerBuffer        1002f620 f   usb_usbfn_eboot_mx25_topaz_v1:i_stub.obj
 0001:0002e648       StringCchLengthW           1002f648 f   usb_usbfn_eboot_mx25_topaz_v1:i_stub.obj
 0001:0002e688       StringCchVPrintfW          1002f688 f   usb_usbfn_eboot_mx25_topaz_v1:i_stub.obj
 0001:0002e6b0       SetDevicePowerState        1002f6b0 f   usb_usbfn_eboot_mx25_topaz_v1:i_stub.obj
 0001:0002e6d8       Sleep                      1002f6d8 f   usb_usbfn_eboot_mx25_topaz_v1:i_stub.obj
 0001:0002e6f4       FslNKDbgPrintfW            1002f6f4 f   usb_usbfn_eboot_mx25_topaz_v1:i_stub.obj
 0001:0002e750       CacheRangeFlush            1002f750 f   usb_usbfn_eboot_mx25_topaz_v1:i_stub.obj
 0001:0002e800       ?HandleClassRequest@@YAXPAU_USB_DEVICE_REQUEST@@PAU_EP0_REQUEST@@@Z 1002f800 f   fsl_serial_pdd_common_topaz_v1:serial_dl.obj
 0001:0002e930       ?HandleGetDescriptor@@YAXPAU_USB_DEVICE_REQUEST@@PAU_EP0_REQUEST@@@Z 1002f930 f   fsl_serial_pdd_common_topaz_v1:serial_dl.obj
 0001:0002eb00       ?HandleTransferComplete@@YAXPAU_STransfer@@@Z 1002fb00 f   fsl_serial_pdd_common_topaz_v1:serial_dl.obj
 0001:0002ef94       USBSerialInit              1002ff94 f   fsl_serial_pdd_common_topaz_v1:serial_dl.obj
 0001:0002fd20       OEMSerialSendRaw           10030d20 f   fsl_serial_pdd_common_topaz_v1:serial_dl.obj
 0001:0002feec       OEMSerialRecvRaw           10030eec f   fsl_serial_pdd_common_topaz_v1:serial_dl.obj
 0001:000304a8       USBKitlSerialInit          100314a8 f   fsl_serial_pdd_common_topaz_v1:serial_dl.obj
 0001:000304e8       USBKitlSerialRecv          100314e8 f   fsl_serial_pdd_common_topaz_v1:serial_dl.obj
 0001:000306a4       USBKitlSerialSend          100316a4 f   fsl_serial_pdd_common_topaz_v1:serial_dl.obj
 0001:000306fc       USBKitlSerialEnableInts    100316fc f   fsl_serial_pdd_common_topaz_v1:serial_dl.obj
 0001:00030700       USBKitlSerialDisableInts   10031700 f   fsl_serial_pdd_common_topaz_v1:serial_dl.obj
 0001:00030704       OALFlushDCache             10031704 f   oal_cache_arm926:flushdc.obj
 0001:00030710       OALCleanDCache             10031710 f   oal_cache_arm926:cleandc.obj
 0001:0003071c       OALFlushDCacheLines        1003171c f   oal_cache_arm926:flushdclines.obj
 0001:0003073c       OALStall                   1003173c f   ethdrv:ethdrv.obj
 0001:000309c0       OEMKitlGetSecs             100319c0 f   ethdrv:ethdrv.obj
 0001:00030b88       memmove                    10031b88 f   fulllibc:memmove.obj
 0001:00031318       memmovebigblk              10032318 f   fulllibc:memmove.obj
 0001:00031db0       __rt_udivrem64by64         10032db0 f   fulllibc:mdsdiv64.obj
 0001:00031ea8       __rt_divrem64by64          10032ea8 f   fulllibc:mdsdiv64.obj
 0001:00031ef8       __rt_udiv64by64            10032ef8 f   fulllibc:mdsdiv64.obj
 0001:00031f08       __rt_urem64by64            10032f08 f   fulllibc:mdsdiv64.obj
 0001:00031f20       __rt_sdiv64by64            10032f20 f   fulllibc:mdsdiv64.obj
 0001:00031f30       __rt_srem64by64            10032f30 f   fulllibc:mdsdiv64.obj
 0001:00031f48       GetRNDISMACAddress         10032f48 f   fsl_usbfn_rndiskitl_mx25_topaz_v1:hwinit.obj
 0001:00031f94       controllerSetup            10032f94 f   fsl_usbfn_rndiskitl_mx25_topaz_v1:hwinit.obj
 0001:00032150       USBClockInit               10033150 f   fsl_usbfn_rndiskitl_mx25_topaz_v1:hwinit.obj
 0001:0003217c       HardwareInitialize         1003317c f   fsl_usbfn_rndiskitl_mx25_topaz_v1:hwinit.obj
 0001:000323b8       PowerDownSchemeExist       100333b8 f   fsl_usbfn_rndiskitl_mx25_topaz_v1:hwinit.obj
 0001:000323d0       BSPUsbXvrEnableVBUSIntr    100333d0 f   fsl_usbfn_rndiskitl_mx25_topaz_v1:hwinit.obj
 0001:00032450       BSPUsbResetPHY             10033450 f   fsl_usbfn_rndiskitl_mx25_topaz_v1:hwinit.obj
 0001:00032464       BSPUsbSetBusConfig         10033464 f   fsl_usbfn_rndiskitl_mx25_topaz_v1:hwinit.obj
 0001:000324a8       BSPUSBInterruptControl     100334a8 f   fsl_usbfn_rndiskitl_mx25_topaz_v1:hwinit.obj
 0001:000324bc       BSPPhyShowDevDiscon        100334bc f   fsl_usbfn_rndiskitl_mx25_topaz_v1:hwinit.obj
 0001:000324d4       BSPUsbSetCurrentLimitation 100334d4 f   fsl_usbfn_rndiskitl_mx25_topaz_v1:hwinit.obj
 0001:000324e8       FslUfnGetKitlDMABuffer     100334e8 f   fsl_usbfn_rndiskitl_mx25_topaz_v1:stub.obj
 0002:00000120       g_dwKITLThreadPriority     10034120     kitlcore:ethdbg.obj
 0002:00000124       g_dwKITLTimerThreadPriority 10034124     kitlcore:ethdbg.obj
 0002:00000128       __security_cookie          10034128     nkstub:nkstub.obj
 0002:0000012c       __security_cookie_complement 1003412c     nkstub:nkstub.obj
 0002:00000130       dpCurSettings              10034130     kitl_log:debug.obj
 0002:00000578       Am79c874Info               10034578     oal_ethdrv_fec_common_topaz_v1:fec.obj
 0002:0000077c       PhyInfo                    1003477c     oal_ethdrv_fec_common_topaz_v1:fec.obj
 0002:00000790       LAN8700Info                10034790     oal_ethdrv_fec_common_topaz_v1:fec.obj
 0002:00000998       Dp83640Info                10034998     oal_ethdrv_fec_common_topaz_v1:fec.obj
 0002:00000ba0       KSZ8041NLInfo              10034ba0     oal_ethdrv_fec_common_topaz_v1:fec.obj
 0002:00000da4       bRndisSendPacketEmpty      10034da4     fsl_rne_mdd_common_topaz_v1:rndis.obj
 0002:00000dd8       RNdisMddSupportedOids      10034dd8     fsl_rne_mdd_common_topaz_v1:hostmini.obj
 0002:00000e68       g_InterruptData            10034e68     fsl_rne_pdd_common_topaz_v1:rndis_pdd.obj
 0002:00001000       g_serial_rev_buf           10035000     fsl_rne_pdd_common_topaz_v1:buffer.obj
 0002:00001000       g_rndis_ep2_buf            10035000     fsl_rne_pdd_common_topaz_v1:buffer.obj
 0002:00003000       g_rndis_ep3_buf            10037000     fsl_rne_pdd_common_topaz_v1:buffer.obj
 0002:00003000       g_serial_send_buf          10037000     fsl_rne_pdd_common_topaz_v1:buffer.obj
 0002:00005000       g_rndis_ep0_buf            10039000     fsl_rne_pdd_common_topaz_v1:buffer.obj
 0002:0002ae04       dwCurrentPacketFilter      1005ee04     vbridge:vbridge.obj
 0002:0002ae08       bValidAddress              1005ee08     vbridge:vbridge.obj
 0002:0002ae0c       bWarnNoMacDone             1005ee0c     vbridge:vbridge.obj
 0002:0002ae10       g_bResetBuffer             1005ee10     vbridge:vbridge.obj
 0002:0002ae14       g_bUOpened                 1005ee14     vbridge:vbridge.obj
 0002:00034cf0       g_pEP3DataWrapper          10068cf0     fsl_rne_pdd_common_topaz_v1:rndis_pdd.obj
 0002:00034cf4       g_devState                 10068cf4     fsl_rne_pdd_common_topaz_v1:rndis_pdd.obj
 0002:00034cf8       g_EP0TransferState         10068cf8     fsl_rne_pdd_common_topaz_v1:rndis_pdd.obj
 0002:00034cfc       g_EP2TransferState         10068cfc     fsl_rne_pdd_common_topaz_v1:rndis_pdd.obj
 0002:00036088       ?g_mddInterface@@3U_UFN_MDD_INTERFACE_INFO@@A 1006a088     fsl_serial_pdd_common_topaz_v1:serial_dl.obj
 0002:00036090       ?g_EP1Transfer@@3U_STransfer@@A 1006a090     fsl_serial_pdd_common_topaz_v1:serial_dl.obj
 0002:000360b0       ?g_RecvBuffer@@3PAEA       1006a0b0     fsl_serial_pdd_common_topaz_v1:serial_dl.obj
 0002:000360d0       ?g_pddInterface@@3U_UFN_PDD_INTERFACE_INFO@@A 1006a0d0     fsl_serial_pdd_common_topaz_v1:serial_dl.obj
 0002:00036130       ?g_EP2Transfer@@3U_STransfer@@A 1006a130     fsl_serial_pdd_common_topaz_v1:serial_dl.obj
 0002:00036150       ?g_EP0Transfer@@3U_STransfer@@A 1006a150     fsl_serial_pdd_common_topaz_v1:serial_dl.obj
 0002:000361b4       ?g_DeviceState@@3W4DEVICE_STATE@@A 1006a1b4     fsl_serial_pdd_common_topaz_v1:serial_dl.obj
 0002:000361b8       ?g_EP0State@@3W4TRANSFER_STATE@@A 1006a1b8     fsl_serial_pdd_common_topaz_v1:serial_dl.obj
 0002:000361bc       ?g_EP1State@@3W4TRANSFER_STATE@@A 1006a1bc     fsl_serial_pdd_common_topaz_v1:serial_dl.obj
 0002:000361c0       ?g_EP2State@@3W4TRANSFER_STATE@@A 1006a1c0     fsl_serial_pdd_common_topaz_v1:serial_dl.obj
 0002:000361c4       ?g_RecvBufferHead@@3GA     1006a1c4     fsl_serial_pdd_common_topaz_v1:serial_dl.obj
 0002:000361c8       ?g_RecvBufferTail@@3GA     1006a1c8     fsl_serial_pdd_common_topaz_v1:serial_dl.obj
 0002:00036200       preallocent                1006a200     <common>
 0002:00036494       g_KitlInterval             1006a494     <common>
 0002:00036498       g_pprcNK                   1006a498     <common>
 0002:000364a0       DfltClnts                  1006a4a0     <common>
 0002:00036640       g_kpriv                    1006a640     <common>
 0002:000366a0       TimerListCS                1006a6a0     <common>
 0002:000366b4       KITLGlobalState            1006a6b4     <common>
 0002:000366c0       SendFmtBuf                 1006a6c0     <common>
 0002:00036cc0       KITLcs                     1006acc0     <common>
 0002:00036cd4       g_pKData                   1006acd4     <common>
 0002:00036ce0       KITLODScs                  1006ace0     <common>
 0002:00036d00       KITLKCallcs                1006ad00     <common>
 0002:00036d20       Kitl                       1006ad20     <common>
 0002:00036d80       KITLClients                1006ad80     <common>
 0002:00036f80       g_oalCacheInfo             1006af80     <common>
 0002:00036fc8       g_pNKGlobal                1006afc8     <common>
 0002:00036fcc       g_pOemGlobal               1006afcc     <common>
 0002:00036fe0       g_oalKitlBuffer            1006afe0     <common>
 0002:00046fe0       g_UUID                     1007afe0     <common>
 0002:00046ff0       g_pBSPArgs                 1007aff0     <common>
 0002:00046ff4       pucRxMax                   1007aff4     <common>
 0002:00046ff8       pucTxConsumer              1007aff8     <common>
 0002:00046ffc       pucTxMin                   1007affc     <common>
 0002:00047000       TxBuffers                  1007b000     <common>
 0002:0004b004       pucRxProducer              1007f004     <common>
 0002:0004b008       EDBGMacAddress             1007f008     <common>
 0002:0004b010       pucTxMax                   1007f010     <common>
 0002:0004b014       pucRxMin                   1007f014     <common>
 0002:0004b018       pucTxProducer              1007f018     <common>
 0002:0004b01c       pucRxConsumer              1007f01c     <common>
 0002:0004b020       RxBuffers                  1007f020     <common>
 0002:0004f040       RndisMdd                   10083040     <common>
 0002:0004f110       g_EP0DataWrapper           10083110     <common>
 0002:0004f120       MDDZONE5                   10083120     <common>
 0002:0004f128       g_mddInterface             10083128     <common>
 0002:0004f140       g_EP1Transfer              10083140     <common>
 0002:0004f160       g_RndisKitlDev             10083160     <common>
 0002:0004f5a4       pUsbDevReg                 100835a4     <common>
 0002:0004f5a8       g_udr                      100835a8     <common>
 0002:0004f5b0       MDDZONE4                   100835b0     <common>
 0002:0004f5b4       PDDZONE                    100835b4     <common>
 0002:0004f5c0       g_EP3Transfer              100835c0     <common>
 0002:0004f5e0       g_pddInterface             100835e0     <common>
 0002:0004f640       MDDZONE3                   10083640     <common>
 0002:0004f660       g_EP2Transfer              10083660     <common>
 0002:0004f680       PDDZONE0                   10083680     <common>
 0002:0004f6a0       g_EP0Transfer              100836a0     <common>
 0002:0004f6c0       MDDZONE0                   100836c0     <common>
 0002:0004f6c4       MDDZONE                    100836c4     <common>
 0002:0004f6c8       MDDZONE2                   100836c8     <common>
 0002:0004f6e0       g_csRegister               100836e0     <common>

 entry point at        0001:0000bbac

 Static symbols

 0001:000095fc       DoRegisterClient           1000a5fc f   kitlcore:ethdbg.obj
 0001:00009a20       NewClient                  1000aa20 f   kitlcore:ethdbg.obj
 0001:00009c6c       RegisterClientPart2        1000ac6c f   kitlcore:ethdbg.obj
 0001:0000a7c0       StartKitl                  1000b7c0 f   kitlcore:ethdbg.obj
 0001:0000aa4c       KITLConnectToDesktop       1000ba4c f   kitlcore:ethdbg.obj
 0001:0000ac24       ChkCnxDsktp                1000bc24 f   kitlcore:ethdbg.obj
 0001:0000ac58       TranCnxDsktp               1000bc58 f   kitlcore:ethdbg.obj
 0001:0000b210       MemCopyToUserPtr           1000c210 f   kitlcore:ethdbg.obj
 0001:0000b258       MemCopyUserPtr             1000c258 f   kitlcore:ethdbg.obj
 0001:0000b2f8       MemCopyFromUserPtr         1000c2f8 f   kitlcore:ethdbg.obj
 0001:0000b7a8       EnableInts                 1000c7a8 f   kitlcore:ethdbg.obj
 0001:0000b83c       KITLInterruptThread        1000c83c f   kitlcore:ethdbg.obj
 0001:0000be7c       vOutputFormatString        1000ce7c f   kitlcore:debug.obj
 0001:0000c118       pOutputByte                1000d118 f   kitlcore:debug.obj
 0001:0000c178       pOutputNumHex              1000d178 f   kitlcore:debug.obj
 0001:0000c210       pOutputNumDecimal          1000d210 f   kitlcore:debug.obj
 0001:0000c260       OutputString               1000d260 f   kitlcore:debug.obj
 0001:0000c338       FormatString               1000d338 f   kitlcore:debug.obj
 0001:0000c854       CheckCfg                   1000d854 f   kitlcore:edbgprot.obj
 0001:0000c8a4       RetransmitCfg              1000d8a4 f   kitlcore:edbgprot.obj
 0001:0000cd60       KITLPollData               1000dd60 f   kitlcore:edbgprot.obj
 0001:0000dc4c       ChkAck                     1000ec4c f   kitlcore:edbgprot.obj
 0001:0000dcac       TranAck                    1000ecac f   kitlcore:edbgprot.obj
 0001:0000e9bc       SendAckNack                1000f9bc f   kitlcore:edbgprot.obj
 0001:0000ec9c       ProcessRecvFrame           1000fc9c f   kitlcore:edbgprot.obj
 0001:0000fce8       ProcessAdminMsg            10010ce8 f   kitlcore:edbgprot.obj
 0001:00010464       KITLDecodeFrame            10011464 f   kitlcore:edbgprot.obj
 0001:000112a8       TimerListInsert            100122a8 f   kitlcore:timer.obj
 0001:00014148       SerialSend                 10015148 f   oal_kitl:kitlserial.obj
 0001:000142dc       SerialRecv                 100152dc f   oal_kitl:kitlserial.obj
 0001:000148d4       ChkSum                     100158d4 f   oal_kitl:kitlserial.obj
 0001:00014950       SerialEncode               10015950 f   oal_kitl:kitlserial.obj
 0001:00014a00       SerialDecode               10015a00 f   oal_kitl:kitlserial.obj
 0001:00014a50       SerialEnableInt            10015a50 f   oal_kitl:kitlserial.obj
 0001:00014aa8       SerialGetDevCfg            10015aa8 f   oal_kitl:kitlserial.obj
 0001:00014adc       SerialSetHostCfg           10015adc f   oal_kitl:kitlserial.obj
 0001:00014c90       Sum                        10015c90 f   oal_kitl:kitleth.obj
 0001:00014d64       DecodeICMP                 10015d64 f   oal_kitl:kitleth.obj
 0001:00014f68       EncodeIP                   10015f68 f   oal_kitl:kitleth.obj
 0001:000151a4       DecodeUDP                  100161a4 f   oal_kitl:kitleth.obj
 0001:000155b0       DecodeDHCP                 100165b0 f   oal_kitl:kitleth.obj
 0001:000158a4       FindDHCPOption             100168a4 f   oal_kitl:kitleth.obj
 0001:00015944       SendDHCP                   10016944 f   oal_kitl:kitleth.obj
 0001:00015c90       EncodeUDP                  10016c90 f   oal_kitl:kitleth.obj
 0001:00015e18       AddDHCPOption              10016e18 f   oal_kitl:kitleth.obj
 0001:00015ecc       RenewDHCP                  10016ecc f   oal_kitl:kitleth.obj
 0001:00016968       GetAddressDHCP             10017968 f   oal_kitl:kitleth.obj
 0001:00016cf8       SendARP                    10017cf8 f   oal_kitl:kitleth.obj
 0001:00016ea4       GetOpARP                   10017ea4 f   oal_kitl:kitleth.obj
 0001:00016f70       KitlEthDecode              10017f70 f   oal_kitl:kitleth.obj
 0001:00017118       DecodeARP                  10018118 f   oal_kitl:kitleth.obj
 0001:00017210       KitlEthEncode              10018210 f   oal_kitl:kitleth.obj
 0001:000172e8       KitlEthGetFrameHdrSize     100182e8 f   oal_kitl:kitleth.obj
 0001:00017300       KitlEthSetHostCfg          10018300 f   oal_kitl:kitleth.obj
 0001:00017328       KitlEthGetDevCfg           10018328 f   oal_kitl:kitleth.obj
 0001:000174b8       KitlEthSend                100184b8 f   oal_kitl:kitleth.obj
 0001:00017730       KitlEthRecv                10018730 f   oal_kitl:kitleth.obj
 0001:0001794c       KitlEthEnableInt           1001894c f   oal_kitl:kitleth.obj
 0001:0001d980       isspace                    1001e980 f   fulllibc:atox.obj
 0001:00020a2c       PDD_SendNotification       10021a2c f   fsl_rne_pdd_common_topaz_v1:rndis_pdd.obj
 0001:00020aac       PDD_RecvNotification       10021aac f   fsl_rne_pdd_common_topaz_v1:rndis_pdd.obj
 0001:00021cd4       RegisterUSBDevice          10022cd4 f   fsl_rne_pdd_common_topaz_v1:rndis_pdd.obj
 0001:000229fc       PDD_DiscardPendingMessages 100239fc f   fsl_rne_pdd_common_topaz_v1:rndis_pdd.obj
 0001:00023730       CeLogMsg                   10024730 f   usb_usbfn_mx25_topaz_v1:i_pdd.obj
 0001:000243a8       GetSetupPacket             100253a8 f   usb_usbfn_mx25_topaz_v1:i_pdd.obj
 0001:000272b0       HandleUSBReset             100282b0 f   usb_usbfn_mx25_topaz_v1:i_pdd.obj
 0001:000277b0       DevStatEvent               100287b0 f   usb_usbfn_mx25_topaz_v1:i_pdd.obj
 0001:00027878       USBControllerRun           10028878 f   usb_usbfn_mx25_topaz_v1:i_pdd.obj
 0001:000291ac       BuildTdBufferList          1002a1ac f   usb_usbfn_mx25_topaz_v1:i_pdd.obj
 0001:00029efc       FlushEndpoint              1002aefc f   usb_usbfn_mx25_topaz_v1:i_pdd.obj
 0001:0002a784       PrimeQh0ForZeroTransfer    1002b784 f   usb_usbfn_mx25_topaz_v1:i_pdd.obj
 0001:0002b1a4       SetDeviceTestMode          1002c1a4 f   usb_usbfn_mx25_topaz_v1:i_pdd.obj
 0001:0002c520       InitQh0                    1002d520 f   usb_usbfn_mx25_topaz_v1:i_pdd.obj
 0001:0002d76c       Log2                       1002e76c f   usb_usbfn_mx25_topaz_v1:i_pdd.obj
 0001:0002f138       ?HandleUSBDeviceRegistration@@YAXXZ 10030138 f   fsl_serial_pdd_common_topaz_v1:serial_dl.obj
 0001:0002f718       ?HandlePDDNotification@@YAHPAXKK@Z 10030718 f   fsl_serial_pdd_common_topaz_v1:serial_dl.obj
 0001:0002fad8       ?HandleSetupPkt@@YAXPAU_USB_DEVICE_REQUEST@@PAU_EP0_REQUEST@@@Z 10030ad8 f   fsl_serial_pdd_common_topaz_v1:serial_dl.obj
 0001:00032214       InitializeMux              10033214 f   fsl_usbfn_rndiskitl_mx25_topaz_v1:hwinit.obj
 0001:0003222c       InitializeTransceiver      1003322c f   fsl_usbfn_rndiskitl_mx25_topaz_v1:hwinit.obj
